:020000040800F2
:1000000000000120C1520008ED250008EF2500087E
:10001000F1250008F3250008F52500080000000080
:10002000000000000000000000000000F7250008AC
:10003000F925000800000000FB250008FD25000848
:100040001153000811530008115300081153000800
:1000500011530008115300081153000811530008F0
:1000600011530008115300081153000811530008E0
:1000700011530008115300081153000811530008D0
:10008000115300081153000811530008000000002C
:1000900000000000000000000000000011530008F4
:1000A00011530008115300081153000811530008A0
:1000B0001153000811530008115300081153000890
:1000C0001153000811530008115300081153000880
:1000D00011530008DD380008F9380008000000005E
:1000E00011530008115300081153000800000000CC
:1000F0000000000000000000000000001153000894
:1001000000000000115300081153000811530008AB
:1001100000000000000000000000000000000000DF
:10012000115300081153000811530008115300081F
:100130001153000800000000000000000000000053
:100140000000000000000000000000001153000843
:100150001153000811530008115300081539000805
:1001600011530008115300080000000000000000B7
:10017000000000000000000000000000000000007F
:100180000000000011530008000000000000000003
:0401900011530008FF
:1001C00010B5054C237833B9044B13B10448AFF391
:1001D00000800123237010BDB81100200000000032
:1001E0004CC9000808B5034B1BB103490348AFF3E2
:1001F000008008BD00000000BC1100204CC90008B0
:1002000081F0004102E000BF83F0004330B54FEAC7
:1002100041044FEA430594EA050F08BF90EA020F34
:100220001FBF54EA000C55EA020C7FEA645C7FEAC7
:10023000655C00F0E2804FEA5454D4EB5555B8BFEA
:100240006D420CDD2C4480EA020281EA030382EA5B
:10025000000083EA010180EA020281EA0303362DED
:1002600088BF30BD11F0004F4FEA01314FF4801CC0
:100270004CEA113102D0404261EB410113F0004FD2
:100280004FEA03334CEA133302D0524263EB430389
:1002900094EA050F00F0A780A4F10104D5F1200E27
:1002A0000DDB02FA0EFC22FA05F2801841F1000182
:1002B00003FA0EF2801843FA05F359410EE0A5F156
:1002C00020050EF1200E012A03FA0EFC28BF4CF087
:1002D000020C43FA05F3C01851EBE37101F000453D
:1002E00007D54FF0000EDCF1000C7EEB00006EEB4A
:1002F0000101B1F5801F1BD3B1F5001F0CD34908D4
:100300005FEA30004FEA3C0C04F101044FEA44522A
:1003100012F5800F80F09A80BCF1004F08BF5FEAB1
:10032000500C50F1000041EB045141EA050130BD91
:100330005FEA4C0C404141EB010111F4801FA4F134
:100340000104E9D191F0000F04BF01460020B1FA89
:1003500081F308BF2033A3F10B03B3F120020CDAC1
:100360000C3208DD02F1140CC2F10C0201FA0CF09F
:1003700021FA02F10CE002F11402D8BFC2F1200C04
:1003800001FA02F120FA0CFCDCBF41EA0C019040BA
:10039000E41AA2BF01EB0451294330BD6FEA040403
:1003A0001F3C1CDA0C340EDC04F11404C4F12002EE
:1003B00020FA04F001FA02F340EA030021FA04F300
:1003C00045EA030130BDC4F10C04C4F1200220FA57
:1003D00002F001FA04F340EA0300294630BD21FA95
:1003E00004F0294630BD94F0000F83F4801306BF5B
:1003F00081F480110134013D4EE77FEA645C18BF4F
:100400007FEA655C29D094EA050F08BF90EA020FE5
:1004100005D054EA000C04BF1946104630BD91EADD
:10042000030F1EBF0021002030BD5FEA545C05D1E0
:100430004000494128BF41F0004130BD14F580041F
:100440003CBF01F5801130BD01F0004545F0FE4193
:1004500041F470014FF0000030BD7FEA645C1ABFC8
:10046000194610467FEA655C1CBF0B46024650EAFF
:10047000013406BF52EA033591EA030F41F400212B
:1004800030BD00BF90F0000F04BF0021704730B5B1
:100490004FF4806404F132044FF000054FF0000186
:1004A00050E700BF90F0000F04BF0021704730B547
:1004B0004FF4806404F1320410F0004548BF40421C
:1004C0004FF000013EE700BF42004FEAE2014FEA71
:1004D00031014FEA02701FBF12F07F4393F07F4F4C
:1004E00081F06051704732F07F4208BF704793F04F
:1004F0007F4F04BF41F40021704730B54FF4607462
:1005000001F0004521F000411CE700BF50EA010264
:1005100008BF704730B54FF000050AE050EA01020D
:1005200008BF704730B511F0004502D5404261EB7D
:1005300041014FF4806404F132045FEA915C3FF4BE
:10054000D8AE4FF003025FEADC0C18BF03325FEA5B
:10055000DC0C18BF033202EBDC02C2F1200300FA0C
:1005600003FC20FA02F001FA03FE40EA0E0021FA31
:1005700002F11444BDE600BF70B54FF0FF0C4CF41F
:10058000E06C1CEA11541DBF1CEA135594EA0C0FD1
:1005900095EA0C0F00F0DEF82C4481EA030621EA0C
:1005A0004C5123EA4C5350EA013518BF52EA033547
:1005B00041F4801143F4801338D0A0FB02CE4FF0F9
:1005C0000005E1FB02E506F00042E0FB03E54FF029
:1005D0000006E1FB03569CF0000F18BF4EF0010E21
:1005E000A4F1FF04B6F5007F64F5407404D25FEA1D
:1005F0004E0E6D4146EB060642EAC62141EA5551D0
:100600004FEAC52040EA5E504FEACE2EB4F1FD0C11
:1006100088BFBCF5E06F1ED8BEF1004F08BF5FEA8F
:10062000500E50F1000041EB045170BD06F0004641
:1006300046EA010140EA020081EA0301B4EB5C04EE
:10064000C2BFD4EB0C0541EA045170BD41F48011E6
:100650004FF0000E013C00F3AB8014F1360FDEBF0B
:10066000002001F0004170BDC4F10004203C35DAE7
:100670000C341BDC04F11404C4F1200500FA05F36A
:1006800020FA04F001FA05F240EA020001F000420B
:1006900021F0004110EBD37021FA04F642EB060181
:1006A0005EEA430E08BF20EAD37070BDC4F10C04AB
:1006B000C4F1200500FA04F320FA05F001FA04F26F
:1006C00040EA020001F0004110EBD37041F100015B
:1006D0005EEA430E08BF20EAD37070BDC4F1200566
:1006E00000FA05F24EEA020E20FA04F301FA05F2CE
:1006F00043EA020321FA04F001F0004121FA04F276
:1007000020EA020000EBD3705EEA430E08BF20EA45
:10071000D37070BD94F0000F0FD101F0004640007F
:1007200041EB010111F4801F08BF013CF7D041EA01
:10073000060195F0000F18BF704703F00046520005
:1007400043EB030313F4801F08BF013DF7D043EAD6
:100750000603704794EA0C0F0CEA135518BF95EA8C
:100760000C0F0CD050EA410618BF52EA4306D1D113
:1007700081EA030101F000414FF0000070BD50EA32
:10078000410606BF1046194652EA430619D094EABC
:100790000C0F02D150EA013613D195EA0C0F05D1A6
:1007A00052EA03361CBF104619460AD181EA0301FA
:1007B00001F0004141F0FE4141F470014FF00000B2
:1007C00070BD41F0FE4141F4780170BD70B54FF04D
:1007D000FF0C4CF4E06C1CEA11541DBF1CEA1355CD
:1007E00094EA0C0F95EA0C0F00F0A7F8A4EB0504AF
:1007F00081EA030E52EA03354FEA013100F08880A6
:100800004FEA03334FF0805545EA131343EA12636E
:100810004FEA022245EA111545EA10654FEA002623
:100820000EF000419D4208BF964244F1FD0404F5DC
:10083000407402D25B084FEA3202B61A65EB030538
:100840005B084FEA32024FF480104FF4002CB6EBF5
:10085000020E75EB030E22BFB61A754640EA0C0075
:100860005B084FEA3202B6EB020E75EB030E22BFB5
:10087000B61A754640EA5C005B084FEA3202B6EBF6
:10088000020E75EB030E22BFB61A754640EA9C00B5
:100890005B084FEA3202B6EB020E75EB030E22BF85
:1008A000B61A754640EADC0055EA060E18D04FEA43
:1008B000051545EA16754FEA06164FEAC30343EAE3
:1008C00052734FEAC2025FEA1C1CC0D111F4801FB0
:1008D0000BD141EA00014FF000004FF0004CB6E7A9
:1008E00011F4801F04BF01430020B4F1FD0C88BF48
:1008F000BCF5E06F3FF6AFAEB5EB030C04BFB6EB53
:10090000020C5FEA500C50F1000041EB045170BD45
:100910000EF0004E4EEA113114EB5C04C2BFD4EB72
:100920000C0541EA045170BD41F480114FF0000EF6
:10093000013C90E645EA060E8DE60CEA135594EA72
:100940000C0F08BF95EA0C0F3FF43BAF94EA0C0F75
:100950000AD150EA01347FF434AF95EA0C0F7FF4EA
:1009600025AF104619462CE795EA0C0F06D152EA3E
:1009700003353FF4FDAE1046194622E750EA410622
:1009800018BF52EA43067FF4C5AE50EA41047FF433
:100990000DAF52EA43057FF4EBAE12E74FF0FF3C98
:1009A00006E000BF4FF0010C02E000BF4FF0010C69
:1009B0004DF804CD4FEA410C7FEA6C5C4FEA430CE2
:1009C00018BF7FEA6C5C1BD001B050EA410C0CBF31
:1009D00052EA430C91EA030F02BF90EA020F002093
:1009E000704710F1000F91EA030F58BF994208BFFA
:1009F00090422CBFD8176FEAE37040F001007047B7
:100A00004FEA410C7FEA6C5C02D150EA013C07D10D
:100A10004FEA430C7FEA6C5CD6D152EA033CD3D058
:100A20005DF8040B704700BF8446104662468C4652
:100A30001946634600E000BF01B5FFF7B7FF002885
:100A400048BF10F1000F01BD4DF808EDFFF7F4FFAE
:100A50000CBF012000205DF808FB00BF4DF808ED39
:100A6000FFF7EAFF34BF012000205DF808FB00BF5C
:100A70004DF808EDFFF7E0FF94BF012000205DF87E
:100A800008FB00BF4DF808EDFFF7CEFF94BF012033
:100A900000205DF808FB00BF4DF808EDFFF7C4FF2C
:100AA00034BF012000205DF808FB00BF53B94AB9EC
:100AB000002908BF00281CBF4FF0FF314FF0FF3066
:100AC00000F072B9ADF1080C6DE904CE00F006F843
:100AD000DDF804E0DDE9022304B070472DE9F047BA
:100AE000089E04468846002B4BD18A42154667D99A
:100AF000B2FA82F24AB1C2F1200701FA02F320FAF7
:100B000007F7954047EA030894404FEA154E230C37
:100B1000B8FBFEF71FFA85FC0EFB178843EA084373
:100B200007FB0CF1994209D9EB1807F1FF3080F06F
:100B30001B81994240F21881023F2B445B1AA4B2F8
:100B4000B3FBFEF00EFB103344EA034400FB0CFC45
:100B5000A44509D92C1900F1FF3380F00781A44581
:100B600040F2048102382C4440EA0740A4EB0C0414
:100B700000271EB1D4400023C6E900433946BDE832
:100B8000F0878B4209D9002E00F0EB800027C6E9E0
:100B9000000138463946BDE8F087B3FA83F7002FE5
:100BA00047D18B4202D3824200F2FA80841A61EB71
:100BB000030301209846002EE0D0C6E90048DDE797
:100BC00002B9FFDEB2FA82F2002A40F08F80491BA0
:100BD0004FEA154E1FFA85F80127B1FBFEFC230CE6
:100BE0000EFB1C1143EA014308FB0CF1994207D9A3
:100BF000EB180CF1FF3002D2994200F2CD8084460E
:100C0000591AA3B2B1FBFEF00EFB101443EA0444E0
:100C100008FB00F8A04507D92C1900F1FF3302D2D8
:100C2000A04500F2B6801846A4EB080440EA0C4048
:100C30009FE7C7F1200CBB4022FA0CFE4EEA030EE0
:100C400001FA07F420FA0CF521FA0CF34FEA1E48DA
:100C50002543B3FBF8F92C0C08FB19331FFA8EFA65
:100C600044EA034309FB0AF49C4202FA07F200FA41
:100C700007F10BD91EEB030309F1FF3080F08780E9
:100C80009C4240F28480A9F1020973441B1BADB25F
:100C9000B3FBF8F008FB103345EA034400FB0AFA03
:100CA000A24508D91EEB040400F1FF336BD2A24524
:100CB00069D90238744440EA0940A0FB0289A4EBD8
:100CC0000A044C45C2464B4654D351D0002E69D03D
:100CD000B1EB0A0564EB030404FA0CFCFD40FC4094
:100CE0004CEA0505C6E90054002747E7C2F1200396
:100CF00020FA03F7954001FA02F021FA03F34FEAD4
:100D0000154E3843010CB3FBFEF71FFA85F80EFBB6
:100D1000173341EA034107FB08F38B4204FA02F45C
:100D200007D9691807F1FF3C2FD28B422DD9023F1A
:100D30002944CB1A81B2B3FBFEF00EFB103341EA1B
:100D4000034100FB08F38B4207D9691800F1FF3C0F
:100D500017D28B4215D902382944C91A40EA0747ED
:100D60003BE73746304609E70746E7E61846FBE625
:100D70004145ABD2B8EB020A69EB0E0201381346CB
:100D8000A4E76046E9E7184695E76746D1E781465C
:100D90007CE702382C4447E7ACF1020C2B442FE7E8
:100DA000384608E73746E9E6704700BF844641EA1F
:100DB000000313F003036DD1403A41D351F8043BD3
:100DC00040F8043B51F8043B40F8043B51F8043B25
:100DD00040F8043B51F8043B40F8043B51F8043B15
:100DE00040F8043B51F8043B40F8043B51F8043B05
:100DF00040F8043B51F8043B40F8043B51F8043BF5
:100E000040F8043B51F8043B40F8043B51F8043BE4
:100E100040F8043B51F8043B40F8043B51F8043BD4
:100E200040F8043B51F8043B40F8043B51F8043BC4
:100E300040F8043B51F8043B40F8043B403ABDD233
:100E4000303211D351F8043B40F8043B51F8043BD5
:100E500040F8043B51F8043B40F8043B51F8043B94
:100E600040F8043B103AEDD20C3205D351F8043B64
:100E700040F8043B043AF9D2043208D0D2071CBF30
:100E800011F8013B00F8013B01D30B880380604659
:100E9000704700BF082A13D38B078DD010F00303CF
:100EA0008AD0C3F10403D21ADB071CBF11F8013B3F
:100EB00000F8013B80D331F8023B20F8023B7BE78E
:100EC000043AD9D3013A11F8013B00F8013BF9D2B9
:100ED0000B7803704B7843708B7883706046704753
:100EE000A2EB0300704700BF02780B78012A28BFED
:100EF0009A42F5D16DE9044540EA0104CDE9026763
:100F00006FF0000C4FEA447212B380EA010414F04F
:100F1000070F6AD100F0070420F0070004F0030572
:100F200021F007014FEAC505F0E8042314F0040F8F
:100F3000F1E804670CFA05F462EA040266EA0406C2
:100F40000AD063EA0403624667EA0407664603E0E0
:100F5000F0E80423F1E8046782FA4CF582EA06041B
:100F6000A4FA8CF46CBB83FA4CF583EA0705A5FA66
:100F70008CF595B950E9022351E9026782FA4CF5E4
:100F800082EA0604A4FA8CF483FA4CF583EA070596
:100F9000A5FA8CF52543DBD09CB92DBAB5FA85F4BA
:100FA00024F0070427FA04F1DDE9026723FA04F3C9
:100FB00003F0FF0001F0FF01FDE80445A0EB010094
:100FC000704724BAB4FA84F424F0070426FA04F132
:100FD000DDE9026722FA04F202F0FF0001F0FF01EE
:100FE000FDE80445A0EB0100704714F0030F3CD16D
:100FF00010F0030428D150F8082B51F8083B82FA6E
:101000004CF582EA0305A5FA8CF55DB950F8042C7D
:1010100051F8043C82FA4CF582EA0305A5FA8CF5F6
:10102000002DE8D02DBAB5FA85F424F0070423FA90
:1010300004F122FA04F202F0FF0001F0FF01FDE8E2
:101040000445A0EB010070474FEAC40420F0030000
:1010500050F8082B21F0030151F8083B0CFA04F476
:1010600062EA040263EA0403C9E710F003041AD039
:10107000A1EB040120F00300E40750F8042B06D094
:101080000FD28B785FFAA2F4E41A06D12BB1CB7899
:101090005FFAB2F4E41A00D11BB920465DF8104B98
:1010A000704701F1040150F8042BCC0721F0030133
:1010B00051F8043B48D824D222F07F4482FA4CF500
:1010C00094EA1325A5FA8CF50AD165B951F8043BC9
:1010D00084EA0204B4EB036F0ED150F8042BEBE763
:1010E0004FEA132355E035F07F454DD10878FDE8F0
:1010F0000445C0F1000070474FEA126203F0FF039D
:1011000047E002EA1C4482FA4CF594EA1345A5FA3A
:101110008CF50AD165B951F8043B84EA0204B4EBBA
:10112000034F0CD150F8042BEBE74FEA134330E0A8
:1011300015EA1C4528D10B884FEA124229E04FEAF4
:10114000124203EA1C4324E002F0FF0482FA4CF549
:1011500094EA1365A5FA8CF50AD165B951F8043BF8
:1011600084EA0204B4EB032F09D150F8042BEBE717
:101170004FEA13630DE015F0FF0F05D10B684FEA3E
:10118000122223F07F4304E04FF00000FDE8044505
:10119000704712BA1BBA82FA4CF482EA0304A4FA2A
:1011A0008CF5B5FA85F402FA04F203FA04F34FEA77
:1011B0001260FDE80445A0EB1360704700000000DA
:1011C00090F800F06DE9024520F007016FF0000C87
:1011D00010F0070491F820F040F049804FF000042F
:1011E0006FF00700D1E9002391F840F000F108000A
:1011F00082FA4CF2A4FA8CF283FA4CF3A2FA8CF342
:101200004BBBD1E9022382FA4CF200F10800A4FAA8
:101210008CF283FA4CF3A2FA8CF3E3B9D1E90423FC
:1012200082FA4CF200F10800A4FA8CF283FA4CF333
:10123000A2FA8CF37BB9D1E9062301F1200182FAED
:101240004CF200F10800A4FA8CF283FA4CF3A2FAF3
:101250008CF3002BC6D0002A04BF04301A4612BA01
:10126000B2FA82F2FDE8024500EBD2007047D1E904
:10127000002304F00305C4F100004FEAC50514F093
:10128000040F91F840F00CFA05F562EA05021CBF64
:1012900063EA050362464FF00004A9E7000000007E
:1012A00001F0FF01102A2BDB10F0070F08D010F817
:1012B000013B013A8B422DD010F0070F42B3F6D11B
:1012C000F0B441EA012141EA014122F007047FF034
:1012D00000070023F0E80256083C85EA010586EA8B
:1012E000010685FA47F5A3FA87F586FA47F6A5FAC7
:1012F00087F68EB9EED1F0BC01F0FF0102F00702D3
:1013000032B110F8013B013A83EA010313B1F8D17D
:101310000020704701387047002D06BF354603385E
:10132000073815F0010F07D1013015F4807F02BF97
:10133000013015F4C03F0130F0BC0138704700BFE8
:101340004FEA410C7FEA6C5C02D150EA013C0AD1C1
:101350004FEA430C7FEA6C5C02D152EA033C02D1B3
:101360004FF0000070474FF0010070474FEA410214
:1013700012F5001215D211D56FF47873B3EB6252E7
:1013800012D94FEAC12343F0004343EA505311F00E
:10139000004F23FA02F018BF404270474FF00000A0
:1013A000704750EA013005D111F0004008BF6FF0DE
:1013B000004070474FF00000704700BF10B5044672
:1013C0000E4B18784FF47A73B3FBF0F30C4A1068A5
:1013D000B0FBF3F000F036FA68B90F2C01D9012008
:1013E0000AE0002221464FF0FF3000F0D7F9034B0E
:1013F0005C60002000E0012010BD00BF0000002064
:101400000800002008B50B4B1A6842F400721A60FD
:101410001A6842F480621A601A6842F480721A6094
:10142000032000F0A9F90020FFF7C8FF01F0C2F87F
:10143000002008BD003C0240034A1168034B1B78A2
:101440000B441360704700BF981700200000002075
:10145000014B1868704700BF981700204A4B5A6824
:1014600022F440325A605A6841680A435A6002685E
:10147000536823F48073536002685368016943EA38
:10148000012353600268536823F04073536002687D
:10149000536881680B4353600268936823F40063C8
:1014A000936002689368C1680B439360826A374B0C
:1014B0009A424BD00268936823F07063936002688D
:1014C0009368816A0B4393600268936823F04053EA
:1014D000936002689368C16A0B43936002689368E3
:1014E00023F00203936002689368017E43EA41039C
:1014F000936090F82030002B33D10268536823F4B6
:10150000006353600268D36A23F47003D3620168F6
:10151000CB6AC269013A43EA0253CB62026893681C
:1015200023F4007393600268936890F8301043EAE4
:10153000412393600268936823F480639360026898
:101540009368416943EA8123936070470268936816
:1015500023F0706393600268936823F040539360B4
:10156000BCE70268536843F4006353600268536841
:1015700023F46043536001684B68426A013A43EACE
:1015800042334B60BEE700BF002301400100000F63
:1015900038B310B50446036C43B1236C13F0100F3D
:1015A0000BD00120002384F83C3010BD00F02AFF4E
:1015B0000023636484F83C30EFE7236C23F4885302
:1015C00023F0020343F0020323642046FFF746FFA3
:1015D00000206064236C23F0030343F001032364C1
:1015E000E0E701207047000030B482B0002301938F
:1015F00090F83C30012B00F0B780012380F83C309C
:101600000B68092B3ED90568EA689BB203EB4303DC
:101610001E3B072404FA03F322EA0303EB60056888
:10162000EA688C680B8803EB43031E3B04FA03F360
:101630001343EB604B68062B3AD805686A6B03EBE3
:101640008303053B1F2404FA03F322EA03036B63BD
:1016500005686A6B4B6803EB8303053B0C8804FA4F
:1016600003F313436B630268404B9A4250D0026805
:101670003E4B9A4255D0002380F83C30184602B0C9
:1016800030BC704705682A699BB203EB430307240B
:1016900004FA03F322EA03032B6105682A698C68C4
:1016A0000B8803EB430304FA03F313432B61C1E7F5
:1016B0000C2B16D805682A6B03EB8303233B1F24EE
:1016C00004FA03F322EA03032B6305682A6B4B68D1
:1016D00003EB8303233B0C8804FA03F313432B63CC
:1016E000C1E70568EA6A03EB8303413B1F2404FA60
:1016F00003F322EA0303EB620568EA6A4B6803EB33
:101700008303413B0C8804FA03F31343EB62AAE71B
:101710000B68122BABD1164A536843F48003536015
:10172000A5E70B68103B012BA5D8114A536843F479
:10173000000353600B68102B9DD10E4B1B6802F108
:10174000467202F52E3202F28332A2FB03239B0C77
:1017500003EB83035A00019202E0019B013B0193DA
:10176000019B002BF9D186E7022088E70020014089
:101770000023014008000020074AD36823F4E063F7
:101780001B041B0C000200F4E060184340F0BF6033
:1017900040F40030D060704700ED00E030B4174BEB
:1017A000DB68C3F30223C3F10704042C28BF04241D
:1017B0001D1D062D18D9033B4FF0FF3505FA04F423
:1017C00021EA0401994005FA03F322EA03031943CD
:1017D00000280BDB0901C9B200F1604000F561404F
:1017E00080F8001330BC70470023E5E700F00F00DD
:1017F0000901C9B2024B1954F4E700BF00ED00E043
:1018000014ED00E0002807DB00F01F02400901236F
:101810009340024A42F82030704700BF00E100E0E8
:1018200000280CDB00F01F02400901239340203008
:10183000034A42F82030BFF34F8FBFF36F8F7047DA
:1018400000E100E00138B0F1807F0AD2064B586019
:10185000064AF02182F823100020986007221A60BF
:1018600070470120704700BF10E000E000ED00E08D
:1018700000230F2B00F2C580F0B482B039E00422BF
:1018800000E00022B2403A4302345E4E46F8242083
:101890005D4A1468EA4302EA04064F6817F4803F81
:1018A00001D045EA0406584C2660646802EA040642
:1018B0004F6817F4003F01D045EA0406524C6660B9
:1018C000A46802EA04064F6817F4801F01D045EAB5
:1018D00004064D4CA660E46822404E6816F4001FD2
:1018E00001D045EA0402484CE26001330F2B00F2BC
:1018F000858001229A400C6804EA0205AA42F4D1CC
:101900004C68022C01D0122C10D1DE08083650F899
:1019100026C003F00704A7000F24BC402CEA040CE7
:101920000C69BC4044EA0C0440F8264004685F009F
:101930000326BE40F64306EA040C4C6804F0030498
:10194000BC4044EA0C0404604C6804F1FF3CBCF168
:10195000010F03D9112C01D0122C10D1846806EA92
:10196000040CCC68BC4044EA0C048460446824EA5B
:1019700002024C68C4F300149C4014434460C268E3
:1019800016408A68BA403243C2604A6812F0805FEB
:10199000ABD0002201921D4A546C44F4804454643C
:1019A000526C02F480420192019A9C08A61C154ACE
:1019B00052F8267003F0030296000F22B24027EA85
:1019C0000207134A90423FF45CAF02F580629042F6
:1019D0000ED002F5806290420CD002F580629042F7
:1019E0000AD002F5806290423FF449AF072249E7EE
:1019F000012247E7022245E7032243E702B0F0BC99
:101A00007047704700380140003C014000380240F8
:101A10000000024012B9090481617047816170477A
:101A2000002800F0BB8170B582B00446036813F053
:101A3000010F3BD0A74B9B6803F00C03042B2CD069
:101A4000A44B9B6803F00C03082B21D06368B3F50B
:101A5000803F4FD0B3F5A02F52D09E4B1A6822F48E
:101A600080321A601A6822F480221A606368002BA0
:101A700050D0FFF7EDFC0546964B1B6813F4003F72
:101A800014D1FFF7E5FC401B6428F5D903208AE157
:101A9000904B5B6813F4800FD8D08E4B1B6813F407
:101AA000003F03D06368002B00F07A81236813F0B5
:101AB000020F55D0874B9B6813F00C0F3ED0854B1F
:101AC0009B6803F00C03082B33D0E368002B68D02D
:101AD000814B01221A60FFF7BBFC05467D4B1B685A
:101AE00013F0020F54D1FFF7B3FC401B0228F5D9C5
:101AF000032058E1774A136843F480331360B5E755
:101B0000744B1A6842F480221A601A6842F48032D8
:101B10001A60ABE7FFF79CFC05466E4B1B6813F49D
:101B2000003FC3D0FFF794FC401B6428F5D9032085
:101B300039E1684B5B6813F4800FC6D1654B1B68B5
:101B400013F0020F04D0E368012B01D001202AE139
:101B5000604A136823F0F803216943EAC103136064
:101B6000236813F0080F40D0636963B35B4B012215
:101B70001A60FFF76DFC0546564B5B6F13F0020FC2
:101B800033D1FFF765FC401B0228F5D903200AE199
:101B9000504A136823F0F803216943EAC103136034
:101BA000DEE74D4B00221A60FFF752FC0546494B19
:101BB0001B6813F0020FD3D0FFF74AFC401B02282A
:101BC000F5D90320EFE0454B00221A60FFF740FCF7
:101BD0000546404B5B6F13F0020F06D0FFF738FC51
:101BE000401B0228F5D90320DDE0236813F0040F21
:101BF00079D0384B1B6C13F0805F33D100230193F5
:101C0000344B1A6C42F080521A641B6C03F0805300
:101C10000193019B0125324B1B6813F4807F23D075
:101C2000A368012B34D0052B38D02A4B1A6F22F031
:101C300001021A671A6F22F004021A67A368002BC8
:101C400036D0FFF705FC0646224B1B6F13F0020F40
:101C500048D1FFF7FDFB801B41F288339842F3D94E
:101C60000320A0E00025D6E71D4A136843F48073E3
:101C70001360FFF7EDFB0646194B1B6813F4807FDA
:101C8000CED1FFF7E5FB801B0228F5D903208AE0BF
:101C9000104A136F43F001031367CFE70D4B1A6F20
:101CA00042F004021A671A6F42F001021A67C5E790
:101CB000FFF7CEFB0646074B1B6F13F0020F11D048
:101CC000FFF7C6FB801B41F288339842F3D903200B
:101CD00069E000BF0038024000004742800E4742E2
:101CE00000700040E5B9A369002B5BD0304A9268D0
:101CF00002F00C02082A58D0022B17D02D4B0022DC
:101D00001A60FFF7A5FB0446294B1B6813F0007F00
:101D100042D0FFF79DFB001B0228F5D9032042E0CB
:101D2000234A136C23F080531364DCE7214B002219
:101D30001A60FFF78DFB05461D4B1B6813F0007FF3
:101D400006D0FFF785FB401B0228F5D903202AE0C7
:101D5000E369226A1343626A43EA8213A26A520861
:101D6000013A43EA0243E26A43EA0263104A5360DB
:101D7000104B01221A60FFF76BFB04460C4B1B68EB
:101D800013F0007F06D1FFF763FB001B0228F5D993
:101D9000032008E0002006E0002004E00120704756
:101DA000012000E0002002B070BD0120FBE700BF71
:101DB0000038024060004742264B9B6803F00C034A
:101DC000042B44D0082B01D0234870472DE9F04B59
:101DD000204B5A6802F03F025B6813F4800F13D067
:101DE0001C4B5968C1F3881100231C48A1FB00015A
:101DF000FEF75CFE174B5B68C3F3014301335B00E6
:101E0000B0FBF3F0BDE8F08B124B5B68C3F38813B3
:101E10001E4600275C010025E41A65EB0705A901B1
:101E200041EA9461A001001B61EB0501CB0043EA8C
:101E30005073C400A01943EB07018B0243EA90538F
:101E40008402204619460023FEF730FED2E70348FD
:101E5000704700BF003802400024F40040787D0144
:101E6000002800F09D8070B504464F4B1B6803F0BE
:101E70000F038B4209D2CBB24B4A1370136803F0A5
:101E80000F038B4201D0012070BD236813F0020FB5
:101E900017D013F0040F04D0444A936843F4E0537E
:101EA0009360236813F0080F04D0404A936843F40A
:101EB000604393603D4A936823F0F003A0680343B6
:101EC00093600D46236813F0010F32D06368012B35
:101ED00021D09A1E012A25D9344A126812F0020F25
:101EE00060D032498A6822F0030213438B60FFF707
:101EF000AFFA06462D4B9B6803F00C036268B3EB08
:101F0000820F16D0FFF7A4FA801B41F28833984263
:101F1000F0D90320B8E7254A126812F4003FE0D157
:101F20000120B1E7214A126812F0007FD9D10120C7
:101F3000AAE71D4B1B6803F00F03AB4209D9EAB2B5
:101F4000194B1A701B6803F00F03AB4201D001203C
:101F50009AE7236813F0040F06D0144A936823F419
:101F6000E053E1680B439360236813F0080F07D038
:101F70000E4A936823F46043216943EAC1039360E6
:101F8000FFF71AFF094B9B68C3F30313084AD35C9E
:101F9000D840084B18600020FFF710FA002073E7C4
:101FA0000120704701206FE7003C024000380240EA
:101FB00068C9000808000020014B1868704700BF7E
:101FC0000800002008B5FFF7F7FF044B9B68C3F338
:101FD0008223034AD35CD84008BD00BF00380240CA
:101FE00078C9000808B5FFF7E7FF044B9B68C3F307
:101FF0004233034AD35CD84008BD00BF00380240DA
:1020000078C900082DE9F84304460268136923F4EF
:102010004053C1680B4313618368026913434269EB
:102020001343C2691A430168CB6823F4164323F0B3
:102030000C031343CB600268536923F44073816936
:102040000B435361C369B3F5004F60D00368B84ACE
:10205000934200F0148102F58062934200F00F81F8
:10206000FFF7B0FF00EB800000EB80006568AD007B
:10207000B0FBF5F5AF4FA7FB05356D092E01FFF756
:10208000A1FF00EB800000EB80006568AD00B0FBB5
:10209000F5F9FFF797FF00EB800000EB8000656823
:1020A000AD00B0FBF5F5A7FB05356D094FF06408F1
:1020B00008FB15952D013235A7FB05356D0905F097
:1020C000F0053544FFF77EFF00EB800000EB800059
:1020D0006668B600B0FBF6F6FFF774FF00EB800011
:1020E00000EB800063689B00B0FBF3F0A7FB0030BF
:1020F000400908FB10684FEA081808F13208A7FBEE
:102100000837C7F3431723682F449F600DE1036826
:10211000874A93425BD002F58062934257D0FFF723
:1021200051FF00EB800000EB800065686D00B0FBA4
:10213000F5F5804FA7FB05356D092E01FFF742FF2E
:1021400000EB800000EB800065686D00B0FBF5F9E6
:10215000FFF738FF00EB800000EB800065686D0042
:10216000B0FBF5F5A7FB05356D094FF0640808FBDA
:102170001595ED003235A7FB05356D096D0005F4A9
:10218000F8753544FFF71EFF00EB800000EB800080
:1021900066687600B0FBF6F6FFF714FF00EB8000F0
:1021A00000EB800063685B00B0FBF3F3A7FB032345
:1021B0005B0908FB13684FEAC80808F13208A7FB5F
:1021C0000837C7F3421723682F449F60ADE0FFF73D
:1021D00009FF00EB800000EB800065686D00B0FB3C
:1021E000F5F5544FA7FB05356D092E01FFF7FAFEF3
:1021F00000EB800000EB800065686D00B0FBF5F936
:10220000FFF7F0FE00EB800000EB800065686D00DA
:10221000B0FBF5F5A7FB05356D094FF0640808FB29
:102220001595ED003235A7FB05356D096D0005F4F8
:10223000F8753544FFF7D6FE00EB800000EB800018
:1022400066687600B0FBF6F6FFF7CCFE00EB800088
:1022500000EB800063685B00B0FBF3F3A7FB032394
:102260005B0908FB13684FEAC80808F13208A7FBAE
:102270000837C7F3421723682F449F6055E0FFF7E4
:10228000B1FE00EB800000EB80006568AD00B0FBA4
:10229000F5F5284FA7FB05356D092E01FFF7A2FEC6
:1022A00000EB800000EB80006568AD00B0FBF5F945
:1022B000FFF798FE00EB800000EB80006568AD0042
:1022C000B0FBF5F5A7FB05356D094FF0640808FB79
:1022D00015952D013235A7FB05356D0905F0F00583
:1022E0003544FFF77FFE00EB800000EB800066685E
:1022F000B600B0FBF6F6FFF775FE00EB800000EBD2
:10230000800063689B00B0FBF3F0A7FB003040093E
:1023100008FB10684FEA081808F13208A7FB0837D5
:10232000C7F3431723682F449F60BDE8F88300BFBD
:10233000001001401F85EB5158B310B5044690F8CA
:1023400039300BB3242384F839302268D36823F45E
:102350000053D3602046FFF755FE2268136923F42B
:10236000904313612268536923F02A035361226862
:10237000D36843F40053D3600020E063202384F843
:10238000393084F83A3010BD80F8383000F09AF9CE
:10239000D8E701207047000000B585B00023009306
:1023A0000193029303931448144A026043608360CC
:1023B0000361037680F82030C362114A8262C360F1
:1023C0000122C26180F830304261FFF7E1F868B95C
:1023D00008230093012301930023029369460648D2
:1023E000FFF702F928B905B05DF804FB00F0E0F84A
:1023F000EEE700F0DDF8F6E79C1700200020014032
:102400000100000F00B589B00023039304930593E6
:1024100006930793026803F1804303F590339A42D1
:1024200002D009B05DF804FB0021019103F58C3363
:102430005A6C42F480725A645A6C02F480720192AF
:10244000019A02911A6B42F002021A631B6B03F0AD
:1024500002030293029B012303930323049303A922
:102460000148FFF705FADCE70004024070B58AB0C6
:102470000024059406940794089409940194224B2F
:102480001A6B42F004021A631A6B02F00402019202
:10249000019A02941A6B42F080021A631A6B02F0DE
:1024A00080020292029A03941A6B42F002021A63AB
:1024B0001A6B02F002020392039A04941A6B42F020
:1024C00001021A631B6B03F001030493049B0F4D7D
:1024D00022464FF470612846FFF79CFA4FF4704390
:1024E000059306940126079605A92846FFF7C0F92B
:1024F0004FF47063059306960794089405A928463F
:10250000FFF7B6F90AB070BD00380240000802407B
:1025100010B594B03022002108A803F081FE0024F9
:10252000039404940594069407940194164B1A6C32
:1025300042F080521A641B6C03F080530193019B9C
:102540000294124A136823F4404343F40043136097
:10255000136803F440430293029B02230893012370
:102560000B9310230C930E9408A8FFF759FA0F232E
:1025700003930494059406940794214603A8FFF757
:102580006FFC14B010BD00BF003802400070004066
:1025900008B5FEF737FFFFF7BBFFFFF767FFFFF751
:1025A000FBFE00F075F800F06DF900F0CFF9FCE7E4
:1025B0007047000082B0002100910B4B5A6C42F42E
:1025C00080425A645A6C02F480420092009A01914F
:1025D0001A6C42F080521A641B6C03F08053019312
:1025E000019B02B0704700BF003802407047FEE711
:1025F000FEE7FEE7FEE770477047704708B5FEF755
:102600001BFF00F0E3FC08BD08B503460B4A126847
:1026100042B10A4A106803446A46934206D8074A00
:10262000136008BD054A06491160F2E702F072FE28
:102630000C2303604FF0FF30F3E700BFD4110020FC
:10264000B01D00200F49D1F8883043F47003C1F861
:1026500088300D4B1A6842F001021A600020986021
:102660001A6822F0847222F480321A60074A5A6093
:102670001A6822F480221A60D8604FF000638B60E1
:10268000704700BF00ED00E0003802401030002429
:1026900008B50A480A4B03604FF4E1334360002356
:1026A0008360C36003610C2242618361C361FFF7F1
:1026B00043FE00B908BDFFF77BFFFBE7E4170020EE
:1026C0000010014000B589B00023039304930593E3
:1026D00006930793026803F1804303F588339A4217
:1026E00002D009B05DF804FB0021019103F5943399
:1026F0005A6C42F010025A645A6C02F010020192B5
:10270000019A02911A6B42F001021A631B6B03F0EB
:1027100001030293029B4FF4C063039302230493CB
:1027200001230593032306930723079303A9024874
:10273000FFF79EF8D5E700BF0000024008B502F0A1
:102740002DFB0121084602F057FD044B1A68596819
:10275000034803F0BBFD02F02FFB08BD0C00002076
:102760002CCB0008284B1B6803B9704710B502F04A
:10277000FFFC002846D004301C2833D8DFE800F0E6
:10278000271F170F32323232323232323232323285
:1027900032323232322F3232323232322F001B4B4F
:1027A0001B68022B1EDD013B184A13601AE0174B11
:1027B0001B68162B16DC0133144A136012E0134B0E
:1027C0005B68022B0EDD013B104A53600AE00F4BA1
:1027D0005B684D2B06DC01330C4A536002E00A4B68
:1027E00000221A6002F02AFD084C2168606802F09D
:1027F00003FD2A2003F07EFD2168606802F0FCFCE6
:10280000FFF79CFF10BD00BFDC1100200C00002072
:10281000164B5B6843B310B5154B9B682BB93C2135
:10282000144802F0BFFC38B910BD134803F04EFD48
:102830000F4B00229A60F2E70A2003F05BFD0D4C7B
:102840002046FEF7BDFC024621460C4803F03EFD43
:102850000B492046FEF748FB10B9044B00225A6092
:10286000034B01229A60DFE7704700BFDC110020B4
:102870000C0000202C18002044CB000858CB000886
:1028800078CB000808B5064800F0B4FB02F07EFAE9
:10289000044B01221A60044803F084FD08BD00BF08
:1028A00080CB0008080800208CCB0008224B1B6856
:1028B000002B40D1214B1B68002B3CD11F4B5B6888
:1028C000002B38D110B51D4B9B6863B102F05EFC44
:1028D00010F0FF0F06D0C0B232281AD0332822D011
:1028E00031280FD010BD02F097FC154803F05AFDB7
:1028F000144803F057FD144803F054FD0F4B012218
:102900009A60E3E70C4B01221A600C4B00229A609C
:10291000E8E70A4B01221A6000229A6002F07CFC70
:10292000FFF70CFFDEE7054C0123636002F074FC47
:102930000023A360D6E770471C000020DC110020B4
:1029400094CB0008A4CB0008B0CB000808B5FFF773
:10295000ADFFFFF707FF00F0DBF900F0A3F8FFF78A
:1029600057FF08BD08B54FF4805000F0A5FB00B933
:1029700008BD00F059F9FBE770B5FEF769FD134B90
:102980001B68C31A642B00D870BD04464FF4804006
:1029900000F088FB05464FF4004000F083FB06463C
:1029A00005B120B105B956B9084B1C60ECE74FF0F2
:1029B000FF3000F025F9054B00225A60F2E70120B4
:1029C00000F01EF9014B01225A60EDE7E8110020EA
:1029D00010B5FEF73DFD2E4BD3ED007AF8EEE77A09
:1029E0009FED2C7A67EE877AB0EE007A77EE877AE1
:1029F000DFED296A86EEA77AFDEEC77A17EE903AE8
:102A0000264AC2ED007A264A9268821A9A422DD945
:102A1000234A9060D3680133D360032B02DD134651
:102A20000022DA601E4B5B6863B31D4BDB684FF41A
:102A300000641C411A4B1B6903B1E44304F4807128
:102A40004FF4807000F0B8FA04F400714FF4007095
:102A500000F0B2FA04F480614FF4806000F0ACFA48
:102A600004F400614FF4006000F0A6FA4FF4005047
:102A700000F022FB28B10A4A1369B3FA83F35B0919
:102A8000136110BD064BDB684FF480749C40D1E7A6
:102A90006C1800203333933F00007A441800002064
:102AA000E811002008B5FFF793FF044B1B6803B93A
:102AB00008BDFFF757FFFFF75FFFF9E71C00002095
:102AC00008B50721012002F0C3FB0121084602F0EE
:102AD00093FB074B1B6843B92021064B1B68064A32
:102AE0001268064803F0F2FB08BD2A21F5E700BF93
:102AF000741800206C18002070180020C0CB00084B
:102B000010B504464168012909DD006802F074FB34
:102B1000A168002002F09CFB4F2003F0EBFBFEF7C6
:102B200097FCE06010BD10B504464168006802F0F3
:102B300063FB0021084602F08BFB202003F0DAFB48
:102B40006368013B6360012B04DD2046FFF7D8FF7B
:102B5000002010BD0120FCE730B10022026042607D
:102B6000024A1368013B1360704700BF6C180020D5
:102B700038B5002400E00134132C19DC22010D4B80
:102B8000D518D358002BF6D06B68002BF3D0FEF786
:102B90005FFCEB68C01A6428EDD92846FFF7C3FF35
:102BA0000028E8D02846FFF7D7FFFFF789FFE2E7C4
:102BB00038BD00BF7818002008B51821054B1868EB
:102BC00002F01AFB0721002002F042FB024803F04A
:102BD0007DFB08BD70180020E4CB000808B5182163
:102BE000054B186802F008FB0721002002F030FBBB
:102BF000024803F06BFB08BD70180020E8CB00080A
:102C000010B5084B1B681C18621E4B2A07D8A3423C
:102C100005D0FFF7E3FF034B1C60FFF7CDFFFFF785
:102C20004FFF10BD7018002010B51B4B1B68132BF5
:102C30002EDC002300E00133132B0CDC1A011749B2
:102C40008A58002AF7D101EB03125268002AF2D108
:102C500001EB031400E00024E4B1114B1B680133C5
:102C600023601723636003F0A5FB0E4B83FB002357
:102C70001A18C317C3EBA203C3EBC303C31A013370
:102C8000A360054A1368013313602046FFF738FF3D
:102C9000FFF716FF10BD00BF6C1800207818002049
:102CA000701800209324499210B5134B28221A6003
:102CB0000123124A1360124A136002F067F802F00F
:102CC000E3FA0721002002F0C3FA02F0A5FAFFF7A9
:102CD00073FFFFF7F5FE00230A4A136006E00A4976
:102CE0001A018C180020606088500133132BF6DD28
:102CF000064B01221A6010BD7018002074180020C5
:102D0000080800206C18002078180020FC11002012
:102D1000A24B1B68002B00F0408110B5A04B1B6834
:102D200053B1A04B1B6853B902F022FA044648B9CC
:102D3000002002F09BFC10BDFFF7B6FFF1E7FFF7A4
:102D400017FFF1E70121282002F056FA00210220A6
:102D500002F07EFA2146944803F0B8FA0434742C49
:102D6000E6D801A353F824F0472F00083D2F0008B0
:102D7000712F00084F2F0008312D0008312D000859
:102D8000312D0008312D0008312D0008312D0008AB
:102D9000312D0008312D0008312D0008312D00089B
:102DA0004F2F0008312D0008312D00084F2F00084B
:102DB000312D0008312D0008312D00087F2F00082B
:102DC000312D0008312D0008312D0008312D00086B
:102DD000312D0008312D00087F2F0008312D00080B
:102DE000312D0008312D0008312D0008312D00084B
:102DF000312D0008312D00084F2F0008312D00081B
:102E0000312D0008312D0008312D0008312D00082A
:102E1000312D0008312D0008312D0008312D00081A
:102E2000312D0008312D0008312D0008312D00080A
:102E3000312D0008312D0008312D0008312D0008FA
:102E4000312D0008312D0008312D0008312D0008EA
:102E5000312D0008312D0008312D0008312D0008DA
:102E6000312D0008312D0008312D0008312D0008CA
:102E7000312D0008312D0008312D00083D2F0008AC
:102E8000312D0008312D0008472F0008312D000892
:102E9000312D0008312D0008312D0008312D00089A
:102EA000312D0008312D0008312D0008312D00088A
:102EB000312D0008312D0008312D0008312D00087A
:102EC000312D0008312D0008312D0008312D00086A
:102ED000312D0008312D0008312D0008312D00085A
:102EE000312D0008312D0008312D0008312D00084A
:102EF000312D0008312D0008312D00083D2F00082C
:102F0000312D0008312D0008472F0008312D000811
:102F1000312D0008312D0008312D0008312D000819
:102F2000312D0008312D0008552F0008712F0008A1
:102F3000312D0008312D00085B2F00084FF0FF30C5
:102F4000FFF75EFEF4E60120FFF75AFEF0E6FFF71A
:102F50006BFEEDE6FFF70CFEEAE60721002002F02B
:102F600077F902F059F9FFF727FEFFF701FEDFE6D8
:102F70000C4A1368B3FA83F35B091360D8E60024A4
:102F8000064B1C600721204602F062F902F044F96A
:102F900002F088F9024B1C60CAE670471C00002052
:102FA000FC11002074180020ECCB00080004014B39
:102FB000986170470008024019B90004024B9861FB
:102FC0007047014B986170470008024008B5FEF752
:102FD0003FFA142806D9044B1B69044A12681340AF
:102FE000034A136008BD00BF000802402000002013
:102FF000B819002010B586B0044600F05BFF00F061
:1030000051FF22462146204600F0DEFF1E490020E7
:1030100001F007FD1D4B1868002302221946806845
:1030200003F0F8F9012411E0194800F05DFA00946A
:103030000346184A092103A803F0ACFA03A800F0DC
:1030400010FAA0B2FFF7B2FF07E06400B4F5803FCA
:1030500016D2114B1B681C42E6D1104B1B681C4258
:10306000F3D00B4800F040FA00940346094A0921C6
:1030700003A803F08FFA0A4903A800F09BF9E4E7DC
:10308000FFF7A4FF06B010BDF4CB00080C08002029
:103090000008024004CC000824000020200000208A
:1030A0000CCC0008034B1B68184214BF0120002001
:1030B000704700BFB81900200D4B1A6802400D4B35
:1030C0001B6800EA03018A420CD023EA0003134381
:1030D00008490B60084B186800B12AB930B932B9F9
:1030E0000120704700207047012070470020704782
:1030F000B8190020101200201412002000B338B5B7
:103100000478FCB1FEF75CF8032801D800201AE02F
:10311000254602F0A5FD2044437803F00303022B6B
:1031200007D0462D08D04F2D0ED0412D06D00020BF
:1031300009E0A4F12005F4E7022004E0032002E006
:1031400000207047002038BD0120FCE770B310B5A7
:103150000446027862B3FEF733F8032801D8002052
:1031600027E0A47802F07CFD2044437803F00303B9
:10317000022B13D0313C1C2C12D8DFE804F01511BF
:10318000111113111111111111111111111111112D
:10319000111111131115111111111B00203CE9E738
:1031A000002006E0022004E0032002E00020704737
:1031B000002010BD0120FCE7E0B110B50446027804
:1031C000D2B1FDF7FDFF032801D8002015E0E47817
:1031D00002F046FD2044437803F00303022B05D0A0
:1031E000442C05D0552C09D0002006E0203CF7E700
:1031F000022002E000207047002010BD0120FCE703
:10320000082834D81D4B53F82030002B32D084B01E
:10321000012812D002281DD008B100200BE00023A5
:103220000193174B1A6B42F001021A631B6B03F0F8
:1032300001030193019B04B0704700200290104BE2
:103240001A6B42F002021A631B6B03F00203029333
:10325000029BF0E700200390094B1A6B42F0040236
:103260001A631B6B03F004030393039BE3E74FF024
:10327000FF3070476FF00100704700BF80C9000841
:103280000038024008281AD8F0B587B0104C54F81E
:103290002060BEB11C4615460F46FFF7B1FF00285F
:1032A00013DB0197029504940C9B03930D9B0593EC
:1032B00001A93046FEF7DCFA002007B0F0BD4FF060
:1032C000FF3070476FF00100F7E76FF00200F4E79E
:1032D00080C9000840B370B5054604783CB3264663
:1032E00002F0BEFC2044437803F00303022B14D009
:1032F000502E15D02C7802F0B3FC2044437803F014
:103300000303022B0ED014F0FF0313D0413BDBB2BA
:10331000092B12D8E0B2413870BDA4F12006E7E7CE
:103320000135E7E7203CEEE74FF0FF3070476FF0E4
:103330000100F1E76FF00200EEE76FF00300EBE74A
:1033400048B370B50446057845B32E4602F088FCB4
:103350002844437803F00303022B17D0502E18D0D3
:103360002378F3B1651C6378F3B102F079FC6378DC
:103370001844437813F0040F19D00A22002128467C
:1033800003F0CEFC012303FA00F070BDA5F1200686
:10339000E4E70134E4E74FF0FF3070476FF00100DD
:1033A000F3E76FF00200F0E76FF00300EDE76FF076
:1033B0000400EAE72DE9F04182B006460C46FFF72B
:1033C00089FF05463046FFF7BBFF002D1FDB064691
:1033D00000281FDB2046FFF791FE07462046FFF737
:1033E000B5FE80462046FFF7E7FE002301930090DC
:1033F00043463A4631462846FFF744FF002803DBA0
:10340000002002B0BDE8F0816FF00100F9E74FF055
:10341000FF30F6E74FF0FF30F3E730B583B00546F5
:10342000FFF758FF04462846FFF78AFF002C12DBFF
:10343000002813DB0022019201230093134601466A
:103440002046FFF71FFF002802DB002003B030BD3D
:103450006FF00100FAE74FF0FF30F7E74FF0FF3071
:10346000F4E730B583B00546FFF734FF044628463D
:10347000FFF766FF002C11DB002812DB002301930D
:103480000093012201462046FFF7FCFE002802DBE4
:10349000002003B030BD6FF00100FAE74FF0FF30BD
:1034A000F7E74FF0FF30F4E770B582B004460E4600
:1034B000FFF710FF05462046FFF742FF002D0DDB0A
:1034C00000280EDB0196002400940123022201460D
:1034D0002846FFF7D7FE204602B070BD4FF0FF3000
:1034E000FAE74FF0FF30F7E741220023082B0FDC0B
:1034F000084951F82310814203D001330132D2B27E
:10350000F4E705485023037042700023837070472E
:103510000248704780C900081812002074CB0008C8
:103520000B7B03BB4A688B689A421CD010B40A68B4
:103530004B68D45C4B6801334B604B685A4203F0D4
:103540007F0302F07F0258BF53424B6001234B734D
:103550000B7303685C600268D36843F04003D36078
:103560005DF8044B7047704770B582B004460E4654
:1035700000F154010068C36823F04003C360E56DA7
:1035800001356B4205F07F0503F07F0358BF5D42B4
:10359000A36DAB420ED0626DE36DD654E56594F831
:1035A000603023B12268D36843F04003D3603046D3
:1035B00002B070BD52B1A36D01335A4203F07F03D4
:1035C00002F07F0258BF5342A365E4E794F86030ED
:1035D0002BB12268D36843F04003D3600DE020464E
:1035E000FFF79EFF09E0019B01330193019941F22E
:1035F00087339942F7DD95420FD12268D36823F0D3
:103600004003D360A26D2168CB6843F04003CB60D8
:103610009542F0D100230193E8E72268D36823F0B4
:103620004003D360B7E730B40468D0F8CC2090F8FA
:10363000D030EBB9D2F8C831D2F8CC118B4217D0C8
:10364000D11891F8DC500133594203F07F0301F0A7
:103650007F0158BF4B42C2F8C831012380F8D130F6
:1036600080F8D03065600268D36843F04003D360CF
:1036700030BC7047F0B583B005460F46D0F8CC603B
:103680000168CB6823F04003CB60D6F8CC4101340D
:10369000634204F07F0403F07F0358BF5C42D6F816
:1036A000C831A34213D0D5F8CC30D6F8CC2113447E
:1036B00083F8DC70C6F8CC4195F8D03023B12A6885
:1036C000D36843F04003D360384603B0F0BD52B135
:1036D00001335A4203F07F0302F07F0258BF534286
:1036E000C6F8C831DFE790F8D0302BB10268D36854
:1036F00043F04003D3600CE0FFF795FF09E0019B26
:1037000001330193019941F287339942F7DD9442E5
:1037100010D12A68D36823F04003D360D6F8C821BB
:103720002968CB6843F04003CB609442EFD100237B
:103730000193E7E72A68D36823F04003D360B2E738
:1037400038B50446D0F8CC50604A13680133136092
:1037500003681B68C3F340135D4A136013684BB3DF
:1037600003681B68C3F340135A4A1360036859681F
:10377000C9B26FF020021A6003681B68C3F34013DC
:10378000554A1360514A536801335360002D31D0BC
:10379000D5F8C43101335A4203F07F0302F07F02AF
:1037A00058BF5342D5F8C0219A424CD1474A93683A
:1037B000013393602368DA6812F0400F19D06FF07C
:1037C00040021A60002D4AD0404A13690133136148
:1037D000D5F8CC21D5F8C8319A426AD0284600F0F5
:1037E0004EFF002801DB23685860384A9369013393
:1037F000936138BDC36E01335A4203F07F0302F078
:103800007F0258BF5342826E9A4217D0426E002AFE
:10381000D0D0C06E1154E3662C4AD3680133D36014
:10382000E36F13F0020FC5D001222046FFF79CFE84
:1038300004F154012046FFF773FEBBE7234A936867
:1038400001339360B6E70022284600F0A7FE1F4A26
:10385000D3680133D3602046FFF7E5FEAAE71B4A91
:10386000136901331361E26DA36D9A4214D0616D47
:10387000A36D5A1CA2652268CB5C5360A36D5A42AB
:1038800003F07F0302F07F0258BF5342A3650F4A43
:10389000936901339361ACE72268D36823F0400356
:1038A000D360002384F86030084A536901335361C0
:1038B0009FE72268D36823F04003D360002384F895
:1038C000D030024A53690133536192E71C12002041
:1038D000BC190020C0190020C419002008B50448F4
:1038E000FFF72EFF034B2022C3F8842108BD00BF41
:1038F0000801002000E100E008B50448FFF720FFC0
:10390000034B4022C3F8842108BD00BFE80100201A
:1039100000E100E008B50448FFF712FF034B8022E6
:10392000C3F8882108BD00BF6805002000E100E061
:1039300084B01C4BD3F8E03083420BD0194BD3F842
:10394000C031834213D0174BD3F8403583421BD08C
:1039500004B0704700230193134B5A6C42F01002DD
:103960005A645B6C03F010030193019BF0E70023A2
:1039700002930D4B1A6C42F400321A641B6C03F470
:1039800000330293029BE3E700230393064B5A6C38
:1039900042F020025A645B6C03F020030393039B04
:1039A000D6E700BF280000200038024038B5036881
:1039B000002B00F088800446DA6822F40052DA60B6
:1039C0001846FFF7B5FF206C30B1FFF74AFD94F8B9
:1039D0005010206CFFF768FD606C30B1FFF71DFDE3
:1039E00094F85010606CFFF75FFDD4F8CC508DB1A7
:1039F000284600F060FE6060AB6803F4E073802B43
:103A000021D00AD9C02B21D0B3F5807F09D1002362
:103A1000A36006E004F17005EAE7402B01D1002322
:103A2000A360AB6813F0080F13D04FF40053E360AA
:103A3000AB6813F0100F13D013F0200F0CD04FF41D
:103A4000C06323610EE00023A360EAE70023A360C4
:103A5000E7E70023E360EBE74FF48063236101E0D5
:103A6000002323610C2363610023E3612046FEF7FA
:103A700063FC94F95100FDF7C5FE636DCBB10023E3
:103A8000A365E36584F8603084F86130636EABB1A0
:103A90000020A066E0660D4BD86098602268D3686D
:103AA00043F02003D3602268D36843F40053D3600B
:103AB00038BD802002F0EAF86065E0E7802002F07F
:103AC000E5F86066E4E76FF00100F1E71C12002002
:103AD00008280CDC10B5094CC300191A4A0111461C
:103AE0002244635833B11046FFF760FF10BD4FF01A
:103AF000FF3070476FF00100F8E700BF280000209A
:103B0000082821DC38B5C0EBC0025301114AD35854
:103B1000EBB1DA6822F02002DA600E4BC200141A10
:103B200061015D58EC6824F04004EC605C58E16889
:103B300021F40051E160101A4201134493F951003D
:103B4000FDF76EFE002038BD4FF0FF3070476FF07C
:103B50000100F8E7280000202DE9F04383B001932D
:103B6000082800F3BD80634CC3001B1A590104EB05
:103B700001096358002B00F0B6805F4B9A4200F0B9
:103B80009E80044603F5A70303F5FF437F339A4263
:103B900006D003F14043013B9A421DD00020A3E030
:103BA000019B1A1D01921868C4EBC4035A01514BC2
:103BB0001344D3F8CC1021B15C22FDF7F7F80020B4
:103BC00092E0C4EBC404630170335C224949194498
:103BD000FDF7ECF8002087E0019B1A1D01921D689B
:103BE000C200121A5101434B0B44D3F878C02A6823
:103BF0001A676A685A67AA689A67EA68DA67D3F840
:103C0000CC308BB1D3F808C02A681A60394B0B440A
:103C1000D3F8CC2069685160D3F8CC20A9689160B2
:103C2000D3F8CC30EA68DA60002100E001311129D4
:103C300017DC0B1D55F823602E48E200171BFB0014
:103C40000B44203340F82360131B5A011044D0F872
:103C5000CC30002BEAD00A1D55F8220043F8220090
:103C6000E4E7C4EBC4035A01224B1344D3F8C83031
:103C7000A96D8B4202D1AB68634516D0DFF8748022
:103C8000E7003B1B58017030404400F017FD3C1B1F
:103C900063019844D8F8CC0010B1A96D00F00EFD76
:103CA0004846FFF783FE00201EE0124B1344D3F872
:103CB000CC30E3B19B6D9942E0D1002014E0019B30
:103CC0001A1D01921968C0EBC000430103F1D8022C
:103CD000084B13441A685B680A604B60002003E0DD
:103CE0004FF0FF3000E0002003B0BDE8F08300207B
:103CF000FAE700BF2800002003440880082816DCEB
:103D000070B516460D4604464FF4EC7001F0BEFF48
:103D1000C4EBC4035A01074B1344C3F8CC0000F0B2
:103D200004FD324629462046FFF7D2FE70BD4FF013
:103D3000FF3070472800002038B50446FFF7E0FE4A
:103D40000546C4EBC4046201034B1344D3F8CC0012
:103D500001F0A4FF284638BD2800002008281EDCFA
:103D600070B51146C0EBC0046201104CA458CCB130
:103D70001A460546E36823F02003E3600B4EC400B7
:103D8000231A58013044D0F8CC0000F04CFC641BDE
:103D90006301F258D36843F02003D36070BD4FF045
:103DA000FF3070476FF00100F8E700BF28000020E7
:103DB00008281CDCC0EBC00253010F4AD358C3B122
:103DC00070B50446DA6822F02002DA600A4EC500B7
:103DD0002A1A53013344D3F8CC0000F017FC2C1BF3
:103DE0006301F258D36843F02003D36070BD002014
:103DF00070470020704700BF28000020082821DC01
:103E0000F8B5154CC1000D1A6E01354626446159AE
:103E1000D9B1002B1CDD1D461746104B00249C61B8
:103E20005C615C601C611C6005E00022395D30460D
:103E3000FFF720FC0134AC42F7DB3046FFF7F3FB21
:103E40002846F8BD4FF0FF3070476FF00100F8E7EB
:103E50004FF0FF30F5E700BF280000201C120020C3
:103E6000014698B1002300E00133302B04DC0A4AFC
:103E700052F82320002AF7D1302B0ADC064A42F8F8
:103E800023100133002042F8230070474FF0FF3029
:103E900070476FF0010070473C120020002070470F
:103EA0001846704708B50248FFF7DAFF08BD00BFA3
:103EB000DCC9000808B50248FFF7D2FF002008BDA2
:103EC00004CA00082DE9F04782B003253B2D05DC2C
:103ED0002B013B4CE3580BB10135F7E73C2D66D085
:103EE000002867D00378002B67D0894607463449FD
:103EF0002A018B1800249C60DC60C3F80490012325
:103F00008B5014E00A2201A9504602F009FF019BE0
:103F10001B7823B92A4B03EB0513D8602DE02D0144
:103F2000274B00225A516FF0020535E00134312C45
:103F300023DC244B53F82460FEB1D6F800804146C0
:103F4000384602F025FD8742F0D14046FDF738F9AA
:103F5000804607EB000A1A4B03EB05139E603B5C9F
:103F6000002BE3D001F07CFE17F8083018444278AB
:103F700012F0040FDAD0002BC4D1114B03EB051360
:103F80009B684BB19C683CB10D4B03EB05134A4653
:103F90002946D868A04718B9284602B0BDE8F0877E
:103FA0002D01074B00225A514FF0FF35F4E74FF037
:103FB000FF35F1E76FF00105EEE76FF00105EBE784
:103FC000C81900203C120020F0B599B00C461546E7
:103FD00088B10646037873B14C4B1B682BB14C4B30
:103FE0001B68586818B301F003FA00213046FFF748
:103FF00069FF00281FDC9CB123788BB1434B1B6900
:1040000033B1434B1B68986800283CD001F0F0F9AD
:1040100001212046FFF756FF002801DD012836D197
:1040200015B12B78002B54D1002019B0F0BD002021
:1040300004F074FBD9E70701DFF8D0C007EB0C03ED
:104040006646186859689A68DB680FC6002647F804
:104050000C602F4B1F682F49304601F027FA78601B
:1040600001A9304600F090FB049B43F00203049347
:104070004FF4E13101A800F021FB01AA314630469E
:1040800000F08CFBB7E7012004F048FBC0E7040117
:104090001E4FE31907F11006186859689A68DB6823
:1040A0000FC60026E6511A4B1C681B49012001F07F
:1040B000FDF9A06001A9012000F066FB4FF4E13199
:1040C00001A800F0FBFA01AA3146012000F066FBCE
:1040D000A6E701212846FFF7F5FE0028A4DD022807
:1040E000A2D00401094EA31906F1200518685968E9
:1040F0009A68DB680FC50023A351054B1C6806496D
:10410000022001F0D3F9E0608EE700BFC81900205B
:104110000C08002000CE000884CD00083B2810D8F1
:104120000C4B03EB00139B6873B110B51C6974B1A1
:1041300013460A460146074800EB0110C068A04735
:1041400010BD4FF0FF3070474FF0FF307047104602
:10415000F6E700BFC81900203B2814D810B50401A9
:104160000E4B1B5993B10D4C04EB0014A36883B1A3
:10417000DC688CB113460A460146084800EB011082
:10418000C068A04710BD4FF0FF3070476FF00100CE
:10419000F8E74FF0FF30F5E70020F3E7C8190020FB
:1041A0003B281AD80301104AD358CBB110B50446A6
:1041B00002EB00139B6863B19A6962B10A4B03EB8F
:1041C00000130146D86890472401074B00221A517A
:1041D00010BD0020F8E70020F6E74FF0FF307047F1
:1041E0006FF00100704700BFC81900203B2814D8A9
:1041F00010B504010E4B1B5993B10D4C04EB001488
:10420000A36883B1DC698CB113460A4601460848AD
:1042100000EB0110C068A04710BD4FF0FF307047A1
:104220006FF00100F8E74FF0FF30F5E70020F3E70B
:10423000C81900203B2811D808B5014603010A4AD5
:10424000D05850B102EB01139B684BB11A6A4AB1C6
:10425000054B03EB0113D868904708BD0020704759
:104260000120FAE70020F8E7C81900203B281BD8F6
:1042700038B5044600010D4B185880B103EB041308
:104280009B686BB15D696DB113460A4621460748CC
:1042900000EB0410C068A8470028C8BF404238BDE2
:1042A0000020F9E70020F7E700207047C819002038
:1042B0003B2809D80301074AD35833B102EB001059
:1042C000836823B15B6800E0002318467047002331
:1042D000FBE700BFC819002008B53B2817DC000128
:1042E000154B1B58D3B101B34FF6FF730B80002061
:1042F00048804FF400534B6001230B814881888133
:10430000C8814FF400730B614B648B6408BD01F0EE
:1043100001F8012303604FF0FF30F7E700F0FAFFE8
:10432000022303604FF0FF30F0E700F0F3FF0323B8
:1043300003604FF0FF30E9E7C819002070B44E6801
:10434000751C95FBF2F402FB14520C68944204D0E5
:1043500083554A60002070BC70474FF0FF30FAE789
:1043600008B50B46802200F5E0715C30FFF7E6FFF0
:1043700008BD08B50B46802200F5E471DC30FFF77C
:10438000DDFF08BD38B505460C46002003E0284691
:10439000FFF7EFFF013410B921780029F7D138BDBC
:1043A00038B505460C461F2909D85E21FFF7E1FF05
:1043B00004F14001C9B22846FFF7DBFF38BDFFF723
:1043C000D8FFFBE72DE9F041D0F80C80D0F8D031D0
:1043D000622B00F3D18000F5AE770E4604464269A9
:1043E00091421AD0A26996421BD00A2E36D0E269B9
:1043F00096423BD0626A964200F09080D4F8D42175
:10440000934240F0A280531CC4F8D431BE54D4F877
:10441000D0310133C4F8D031A4E0002AE2D0002525
:1044200008E0002AE1D0002504E0795D2046FFF78E
:1044300097FF0135D4F8D031AB42F6DC3146204647
:10444000FFF78EFF002384F85C31C4F8D431C4F840
:10445000D03118F0020003D1BDE8F0810025E9E772
:1044600031462046FFF785FF0020F5E7002AC1D03E
:10447000D4F8D4010028EFD0431EFD5C03E0431EB6
:104480003A5CFA540130D4F8D0318342F7DAD4F8E8
:10449000D421013AC4F8D421013BC4F8D03118F03A
:1044A0000200D9D09A4215D01F2D21D83449204678
:1044B000FFF768FF33492046FFF764FFD4F8D46163
:1044C000D4F8D031B34218DDB95D2046FFF768FF5C
:1044D0000136F5E72C492046FFF754FF1F2D01D97F
:1044E0000020B9E728492046FFF74CFF0020B3E73A
:1044F00026492046FFF746FFDCE71F2D09D824494F
:104500002046FFF73FFF23492046FFF73BFF0020EF
:10451000A2E720212046FFF72CFFF4E7002A3FF412
:104520006DAF002384F85C31C4F8D431C4F8D031C5
:1045300018F0020090D018492046FFF723FF002012
:104540008AE75A1CFB5CBB541346D4F8D4219A4228
:10455000F7DD531CC4F8D431BE54D4F8D031013344
:10456000C4F8D03118F002003FF476AF314620464F
:10457000FFF716FF00206FE74FF0FF306CE700BF3A
:104580008CCD00089CCD000888CD000894CD000893
:10459000A0CD0008A4CD0008A8CD0008F8B580B3D0
:1045A0000C4606460268C56805F002070A2914D0C1
:1045B0000D2917D012F0080F01D004F07F0415F078
:1045C000010517D121463046FFF7CAFEBFB121468B
:1045D0003046FFF7E5FE2F4611E012F4807FE9D068
:1045E0000D24E7E712F0400F0ED112F0800FE1D05A
:1045F0000A24DFE721463046FFF7E4FE002738466D
:10460000F8BD4FF0FF37FAE70027F8E7034638B167
:10461000D0F8C401D3F8C031C01A18BF01207047C8
:104620004FF0FF30704720B370B5044615460E4674
:10463000FFF7ECFF00281FDBD0B1002010E023447F
:1046400093F85C3033540130D4F8C03101335A420E
:1046500003F07F0302F07F0258BF5342C4F8C03119
:10466000D4F8C421D4F8C0319A4201D0A842E6DB84
:1046700070BD4FF0FF3070476FF00100F8E7014662
:1046800098B1D0F8CC31D0F8C821934210D0531C47
:10469000584203F07F0300F07F0058BF43420A44B2
:1046A00092F8DC00C1F8C83170474FF0FF30704716
:1046B0006FF001007047806D7047000010B484688F
:1046C00044F4007424F4F8348460816500220A4BB9
:1046D00003EBC2035B68002B0ADB8B4201D0013283
:1046E000F5E724F40074044B53F832301C43846023
:1046F00000205DF8044B70472CCA0008036823F4BF
:10470000BF6323F004030360436823F001034360A5
:10471000C36823F4507323F00303C360836823F456
:10472000E87343F480738360704758B310B5044650
:104730004FF4EC72002101F073FD4FF41641204656
:10474000FFF7BCFF2046FFF7D9FF042323617F2337
:10475000E361152363620323E3621C2323631A23AB
:1047600063631123E363132323641223A3621723D8
:104770002362162363640F23A3640023A361192318
:10478000A36310BD7047000008B50A46024900F057
:104790006EF9002008BD00BF02445C8008B50249E4
:1047A00000F065F9002008BD01445C402DE9F041AE
:1047B0000E4600230B704FF496424A604B7008225D
:1047C0008A600125CD608B7001F070FF80464949F9
:1047D00002F0DAF904463CE0203C4BE0632F15DCA4
:1047E000E4B2323C062C2FD8DFE804F0042E0A078E
:1047F0002E2E0D000023337026E00123337023E0BA
:104800000223337020E0032333701DE0776001350D
:104810001AE0E4B2303C232C15D8DFE804F04A4714
:104820001414141414141414141414141414141448
:104830001414143E1414141414141444123B1414B9
:1048400014410023737001352A49002002F09CF9BD
:104850000446002C48D000221146204602F060FA9F
:104860000746247801F0FCF92044437803F0030361
:10487000022BB1D06B1E042BE6D801A252F823F014
:10488000DD47000813480008B9480008BF48000881
:10489000C548000801237370D5E702237370D2E77F
:1048A00003237370CFE704237370CCE70523737081
:1048B000C9E706237370C6E7B7600135C4E7F76040
:1048C0000135C1E7E4B24E2C05D0532C06D0482C5C
:1048D00007D00135B8E70023B370FAE70123B370BE
:1048E000F7E70223B370F4E7404601F0D7F9002060
:1048F000BDE8F081B8CD000808B5FFF7DFFE08BDC0
:1049000060B1836823F4E0738360052907D006292A
:1049100009D007290BD043F480738360704743F0BC
:1049200040038360704743F080038360704743F027
:10493000C0038360704728B1022904D0826822F046
:10494000080282607047826842F008028260704705
:1049500068B1836823F0804323F03003836001292A
:1049600006D0022908D003290AD004290ED07047A6
:1049700043F030038360704743F010038360704757
:1049800043F0804343F010038360704743F080435B
:1049900043F030038360EAE720B121B102290BD054
:1049A000012912D07047826822F4001282600268E6
:1049B00022F4606202607047026822F46062026062
:1049C000826842F4001282607047826822F400120A
:1049D0008260026842F4606202601122C2631322A4
:1049E0000264DFE710B584B0044608466946FFF765
:1049F000DDFE01992046FFF77FFF9DF8011020465C
:104A0000FFF7A6FF02992046FFF77AFF0399204699
:104A1000FFF791FF9DF802102046FFF7BDFF04B09D
:104A200010BD30B599B004460D4601A9FFF7ACFEA4
:104A3000294601A8FFF7D6FF01AA00212046FFF76B
:104A4000ADFE19B030BD08B5FFF7AAFB08BD08B52B
:104A5000FFF72EFC08BD08B5FFF7C8FB08BD08B579
:104A6000FFF77AFB08BD08B5FFF758FB08BD0EB489
:104A700000B582B003AA52F8041B0192FFF7F6FBBF
:104A800002B05DF804EB03B07047000030B40A4D8B
:104A90002A68511C094C84FB0134CB17C3EBA413C7
:104AA000C82404FB13136968994203D005EB820202
:104AB00090602B6030BC7047041300201F85EB51C1
:104AC0000B4A536802EB83018868126893420CD04A
:104AD0000133084981FB0321DA17C2EBA112C82177
:104AE00001FB1232024B5A6070470020704700BF32
:104AF000041300201F85EB5138B504468B4B93F807
:104B000028331B2B04D01B2800F02181204638BD00
:104B1000864D05F54A70FCF753FB2B1883F82843A4
:104B200001300544002385F82833022804DD7F4B3B
:104B300093F82A334D2B0AD07C4B93F829335B2B07
:104B400077D07A4B002283F828232046DFE7062817
:104B5000F2D1764B93F82B33203B512B2AD8DFE848
:104B600003F04F2B2E29292929293A3D40292929AB
:104B70002929313437292929292929292929292984
:104B80002929292929292929292929292929292995
:104B90002929292929292929292929292929292985
:104BA000292943462929292929292929292929293E
:104BB0002929494C002325E06FF0320322E06FF0F1
:104BC00033031FE06FF034031CE06FF0350319E08E
:104BD0006FF0360316E06FF0370313E06FF0380321
:104BE00010E06FF039030DE06FF03A030AE06FF068
:104BF0003B0307E06FF03C0304E06FF03D0301E08E
:104C00006FF0310323F07F4424F0FF04474A92F809
:104C10002C33203B92F82D0320381B0403F47F0330
:104C20002343000284B244EA0300002382F82833BD
:104C30006DE701F015F82044437813F0030F2CD0F2
:104C40003A4B002283F82823A4F14103072B3FF6B7
:104C50005DAF01A252F823F0794C0008614D0008C5
:104C60007F4C0008854C0008974C0008914C0008C8
:104C70000D4B00088B4C00084FF0FF3047E76FF0FA
:104C8000030044E76FF0020041E76FF004003EE7E5
:104C90006FF005003BE7002039E77E2C01D00020B3
:104CA00035E72248002180F828130A4600F22A300E
:104CB00002F036F80138172843D8DFE800F00C542A
:104CC0000F121518424242421B1E212427422A2D50
:104CD000303339423C3F6FF0040018E76FF00800B2
:104CE00015E76FF0050012E76FF006000FE76FF0B1
:104CF00007000CE76FF0090009E76FF00A0006E70C
:104D00006FF00B0003E76FF00C0000E76FF00D0091
:104D1000FDE66FF00E00FAE66FF00F00F7E66FF0B9
:104D20001000F4E66FF01100F1E600BF041300205C
:104D30006FF01200EBE66FF01300E8E66FF014007E
:104D4000E5E60024094B83F828432046DFE6074BBD
:104D50001B2283F82823002483F829432046D6E623
:104D60006FF00100D3E66FF01500D0E604130020C9
:104D7000054B0022C3F88C23C3F8902383F89423B7
:104D8000C3F85C24704700BF04130020024B0122CB
:104D9000C3F88C23704700BF0413002008B50448F3
:104DA00001F094FA034B1B68986800F05FFC08BDA3
:104DB0009CCD00080C08002008B5044801F086FAD4
:104DC000034B1B68986800F051FC08BDA4CD000897
:104DD0000C08002008B50146044801F077FA044B9E
:104DE0001B68986800F042FC08BD00BF04CE0008B4
:104DF0000C08002008B50146044801F067FA044B8E
:104E00001B68986800F032FC08BD00BF0CCE00089B
:104E10000C080020F0B583B08DF80700B64BD3F82E
:104E20008C337BB1B54B1B6833B1C0B2FFF764FE66
:104E300030B1FFF72BFE03E09DF80700FFF726FED9
:104E400003B0F0BDAE48FCF7BBF9044607469DF839
:104E50000700FFF751FE05460028F1D0A64BD3F816
:104E60005C64002EECD110F1030F35D010F1040F6B
:104E70003ED010F1050F4BD0012849D010F1060F9C
:104E800052D0052850D0C31E012B5CD90A285FD010
:104E90000D285DD008286AD07F2800F0A38010F18B
:104EA000090F00F09F800B2800F0D3800028C7DB9B
:104EB00000F0D6FE2844437813F0970FC0D0C72CDB
:104EC000BEDC8D4AD2F890331A4492F89423002A1B
:104ED00000F0DB802246F3E0D3F89033002BAFDD07
:104EE000013B854AC2F890330120FFF773FFA7E723
:104EF000814BD3F89023134493F89433002B9FD025
:104F000001327D4BC3F890230120FFF773FF97E731
:104F1000794BD3F89003002892DDFFF75BFF764BC7
:104F20000022C3F890238BE7734BD3F8900303441C
:104F300093F89433002B83D0201AFFF75BFF6E4B5E
:104F4000C3F890437CE76C4B0122C3F85C2477E7FD
:104F5000694B0122C3F85C2406E0674B334493F8A5
:104F60009403FFF793FD0136BE42F6DB68E7624B20
:104F7000D3F8900300287FF763AF034605E05D1E7A
:104F80005D4A2A4482F8941301335B4A1A4492F82A
:104F900094130029F3D1631E574D2B44002283F84C
:104FA00094230138C5F890030120FFF713FFFFF7A2
:104FB000F5FED5F890331D4495F8942362B150491D
:104FC0001944504801F082F94F4B1B68986800F073
:104FD0004DFBFFF7F1FE33E701224C49104603F089
:104FE000B1FBF6E7444AD2F890331A4492F894237E
:104FF000002A3FF425AF013305E0581E3E49014425
:1050000081F8942301333C4A1A4492F89423002AED
:10501000F3D1631E384D2B4483F89423FFF7BEFE73
:10502000D5F890331D4495F8942362B1344919445E
:10503000344801F04BF9344B1B68986800F016FBBC
:10504000FFF7BAFEFCE601223049104603F07AFB76
:10505000F6E7294BD3F89003002801DDFFF7BAFEED
:10506000FFF79CFE05E001222849104603F06AFB89
:1050700027467C1E002FF6D1FFF79EFE1E4B002216
:10508000C3F8902383F89423DAE6591C1A4AC2F82D
:105090009013134483F894530A44002382F8943302
:1050A00001220DF10701104603F04CFBC8E6561C27
:1050B0001149881890F89403314481F89403013A17
:1050C0009342F4DD0C4E5A1CC6F89023334483F807
:1050D0009453FFF763FED6F89023511E06F56576CC
:1050E000A21A02323144012003F02CFBFFF764FEC8
:1050F0000120FFF77FFEA3E604130020080800202C
:105100009816002014CE00080C080020F0CB0008F0
:1051100000B583B0144B1B68586800F0B9FAFFF76C
:1051200089F880B1104B1B68586800F0B1FA012271
:105130000DF1070103F0FAFA0028EBDB9DF80700F8
:10514000FFF768FEE6E7094BD3F88C332BB9074B22
:10515000D3F85C0403B05DF804FB044B58681B688B
:10516000C01A18BF0120F5E70C0800200413002026
:1051700008B5FFF7CDFF044BD3F88C0300B908BD89
:10518000FFF79EFCFBE700BF0413002008B5044BAB
:105190000122C3F88C23FFF7BBFFFFF791FC08BD8A
:1051A0000413002070B505460E46124B0022C3F8CA
:1051B0008C23FFF7ADFFDDB1FFF782FC00242C70DC
:1051C00001E0FFF77DFC48B1731EA34206DD002815
:1051D000F7DD2855013400232B55F2E7002C03DCC2
:1051E000044BD3F85C0410B1FFF7C2FD012070BD81
:1051F0000020FCE70413002008B50246044801F033
:1052000065F8044B1B68986800F030FA08BD00BFD1
:1052100028CE00080C08002008B5064801F056F812
:1052200001210846FFF7E8FF034B1B68986800F070
:105230001DFA08BD34CE00080C08002008B5FFF7A1
:10524000ADFD202001F056F8FFF7B6FD08BD0000C7
:1052500010B50C4600280CDA002C04DB04F11E010A
:10526000074801F033F8074B1B68986800F0FEF917
:1052700010BD00F12801024801F028F8ECE700BF5A
:105280003CCE00080C08002008B5044801F01EF8C8
:10529000034B1B68986800F0E9F908BD44CE00088C
:1052A0000C08002008B5044801F010F8034B1B68F7
:1052B000986800F0DBF908BD4CCE00080C0800200F
:1052C000DFF834D0002103E00C4B5B58435004312D
:1052D0000B480C4B42189A42F6D30B4A02E00023CB
:1052E00042F8043B094B9A42F9D3FDF7ABF900F0C1
:1052F00081FCFDF74DF970470000012030D1000816
:1053000000000020B8110020B8110020B01D0020BE
:10531000FEE70000014B1868704700BF0C08002032
:1053200070B5002948D005460C4610B1836B002BA0
:1053300048D0626EB4F90C30D00740D4990530D50E
:105340002146284600F0BAF8E36A064633B1E1691F
:10535000284698470028B8BF4FF0FF36A3891A06A1
:105360003CD4216B41B104F14003994202D028465C
:1053700000F022FB00232363616C21B1284600F07A
:105380001BFB0023636400F081FA636E0022DB07DD
:10539000A2811FD5A06D00F073FC00F07DFA3046AD
:1053A00070BDA06D00F06EFCB4F90C30002BC7D1BD
:1053B000666E16F0010616D00026304670BD002B32
:1053C000FAD0BDE700F0E4F9626EB4F90C30D00712
:1053D000F5D4B3E7A06D00F057FCDBE72169284660
:1053E00000F0EAFABDE7A06D00F04EFC304670BD5B
:1053F000024B01461868FFF793BF00BF0C0800205E
:1054000070B5134682B00E4601AA1946044600F054
:1054100049FA00282CD00546204600F0E5F904465C
:1054200030B3436ED80715D4A389990524D51B48FA
:105430001B491C4A1C4BA581C4E90740C4E9091259
:10544000E681E362AB0510D4A06D00F01DFC2046A0
:1054500002B070BD11481249124A134BA581C4E92C
:105460000740C4E90912E681E362204602B070BD3C
:105470000024204602B070BDA06D00F003FC074A76
:10548000636E07480749A581C4E90742064AE262FC
:10549000DA07E681C4E90901E7D4D3E72566000805
:1054A0004966000885660008A5660008024B0A46A2
:1054B00001461868FFF7A4BF0C080020B1F90C30B2
:1054C0009AB22DE9F0410C461107804644D4626837
:1054D00043F40063002AA38159DDA56A002D53D04F
:1054E00000229BB2D8F80060E169C8F8002013F4EC
:1054F000805240F0838001234046A847421C4AD096
:10550000A389A56AE1695B0705D56268236B801AE8
:105510000BB1E36BC01A024600234046A847471C64
:1055200045D0B4F90C302269226023F400630022D4
:10553000A381DB04626000D52065216BC8F80060A0
:1055400011B304F14003994202D0404600F034FA0E
:1055500000202063BDE8F0812669AEB12568266091
:1055600092070CBF63690023AD1BA3600AE02B46C2
:105570003246676AE1694046B8470028A5EB000556
:1055800006442BDD002DF2DC0020BDE8F081E26B4B
:10559000002AA2DCF8E7D8F80030002BB0D01D2B91
:1055A00001D0162B2CD1C8F800600020EDE7D8F808
:1055B00000101D291AD8154BB4F90C20CB40DB4341
:1055C00013F0010314D1256922F40062C4E90053E9
:1055D000D504A281B1D50029AFD1ADE7A38943F0AD
:1055E0004003A3814FF0FF30BDE8F081B4F90C20F7
:1055F00042F04002A2814FF0FF30C6E7206D82E703
:10560000A38943F04003A381BFE700BF010040200E
:1056100038B50D46044608B1836BA3B1B5F90C004B
:10562000B8B16B6EDB0701D481051AD52046294637
:10563000FFF744FF6B6EDA07044602D4AB899B0583
:105640000AD5204638BD00F0A3F8B5F90C000028B3
:10565000E7D10446204638BDA86D00F015FB204672
:1056600038BDA86D00F00EFBE0E700BF20B1054B90
:1056700001461868FFF7CCBF034B0449186800F0D7
:105680008FBA00BF0C08002074CE00081156000825
:1056900038B51B4D2B6804460BB19A6BA2B1626EF4
:1056A000B4F90C30D1070AD413F4007310D0B4F954
:1056B0000E503BB9A06D00F0E7FA284638BDBBB1EB
:1056C000B4F90E50284638BD184600F061F8E6E7F8
:1056D000A06D00F0D7FAB4F90C30626E43B1D20776
:1056E000B4F90E50EED403F40073002BEAD1E1E7D5
:1056F0002B6809211960D3074FF0FF35DAD5E1E7B0
:105700000C08002010B5002304468181C281C0E945
:10571000003383604366C0E904338361194608227D
:105720005C3000F07DFD07480749084A084BE362FA
:10573000C4E90740C4E9091204F15800BDE810406B
:1057400000F09CBA256600084966000885660008D6
:10575000A5660008014900F023BA00BF21530008E4
:1057600070B54A1E682505FB02F50E4605F1740169
:1057700000F09CFA044640B100210C30666005F14F
:1057800068022160A06000F04BFD204670BD00BFA4
:1057900010B50446124800F075FAA26BD2B904F5B0
:1057A0003B731048C4F8E8320321C4F8E022E063F8
:1057B000C4F8E41260680421FFF7A4FF0122092164
:1057C000A068FFF79FFF02221221E068FFF79AFF0F
:1057D0000123A3630248BDE8104000F055BA00BFA2
:1057E000941D00205557000870B50646244800F067
:1057F00049FA244B1D68AB6B83B305F53875D5E9C1
:105800000134013B05D525E0013B5A1C04F1680435
:1058100020D0B4F90C20002AF6D100251A4BE36001
:1058200004F15800656600F029FA154800F02CFADA
:105830002560C4E90155C4E90455A561294608223B
:1058400004F15C0000F0ECFCC4E90C55C4E911550E
:10585000204670BD2C682CB12546D0E72846FFF7BE
:1058600097FFCAE704213046FFF77AFF0446286015
:105870000028F1D1024800F007FA0C233360E7E773
:10588000A81D002074CE00080100FFFF014800F0B1
:10589000F9B900BFA81D0020014800F0F5B900BF0C
:1058A000A81D00200B78722B30B431D0772B2AD072
:1058B000612B04D01623036030BC002070474FF4E6
:1058C000027501244FF4847011F8013F8BB1622BF3
:1058D00016D0782B11D02B2BF6D111F8013F20F0E8
:1058E0001C0024F0030440F0100044F00204002BDC
:1058F000EDD12C43146030BC704744F40064E3E7FE
:1059000044F48034E0E74FF4C06501240820DBE76D
:1059100000252C460420D7E7F8B5244F0C46064650
:1059200000F0C8FCBB685D68C4F57E610F3125F0EE
:105930000305294421F47F6121F00F01A1F5805472
:10594000B4F5805F07DB0021304600F051FDBB68F5
:105950002B44984204D0304600F0B2FC0020F8BD41
:105960006142304600F044FD01300DD0104BBA6862
:1059700019682D1B45F001053046091B556019605B
:1059800000F09EFC0120F8BD0021304600F030FD03
:10599000BA68831A0F2BDEDD064C0549246843F0F4
:1059A0000103001B53600860D5E700BFA40D002071
:1059B00064170020AC110020002953D0F8B50C4624
:1059C000064600F077FC54F804CC714F2CF001012E
:1059D000A4F108056B18B8685A68984222F00302CF
:1059E00053D01CF0010F5A6003EB02003BD154F876
:1059F00008CC4068A5EB0C0507F1080EAC687445AF
:105A0000614400F0010075D0D5F80CC0C4F80CC09A
:105A1000CCF8084060B341F001036B606950B1F508
:105A2000007F50D34B0A042B70D88B0903F1390443
:105A3000E40003F1380238193B590838984278D00D
:105A40005A6822F003028A4271D99B689842F7D1C2
:105A5000C368C5E902039D60C5603046BDE8F840F3
:105A600000F02EBC7047406800F001000028D2D141
:105A70009868484C1144A04241F0010262D0DB68B2
:105A8000C36098606A606950C9E71CF0010F0A445E
:105A900007D154F8083CED1A1A44D5E90213CB603B
:105AA00099603D4B1B6842F0010193426960BD6003
:105AB00004D83A4B30461968FFF72EFF3046BDE850
:105AC000F84000F0FDBBC90878684A1C0123891022
:105AD0008B40034307EBC20157F832007B60083963
:105AE000C5E9020147F83250C5603046BDE8F840CC
:105AF00000F0E6BB002845D10A44D3E9021342F086
:105B00000100CB6099606860AA50D7E7142B08D9D0
:105B1000542B1ED80B0B03F16F04E40003F16E024B
:105B200089E703F15C04E40003F15B0283E71846B4
:105B30008EE793107968012202FA03F30B437B602E
:105B4000034686E7C7E90455C5E902006A60695063
:105B5000B4E7B3F5AA7F06D8CB0B03F17804E400D1
:105B600003F1770267E740F25452934206D88B0C58
:105B700003F17D04E40003F17C025CE74FF47E74E2
:105B80007E2258E741F001026A60196096E700BF83
:105B9000A40D0020AC0D0020B011002094170020AF
:105BA0002DE9F84310F538771FD0884606464FF0A8
:105BB0000009D7E90154013D11D4A389012B05F156
:105BC000FF352146304606D9B4F90E30013302D0F4
:105BD000C04749EA00096B1C04F16804EDD13F6835
:105BE000002FE6D14846BDE8F883B9464846BDE8EF
:105BF000F88300BF70B50D4E0D4D761BB61006D064
:105C00000024013455F8043B9847A642F9D1094EC7
:105C1000094D761B06F09AFEB61006D0002401341A
:105C200055F8043B9847A642F9D170BD24D100082D
:105C300024D100082CD1000824D10008044B054AC7
:105C40001B685B6B002B08BF134693F82801704755
:105C50000C080020380C0020D0F8EC00704700BF82
:105C6000044B054A1B685B6B002B08BF1346D3F837
:105C7000EC0070470C080020380C0020704700BF73
:105C8000704700BF704700BF704700BF024B01461E
:105C9000186800F00BB800BF0C080020024B01464A
:105CA0001868FFF789BE00BF0C0800202DE9F04FEF
:105CB00001F10B05162D83B0064623D8102900F2FA
:105CC000B98000F0F7FA102518230220C54F3B4495
:105CD000A3F108025C68944200F06681636823F0D7
:105CE00003032344D4E902515A68E96042F00102F7
:105CF0008D6030465A6000F0E3FA0834204603B065
:105D0000BDE8F08F35F0070500F19480A94200F25C
:105D1000918000F0CFFAB5F5FC7FC0F083816B0A6B
:105D200000F08F80042B00F24681AB0903F13900AB
:105D300003F1380CC300AB4F3B44A3F108015C688E
:105D4000A14206D10CE0002A80F21D81E468A14244
:105D500006D0636823F003035A1B0F2AF3DD604665
:105D60003C69DFF894C2644571D0636823F0030393
:105D70005A1B0F2A00F34481002AC7E904CC80F2A1
:105D80002681B3F5007F80F06981DB08591C7A68B1
:105D900057F83180C4F808804FF0010E9B100EFABE
:105DA00003F307EBC10E1343AEF10802E2607B6020
:105DB00047F83140C8F80C408210012494409C42BE
:105DC0004BD81C4206D120F0030064001C4200F1B5
:105DD0000400FAD007EBC009CE468046DEF80C304E
:105DE0009E4507D122E1002A80F22981DB689E4589
:105DF00000F01C81596821F003014A1B0F2AF2DDD3
:105E0000D3E9028E5C1945F001055D6042F00105A1
:105E1000C8F80CE03046CEF80880C7E90444C4E96D
:105E200002CC65605A50019300F04AFA019B03F1DD
:105E3000080463E700240C232046336003B0BDE868
:105E4000F08F4FF4007340204FF03F0C73E77B68F6
:105E50008210012494409C42B3D9BC68636823F04B
:105E60000309A94503D3A9EB05030F2B7BDC5E4B8C
:105E7000DFF888A11A68DAF80030013305EB020870
:105E800000F0488108F5805808F10F0828F47F6871
:105E900028F00F084146304600F0AAFAB0F1FF3F63
:105EA000834600F0048104EB0900584500F2FD80B0
:105EB0004E4A13684344136000F04D81DAF8001035
:105EC00001311BBFABEB00001B18CAF800B0136018
:105ED0001BF0070300F03481C3F10801C3F58053C0
:105EE0008B440833D844C8F30B08A3EB0808414699
:105EF0003046019200F07CFA431C019A00F0468182
:105F0000A0EB0B01414441F001011368C7F808B050
:105F10004344BC42CBF80410136015D0B9F10F0F05
:105F200040F230816068A9F10C0121F0070100F016
:105F3000010004EB010C08434FF0050E0F296060CF
:105F4000CCE901EE00F23A81294A2A481168BC687E
:105F50008B42016888BF136062688B4222F00302A3
:105F600088BF0360A7E0621943F0010345F0010513
:105F700065603046BA60536000F0A2F908342046EC
:105F800003B0BDE8F08F2344E1685A68A56842F089
:105F90000102E96030468D605A6000F091F90834E2
:105FA000204603B0BDE8F08FDC68A34208BF023092
:105FB0003FF4D6AE92E6142B71D9542B00F2AD808B
:105FC0002B0B03F16F0003F16E0CC300B3E6234407
:105FD00030465A6842F001025A60083400F070F905
:105FE0008CE600BFA40D0020941700206417002049
:105FF0008C17002090170020AC0D0020AC11002061
:10600000611945F0010E42F00105C4F804E0304684
:10601000C7E90411C1E902CC4D60E25000F050F92B
:1060200008346BE6E80805F108034FE608F10108BB
:1060300018F0030F0EF1080E7FF4D0AE52E01944B1
:106040001C464A68DB6854F8085F42F001024A6067
:106050003046EB609D6000F033F94FE65A0A042A9F
:1060600035D9142A6FD802F15C01C9005B3207EB05
:10607000010E7958AEF1080E8E4558D04A6822F0CC
:1060800003029A4202D989688E45F7D1D1F80CE013
:106090007B68C4E9021ECEF80840CC608CE603F1B0
:1060A0005C0003F15B0CC30045E6BC4272D0BC68E7
:1060B000626822F003029542A2EB050302D80F2B7F
:1060C0003FF751AF304600F0FBF8002416E69A097E
:1060D00002F13901C9003832C9E7D9F80090994571
:1060E00040F0838010F0030FA9F1080300F1FF30A6
:1060F000F3D17B6823EA04037B6064009C423FF693
:10610000ACAE1CB9A9E6640008F104081C42FAD040
:1061100040465FE608F11008BCE6B3F5AA7F26D832
:10612000EB0B03F1780003F1770CC30003E67B6807
:1061300092104FF0010808FA02F213437B60A8E7BF
:106140004FF48053CEE6542A29D81A0B02F16F017E
:10615000C9006E328BE7C0F30B0100297FF4AEAEAD
:1061600009EB0802B96842F001024A60ECE640F22D
:10617000545293421CD8AB0C03F17D0003F17C0C0C
:10618000C300D8E50123CBF804309BE701214FF091
:106190000008BAE6164A1368434413608EE6B2F567
:1061A000AA7F14D8DA0B02F17801C90077325EE7D2
:1061B0004FF47E737F204FF07E0CBCE504F10801A4
:1061C00030460192FFF7F8FB019A1368BCE640F2F3
:1061D00054518A4205D89A0C02F17D01C9007C32E3
:1061E00045E74FF47E717E2241E77B6885E700BF7B
:1061F0006417002082B049B15AB16BB113780B60BB
:106200001278101C18BF012002B0704701A9002AA3
:10621000F3D1104602B070476FF00100F4E700BF01
:10622000F0B4860743D0541E002A3ED0CAB20346BB
:1062300002E014F1FF3438D303F8012B9D07F8D1A5
:10624000032C2BD9CDB245EA05250F2C45EA05458F
:1062500016D9A4F110073F0903F1200606EB071633
:1062600003F1100242E9045542E902551032B242EC
:10627000F8D104F00F040137032C03EB07130DD9F9
:106280001E462246043A032A46F8045BFAD8221F27
:1062900022F003020432134404F003042CB1C9B207
:1062A0001C4403F8011B9C42FBD1F0BC7047144610
:1062B0000346C5E70148FFF7E5BC00BF981D002075
:1062C0000148FFF7E1BC00BF981D00200FB400B5E6
:1062D000074983B004AB086853F8042B8168019325
:1062E00002F03EFA03B05DF804EB04B0704700BF63
:1062F0000C080020034B1B6801469A68184605F0FD
:10630000D3BD00BF0C08002070B5054688B0084614
:106310000C46FAF755FF224AAB6B04940126441C45
:1063200004A90692022203940590AC680796CDE971
:1063300001121BB3616EB4F90C30CE079AB201D4CE
:10634000900525D5910406D4626E43F4005322F4DF
:106350000052A3816266284601AA214604F0EAFFA2
:10636000636E00280CBF0A254FF0FF35DA0702D410
:10637000A3899B0506D5284608B070BD2846FFF7BF
:1063800007FAD7E7A06DFFF77FFC284608B070BD7D
:10639000A06DFFF777FCB4F90C309AB2D2E700BFDA
:1063A00084CE0008024B01461868FFF7ADBF00BF5E
:1063B0000C0800200B4B0C481968D1E92A2330B493
:1063C0000A4C00FB02F004FB0300A2FB0423541C54
:1063D000034443F1000525F00040C1E92A4530BCE3
:1063E000704700BF0C0800202DF451582D7F954CAC
:1063F00038B5074C0023054608462360FCF704F92E
:10640000431C00D038BD2368002BFBD02B6038BD67
:10641000AC1D00202DE9F0435D4C256883B0044697
:10642000884616461F4615B1AB6B002B7ED0022E58
:1064300005D0012E00F2A980002FC0F2A680636E65
:10644000DA0735D521462846FFF7E2F8216B41B13E
:1064500004F14003994202D02846FFF7ADFA002329
:106460002363B4F90C3000221806A261626061D483
:1064700023F44A6323F00303022EA3811FD10025D6
:10648000616E002004F1430243F00203A060C907DB
:106490004FF00100A3812260C4E9042004D49B05CD
:1064A00002D4A06DFFF7F0FB284603B0BDE8F083EF
:1064B000A3899B05C6D4A06DFFF7E4FBC2E701AB3F
:1064C0006A462146284605F0D7F8A3891843A081DB
:1064D000002F36D1009F3846FFF7D8FB80460028B2
:1064E00042D0A38943F08003A381AB6B7BB3009AB6
:1064F000B4F90C30C4F80080BA421CBF43F4006306
:10650000A381012E04BF43F00103A3819BB213F0CA
:106510000802C4E904871ED1A260656E15F001056A
:10652000BDD00025284603B0BDE8F0832846FFF71C
:106530002FF97CE721692846FFF73EFAB4F90C30C1
:1065400096E7B8F1000FC6D0AB6B002BCFD1284631
:10655000FFF71EF9CBE7DA0704D57F420022A761D7
:10656000A260DAE7A760D8E7DDF80090B94504D16A
:10657000B4F90C304FF0FF3582E74846FFF786FB51
:1065800080460028F4D04F46ABE74FF0FF358BE74D
:106590000C0800200CB430B5214B00299DB01C68BC
:1065A00038DB4FF4027302900690ADF8143021A846
:1065B00019D001390346209A0491079101904FF6B2
:1065C000FF7502A92046ADF8165000F0C1FB421C31
:1065D00001DA8B232360029B00221A701DB0BDE8F4
:1065E000304002B0704703460491079101904FF686
:1065F000FF75209AADF8165002A9204600F0A8FBBE
:10660000431C04DB1DB0BDE8304002B070478B2353
:106610002360F7E78B2323604FF0FF30F2E700BFE2
:106620000C08002010B50C46B1F90E1005F074FCF2
:10663000002803DB236D0344236510BDA38923F4E5
:106640008053A38110BD00BF2DE9F0411646B1F97A
:106650000C201F46D3050C460546B1F90E1007D590
:106660000022022304F0F2FFB4F90C20B4F90E105A
:1066700022F48052A2813B4632462846BDE8F041D2
:1066800003F0FCBD10B50C46B1F90E1004F0DEFFAE
:10669000A389421C0EBF23F4805343F4805320652A
:1066A000A38110BDB1F90E1003F074BE024B014678
:1066B000186800F003B800BF0C08002070B506464B
:1066C00008460C46FAF77CFD451C29463046FFF784
:1066D000EDFA064618B12A462146FAF767FB30461E
:1066E00070BD00BF4FF0010C2DE9F041644600265B
:1066F0004FF0FF3533198B4200EB05070DD23F5D9C
:1067000010F803E0BE452DD21E460124A3EB050C74
:1067100033198B4200EB0507F1D34FF00108C2F8A3
:1067200000C0444600264FF0FF3733198B4200EB80
:10673000070C0ED21CF804C010F803E0E64518D987
:106740001E460124A3EB070833198B4200EB070C0C
:10675000F0D30137681C874224BFC2F80080384656
:10676000BDE8F0810CD04FF0010C3546644666441C
:10677000C0E70BD04FF00108374644464644D4E703
:10678000644512BF01341E460124B3E7444512BFDD
:1067900001341E460124C8E72DE9F04FADF2144D37
:1067A000914605468B461046194603AA1C46FFF73C
:1067B00099FF03AB80460DF20C4243F8044F93421D
:1067C000FBD154B1631E09F1FF3204A812F8011F76
:1067D00040F8213013F1FF33F8D20399424649447F
:1067E000484604F0C1FF00286ED108F1FF33019341
:1067F0004B448246009323460746544658469A46E1
:1068000007EB0A06321A00212844FAF749FD00284E
:1068100055D1002E53D0AB1904AA13F8013C52F8FD
:1068200023304BB124B1039A9A4201D9AAEB020357
:106830001F4400243046E3E7444523460AF1FF3C69
:1068400038BF4346634513D2FA1819F8030015F808
:1068500002E086452A4409EB030106D02BE011F83B
:1068600001EF12F8010F864525D101336345F6D3B8
:10687000019B4445194680F08780FB18009AE85C2C
:10688000127882422B447FD1009804F1FF3B06E04E
:1068900010F801ED13F801CDE64503D111464A1E6B
:1068A0009345F5D101348C4270D8039C304627447F
:1068B000AAEB0404A4E7C8F101021744B8E70020DA
:1068C0000DF2144DBDE8F08FA4EB0803434538BF2B
:1068D0004346013308F1FF37039309EB070358469A
:1068E0004FF0000AC34698460AEB0406321A00210C
:1068F0002844FAF7D5FC0028E1D1002EDFD0AB19EF
:1069000004AA13F8013C52F82330A3BB611E8B4547
:1069100015D20AEB0B0219F80B3015F802C09C4592
:106920002A4409EB0B005B4606D027E010F801EF84
:1069300012F801CFE64521D101338B42F6D37B1CFF
:1069400012D00AEB070398F80000E95C884205EBD7
:1069500003020FD1434605E013F8010D12F8011DA3
:10696000884207D14B45F7D105EB0A000DF2144DD3
:10697000BDE8F08F039B9A443046B5E7CBF10102A6
:1069800092449A443046AFE741468BE7E81997E7CF
:106990002DE9F04F02780E4685B0054609788AB396
:1069A000A1B18446741C0846012701E068B11C4669
:1069B000904214BF002707F0010723461CF8012F5F
:1069C00013F8010B002AF1D1F0B91FB1284605B028
:1069D000BDE8F08F681C05F097FC0746A0B1A41B2A
:1069E000012C16D0254485422CBFA5EB00094FF0A1
:1069F00001091F2C0FD9234632464946FFF7CCFE2A
:106A00000546E3E70029E1D00025284605B0BDE8AA
:106A1000F08F0546DAE703AA21463046FFF762FE0B
:106A20000399804602463144304604F09DFE00281A
:106A30004ED108F1FF330193F318824605460093C7
:106A40004846B3466619321A00213844FAF728FC42
:106A50000028D9D1002ED7D0D045434638BF534661
:106A60009C4212D95A191BF80310B85C81423A446F
:106A70000BEB030C06D072E01CF8010F12F8011F9B
:106A800088426CD101339C42F6D1019BD045194616
:106A900077D9EB18009AF85C127882423B4470D1A7
:106AA00000980AF1FF3906E010F801ED13F801CD66
:106AB000E64503D111464A1E4A45F5D10AF1010ABD
:106AC0008A454AD8039B30461D44A4EB030AB9E724
:106AD000A4EB0803434538BF4346013308F1FF3AAE
:106AE000039306EB0A0348460025B3469946661908
:106AF000321A00213844FAF7D3FB002884D1002E43
:106B000082D0444514D908EB05021BF80830B85C64
:106B100098423A440BEB0801434606D027E011F8AF
:106B200001CF12F8010F844521D101339C42F6D1E7
:106B3000BAF1FF3F11D005EB0A0399F80020F95C88
:106B400091423B4419D14A4605E012F8010D13F871
:106B5000011D884211D15A45F7D13D4436E7C8F1AD
:106B6000010215441D444FF0000A30466AE7C8F19F
:106B7000010215441D443046B9E7039B30461D44CD
:106B8000B5E741469AE700BF024B1A6801235C3221
:106B900000F002B80C080020F0B420B307460D4600
:106BA00017F8016B01E0A64216D015F8014B002C36
:106BB000F9D1EEB13E460C4616F8015B00E073B128
:106BC00014F8013B9D42FAD15DB100233B70166081
:106BD00006463046F0BC704763B13846DEE73746BC
:106BE000E8E72E46F3E710680028D7D10646F0E71D
:106BF0001660EEE7176006460370EAE72DE9F84FE6
:106C00000E468046174699460D4600E025462C461E
:106C10000A9814F801BBFFF71FF85844417811F0A7
:106C20000801F3D1BBF12D0F57D0BBF12B0F04BFDF
:106C300095F801B0AC1CB9F1000F04D0B9F1100FF8
:106C400050D0CC4605E0BBF1300F55D04FF00A09CB
:106C5000CC4600290CBF6FF0004E4FF0004E0025CF
:106C6000BEFBFCF328460CFB13EA05E029D00CFB25
:106C70000020012514F801BBABF13002092A05D927
:106C8000ABF14102192A0BD8ABF1370291450FDD68
:106C9000B5F1FF3FEED08342E8D24FF0FF35E9E790
:106CA000ABF16102192A03D8ABF157029145EFDC31
:106CB0006B1C0BD001B140420FB14DBB3E60BDE833
:106CC000F88F9245D3DA4FF0FF35D3E72223C8F887
:106CD0000030FFB1661E7046F0E7AC1C95F801B0BD
:106CE0000121A8E7BBF1300FABD1237803F0DF031C
:106CF000582B06D0CC46ACE7237803F0DF03582BA3
:106D00000AD14FF0100C94F801B0E1460234A0E72C
:106D10008646DFE77046D2E74FF00809CC4698E791
:106D200030B5084C084B25686C6B83B0002C08BF4D
:106D30001C46009413460A4601462846FFF75EFFAC
:106D400003B030BD0C080020380C0020000000000B
:106D50002DE9F04FD7B00C46069193460993039066
:106D600004F066FC036817931846FAF729FAA3891A
:106D700016901F0603D52369002B00F055870023CA
:106D80005E469FED8F7B1093CDE92B331593CDE9B4
:106D900019331B93189305932DAB2A939946337897
:106DA0008DED127B002B00F0CE82252B344602D1D4
:106DB0001CE0252B03D014F8013F002BF9D1A51BB3
:106DC00085B1DDE92B3201332A44072BC9F8006075
:106DD000C9F80450CDE92B327CDC09F10809059B88
:106DE0002B4405932378002B00F0AD8200236778B5
:106DF000079398468DF88B3004F1010B4FF0FF3A62
:106E00002B250BF1010BA7F120035A2B00F2E48391
:106E1000DFE813F0A503E203E203A003E203E203C9
:106E2000E2038103E203E203B503B003E20372016C
:106E30005801E2033B03C600C600C600C600C600F8
:106E4000C600C600C600C600E203E203E203E20396
:106E5000E203E203E2034003E2037701F0024003AE
:106E600040034003E203E203E203E203EB02E20336
:106E7000E2038400E203E203E203C202E203CE0380
:106E8000E203E203AC02E203E203E203E203E20311
:106E9000E203E203E2034003E2037701DA00400386
:106EA00040034003C103DA005B00E2031E03E20378
:106EB000060386002B035B00E203C2025D0029018A
:106EC000E203E2033801E2035D0048F020089BF88A
:106ED000007096E72AAA0699039805F0BBFA80B9D4
:106EE0000DF1B4097BE72AAA5946504605F0B2FADB
:106EF000002801F0C5800A9B1BB10A990398FEF790
:106F00005BFD069B9B8913F0400F059B18BF4FF05C
:106F1000FF330593059857B0BDE8F08F48F010088F
:106F200018F0200F00F07385099C073424F0070344
:106F3000D3E9004503F10802099228F48063002296
:106F400000218DF88B10BAF1FF3F56A9049100F093
:106F5000A78454EA050123F080085BD1BAF1000F41
:106F600040F09687002A40F01F8513F0010356AECB
:106F7000089302D0302306F8013D00230A930F93B3
:106F800014931193089B9DF88B205345B8BF53462B
:106F90000493002A00F0C880049B01330493C3E0EB
:106FA000A7F1300300221BF8017B02EB820203EB06
:106FB0004202A7F13003092BF5D9079223E700BF5E
:106FC000000000000000000043469E0640F11782CA
:106FD000099C073424F00704D4E9000104F10802F5
:106FE000099204460D46002871F1000205DA2D22AF
:106FF000644265EB45058DF88B2056AABAF1FF3F38
:10700000049200F0E38654EA05014FF0010223F0F8
:107010008008A3D0012A00F04784022A00F0EF8202
:1070200056A900E03146E20842EA4572E80804F059
:10703000070305461446303354EA050201F8013CC3
:1070400001F1FF36EED118F0010F00F0E882302B8D
:1070500000F0E582049A02393023521A06F8013C06
:1070600008920E4689E743469E0640F1A682099C97
:10707000073424F0070202F10801D2E90045099122
:1070800001225DE7B64B159318F0200F00F07481D4
:10709000099C073424F00703D3E9004503F10802F3
:1070A000099218F0010F09D054EA050306D03023E5
:1070B0008DF88D7048F002088DF88C3028F48063CC
:1070C00002223DE79BF800702A2F0BF1010201F02C
:1070D000EB82A7F13003092B93464FF0000A3FF6ED
:1070E00092AE1BF8017B0AEB8A0A03EB4A0AA7F16E
:1070F0003003092BF5D986E69BF8007048F00408A8
:107100007FE60998002301688DF88B301A468DF8C8
:10711000F4100123011DCDE9083104930A9292462F
:107120000F92149211923DAE18F002030B9302D00D
:10713000049B0233049318F084032C9C0E933FD1DC
:10714000079B04995D1A002D3ADD102D2B9A29DD3D
:1071500049462046B14610232097039C069E04E032
:10716000103D102D01F1080118DD01327D4F103066
:10717000072ACDE92B20C1E90073F1DD2AAA3146A7
:1071800020460C9305F066F900287FF4B4AE103D5C
:10719000102DDDE92B202DA90C9BE6DC209F4E460F
:1071A0000446894601326F4B2C44072ACDE92B2433
:1071B000C9E9003500F37C859DF88B2009F10809A9
:1071C00072B12B9A013201340DF18B000121072A93
:1071D000CDE92B24C9E9000100F3738309F1080903
:1071E0000B9B6BB12B9B0133023423A90222072B8B
:1071F000CDE92B34C9E9001200F36F8309F10809C6
:107200000E9B802B00F07982089BAAEB0305002DD2
:1072100035DD102D2B9A544B26DD49462046B146CC
:107220004FF0100A069E1C4604E0103D102D01F19F
:10723000080115DD01321030072ACDE92B20C1E904
:10724000004AF2DD2AAA3146039805F003F9002826
:107250007FF451AE103D102DDDE92B202DA9E9DC86
:107260004E4623468946044601322C44072ACDE97E
:107270002B24C9E9003500F33C8309F1080918F40F
:10728000807F40F0DB812B9B089AC9F800600133B6
:107290001444072B2C94C9F804202B9300F3A182EB
:1072A00009F1080918F0040F33D0079B049A9D1ABE
:1072B000002D2EDD102D2B9B21DD1026039FDDF8E8
:1072C000188004E0103D102D09F1080917DD013385
:1072D000244A1034072BCDE92B34C9E90026F1DD0F
:1072E0002AAA4146384605F0B5F800287FF403AED7
:1072F000103D102DDDE92B340DF1B409E7DC01332D
:10730000184A2C44072BCDE92B34C9E9002500F39A
:10731000A583059B079A04998A42ACBF9B185B180A
:107320000593002C40F0258200232B930A9B1BB170
:107330000A990398FEF740FB0DF1B4095E463378D5
:10734000002B7FF432AD2C9B002B3FF4DAAD069C72
:1073500003982AAA214605F07DF8A389D3E500BF4A
:1073600098CE0008CCCE0008DCCE0008AE4B1593BA
:1073700018F0200F7FF48CAE099A18F0100F02F16C
:10738000040340F0798318F0400F099A00F07083ED
:1073900014880993002584E6099B1E6800258DF852
:1073A0008B501C1D002E00F07384BAF1FF3F00F0DB
:1073B0005F86524629463046F9F772FF0A90002848
:1073C00000F09A870A9B9B1B0893AA4623EAE37363
:1073D00009940493CDF828A0CDF83CA0CDF850A096
:1073E000CDF844A09DF88B20D3E548F008089BF821
:1073F000007006E548F010039E063FF5E9AD0999D7
:10740000DD0601F1040200F151835C06099940F1A7
:107410004A83B1F900400992E51720462946E2E582
:10742000099A18F0200F52F8043B099240F0458366
:1074300018F0100F40F07C8518F0400F40F02E86B9
:1074400018F4007F00F07485059A1A705E4676E79E
:107450009BF800706C2F03BF9BF8017048F0200868
:107460000BF1010B48F01008CBE409996F4B0C6845
:10747000159347F630020431ADF88C2048F0020332
:1074800009910025022278275AE548F080089BF8E8
:107490000070B6E4099C073424F0070494ED007BE7
:1074A00052EC171B22F000431D938DED1C7A08341B
:1074B000DDE91C014FF0FF325D4B09948DED127B2D
:1074C000F9F73EFF002840F0FF824FF0FF32584BA3
:1074D000DDE91C01F9F7CCFA002840F0F582002222
:1074E0000023DDE91201F9F7B9FA002840F0E3863C
:1074F0009DF88B204F4E504B0020032104910A90A1
:1075000028F08008472FD8BF1E46089182460F906A
:10751000149011903DE5039F384604F089F84368C4
:1075200018931846F9F74CFE1B900446384604F0B1
:107530007FF883681A93002C3FF4C9AC9BF8007065
:10754000002B3FF45EAC1B78002B3FF45AAC48F4A0
:10755000806856E448F001089BF8007051E49DF8FB
:107560008B309BF80070002B7FF44BAC20238DF800
:107570008B3046E48DF88B509BF8007041E4099BFA
:107580009BF800701A680792002A03F10403C0F206
:107590005A83099335E49BF80070682F03BF9BF86A
:1075A000017048F400780BF1010B48F0400828E422
:1075B00048F010039E063FF55AAD099ADD0602F128
:1075C000040100F161825C06099A40F15A82148834
:1075D000099100250122B3E4002F3FF4B4AE00234B
:1075E00001211A4604918DF8F4708DF88B300A93BE
:1075F0009A460F931493119308913DAE94E5159814
:1076000056AE230904F00F0143EA05732A091C460C
:107610001546435C06F8013D54EA0503F1D1049B8D
:107620009B1B0893A9E400BFACCE000898CE0008CD
:10763000FFFFEF7F8CCE000888CE0008652F40F357
:10764000DC8000220023DDE91201F9F7FDF90028B2
:1076500000F060812B9BAD4AC9F800200133013452
:107660000122072BCDE92B34C9F8042000F33C8418
:1076700009F10809249B109A2C9C934280F2E9811D
:107680002B9B179AC9F80020169AC9F804200133D9
:107690001444072BCDE92B3400F3EE8209F10809DD
:1076A000109B5D1E002D7FF7FDAD102D2B9A984B82
:1076B00040F30384194610262346039FDDF818A0E3
:1076C0000C4605E009F10809103D102D40F3F28346
:1076D00001321033072ACDE92B23C9E90046F1DD39
:1076E0002AAA5146384604F0B5FE00287FF403ACC0
:1076F000DDE92B230DF1B409E6E7079B049A9D1AF7
:10770000002D7FF781AD102D2B9A814B25DD494649
:107710002046B1461C46069E04E0103D102D01F1A6
:10772000080116DD013210301023072ACDE92B2085
:107730000C604B60F1DD2AAA3146039804F08AFE02
:1077400000287FF4D8AB103D102DDDE92B202DA9AA
:10775000E8DC4E4623468946044601322C44072A7B
:10776000CDE92B24C9E9003500F3B18309F10809FB
:107770004AE52AAA0699039804F06CFE00283FF413
:10778000D3ADFFF7B8BB2AAA0699039804F062FEAE
:1077900000287FF4B0AB249B2C9C0DF1B4091BB9DD
:1077A000109A002A00F092842B9A1799C9F80010B9
:1077B0001699C9F8041001320C44072A2C942B9214
:1077C00000F3A78509F10809002BC0F22086109B61
:1077D00001321C44072ACDE92B24C9E900637FF755
:1077E0005FAD2AAA0699039804F034FE00287FF4BE
:1077F00082AB2C9C0DF1B40954E5109A2B9B012A05
:1078000004F1010403F1010509F1080740F30E81B9
:107810000123072DC9F80060CDE92B54C9F80430C5
:1078200000F31D83169B179A691C1C4407290B91B2
:10783000CDE92B14C7E9002300F31D8308370B9A09
:10784000531C1D460895109D0E9300220023DDE970
:10785000120105F1FF3A07F10809F9F7F5F80028D8
:1078600040F0A780089DC7F804A001365444072DB6
:107870003E602C942B9500F3EF810B9A07F11003D7
:1078800002324F4608929946199A7A601444089A2F
:107890002C9426AB072A2B923B607FF703ADA0E721
:1078A000012A98467FF4B9AB002D08BF0A2C80F05E
:1078B000938256AE3034012306F8014D0893FFF74A
:1078C0005CBB2AAA0699039804F0C4FD00287FF443
:1078D00012AB2C9C0DF1B40982E42AAA06990398F4
:1078E00004F0B8FD00287FF406AB2C9C0DF1B40920
:1078F00086E42AAA0699039804F0ACFD00287FF4D8
:10790000FAAA2C9C0DF1B409B9E400BFC8CE000856
:10791000DCCE0008249B002B40F37581DDE91023A9
:107920009342A8BF1346002B1D460DDD2B9BC9F8C3
:10793000006001332C44072B2C94C9F804502B937E
:1079400000F3BE8409F10809119B002DA8BF5B1B41
:10795000002B1D4640F3D481102D2B9ABC4B40F3D5
:10796000BB81184621464B461027B146DDF80CA0D6
:10797000069C064604E00833103D102D40F3A78115
:1079800001321031072ACDE92B21C3E90067F2DD6E
:107990002AAA2146504604F05DFD00287FF4ABAAD8
:1079A000DDE92B212DABE7E7CDF820A056AEFFF7A0
:1079B000E4BABAF1000F7FF767AFBAF1100FA44B2A
:1079C00040F34E86194622463B461026DDF80C90C1
:1079D000069C0E9D0F4607E00833AAF1100ABAF183
:1079E000100F40F38D8201351032072DCDE92B5257
:1079F000C3E90076F0DD2AAA2146484604F02AFDB4
:107A000000287FF478AADDE92B522DABE5E7099A2F
:107A100018F0100F02F1040340D118F0400F099A3A
:107A200038D0148809930025FFF787BA18F0010FA2
:107A30007FF4EEAE0122072DC9F80060CDE92B548A
:107A4000C9F8042000F308810233089309F11009F2
:107A50001AE718F0010F7FF413AE23E42AAA06995F
:107A6000039804F0F7FC00287FF445AA2C9C50E40E
:107A700018F4007F40F00D83146809930025FFF788
:107A800010BB980500F10F831468099101220025AD
:107A9000FFF756BA18F4007F40F013831468099377
:107AA0000025FFF74ABA980500F103830C68099294
:107AB000E51720462946FFF796BA059A1046D117D2
:107AC000C3E900015E463AE4DDE9120102460B46D5
:107AD000F9F736FC002840F09985612F00F0078403
:107AE000412F00F0F98248F4807327F02002BAF1A8
:107AF000FF3F0E930492139B00F01F85472A00F06E
:107B00001685002BC0F2E9839DED127BCDE90A00BA
:107B10008DED1E7B662F00F0DD84462F00F0628520
:107B2000049B0398452B0CBF0AF10105554628AA72
:107B300025ABCDE90032022124AB2A469DED1E0B78
:107B400002F0CEFC672F064640F0958518F0010F35
:107B500040F0F784289B40469B1BDDF8388010934B
:107B6000249B1193049B472B00F07183049B462BAD
:107B700000F007840499119BFAB2412908BF0F3223
:107B800003F1FF3306BFD2B201210021002B249361
:107B9000B8BF119B8DF89820BABFC3F101032D2205
:107BA0002B22092B8DF8992000F3E584002940F061
:107BB0006A8530228DF89A200DF19B0230331370C4
:107BC000531C26AA9B1A109A1993012A134408934E
:107BD00040F32885089B169A1344089300230F93BB
:107BE00014931193089B20F4806023EAE37340F41C
:107BF000807804930B9B002B40F03C839A469DF8C1
:107C00008B20FFF7C6B92B9A1249C9F80010013230
:107C100001340121072ACDE92B24C9F804103FF7CC
:107C2000B2AD09F10809BAE540210398FEF73EF824
:107C3000069B18601861002800F05385069A4023BF
:107C40005361FFF79CB8524207920993FFF756BA67
:107C5000DCCE0008C8CE00082AAA0699039804F0D2
:107C6000F9FB00287FF447A9DDE92B3401330893A1
:107C70000DF1BC092DAF07E62AAA0699039804F076
:107C8000E9FB00287FF437A92C9C0DF1B40907E526
:107C90005346062B28BF0623B2460F96149611961C
:107CA0000A9632460493CDE90834A44EFFF771B921
:107CB0002AAA0699039804F0CDFB00287FF41BA99B
:107CC0009DF88B202C9C0DF1B409FFF779BA0C4676
:107CD00031464E4699460B4601322C44072ACDE9DF
:107CE0002B24C9E9003540F3D1812AAA06990398CB
:107CF00004F0B0FB00287FF4FEA82C9C0DF1B40921
:107D0000119B18F4806F33449A4640F01B81249BEA
:107D1000109A934249DB18F0010F46D1109AB5181A
:107D2000A5EB0A05D31A9D42A8BF1D46002D0DDD07
:107D30002B9AC9F800A001322C44072A2C94C9F8C8
:107D400004502B9200F33C8309F10809002DACBFCD
:107D50005D1B1D46002D7FF7A5AA102D2B9A784B91
:107D600040F3AB80194610262346039FDDF818A088
:107D70000C4605E009F10809103D102D40F39A80EA
:107D800001321033072ACDE92B23C9E90046F1DD82
:107D90002AAA5146384604F05DFB00287FF4ABA8C0
:107DA000DDE92B230DF1B409E6E72B9A1799C9F801
:107DB00000101699C9F8041001320C44072A2C94BB
:107DC0002B9200F3B58209F10809A7E7002D08BF3F
:107DD0000A2C9846FFF46DAD08F480630022CDF8BC
:107DE00020900A97CDF82C8056AE9146DDF8688039
:107DF0001F460AE00023204629460A22F8F756FECD
:107E000004460D4654EA050346D00A2200232046C4
:107E10002946F8F74BFE303206F8012C09F101092A
:107E2000013E002FE6D098F800309945E2D1B9F133
:107E3000FF0FDFD0002D08BF0A2CDBD31B9B189946
:107E4000F61A1A46304604F0D3FA98F80130002B9F
:107E500000F0898308F101084FF00009CAE72AAA57
:107E60000699039804F0F6FA00287FF444A8DDE9A7
:107E70002B542DAFD6E42AAA0699039804F0EAFA07
:107E800000287FF438A8DDE92B342DAF0B93D6E41E
:107E9000012A7FF4C2A80CE5049BCDF840909B1BFF
:107EA000DDF82090CDF868800A9FDDF82C800893DB
:107EB000FFF763B821461C460B4601322C44072AC3
:107EC000CDE92B24C9E900357FF7EAA989E42AAA7C
:107ED0000699039804F0BEFA00287FF40CA82C9CA5
:107EE0000DF1B409FFF790B92AAA0699039804F096
:107EF000B1FA00287EF4FFAF0DF1B409FFF7BABB69
:107F000014463A461F4613462A460132089207F1A4
:107F10000802C7E9003A089B2B935444072B2C9482
:107F20003FF79AAE0133089302F108091746ABE414
:107F3000059A1A605E46FFF702BA00BFC0CE00087D
:107F4000DCCE0008109BCDF82CB0F3180893149BDE
:107F5000CDF838804A460C96C24FDDF86C90DDF8BB
:107F60006880DDF818B056462146DDF80CA0002BDD
:107F70005ED00F9B002B5FD1149B013B08F1FF38B3
:107F800014932B9B1898106001334944072B2C91B4
:107F9000C2F804902B9353DC0832089898F800300C
:107FA000851B9D42A8BF1D46002D0BDD2B9B166037
:107FB00001332944072B2C9155602B934BDC98F807
:107FC00000300832002DACBF5D1B1D46002D2BDD9F
:107FD000102D2B981CDD102404E0103D102D02F113
:107FE000080215DD013010310728CDE92B01C2E967
:107FF0000074F2DD2AAA5946504604F02BFA0028F4
:108000007EF479AF103D102DDDE92B012DAAE9DCBE
:10801000013029440728CDE92B01C2E900753EF75C
:1080200062AF98F8003008321E44149B002BA0D198
:108030000F9B002B00F0FB800F9B013B0F93A0E7F1
:108040002AAA5946504604F005FA00287EF453AF98
:108050002C992DAAA1E72AAA5946504604F0FAF90C
:1080600000287EF448AF98F800302C992DAAA9E793
:108070003046F9F7A5F8AA4603460890FFF7A6B9D7
:1080800098F800302C992DAA1E44CEE709F1080972
:1080900036E6147809930025FFF703B8059A1A808D
:1080A0005E46FFF74CB91478099100250122FEF7CE
:1080B00047BF91F900400992E51720462946FEF78F
:1080C00092BF147809930025FEF737BF18F0010F0F
:1080D0003FF4E8A8FFF768BB30238DF88C305823B5
:1080E000BAF1630F8DF88D3048F0020400F3B681C9
:1080F00048F481730E9327F0200304930022139B0E
:108100000A92A0463DAE002BC0F2E8809DED127BA6
:108110008DED1E7B00230B93612F00F06081412FBA
:108120007FF4F8AC24A89DED1E0B04F0B9F80022F2
:108130004FF07F5351EC100BF8F71EFA002200238A
:10814000CDE90C01F8F780FC002840F04382464B53
:1081500008930AF1FF34CDE90F9B1197CDF850A099
:10816000B1462196CDF88080DDF820A0DDE90C67CE
:1081700003E0F8F769FC20BBA94600223B4B3046E0
:108180003946F8F7F9F90F460646F9F7EFF8804651
:10819000F8F788F902460B4630463946F8F734F8C6
:1081A0004D461AF808C005F801CBB4F1FF3FA346CD
:1081B00006460F464FF000024FF0000304F1FF3473
:1081C000D7D1304639460022294B119FDDF850A007
:1081D000CDF844904446DDF83C90DDF88080CDF841
:1081E0003CB0219EDDF840B0CDE90C01F8F754FC1D
:1081F000002840F0AA80DDE90C0100221C4BF8F7B2
:1082000023FC18B12346DB0700F19F800F9B002B56
:1082100007DB0F9B01332B44302205F8012BAB42C7
:10822000FBD1AB1B40461093DDF8388098E4B24692
:10823000109B0C9ECDF86880F3189A459146DDF8A6
:108240002CB0DDF838800C4628BF9A465FE5119BBC
:10825000DA1C01DB534514DD023F27F020030493B1
:1082600088E400BFDCCE0008ACCE0008000030403F
:108270000000E03F2D228DF88B204FF0000AFEF722
:108280008BBE119B10998B42C0F29080C20740F1C7
:10829000A681169A13440893470503D5119B002B1A
:1082A00000F3EF80089B23EAE3730493672700231E
:1082B0000F9314939EE42D228DF88B20FFF71AB9AB
:1082C0002AAA0699039804F0C5F800287EF413AE94
:1082D0002C9C0DF1B409FFF737BB0A90DDE91212AF
:1082E00002F100431F932D231E910B9314E73023BB
:1082F0008DF88C307823F3E6CDF810A0CDF820A0CF
:10830000099482460F90149011909DF88B20FEF7EF
:1083100040BE2AAA0699039804F09CF800287EF42F
:10832000EAAD249BDDE92B240DF1B409FFF74CBA2B
:108330002AAA0699039804F08DF800287EF4DBAD94
:10834000249B2C9C0DF1B409E8E4119B2893089B15
:1083500015F8012CD97B91422B4609D1302003F826
:10836000010C289B5A1E289213F8012C9142F6D03A
:10837000392A0BBF089A0132927AD2B203F8012C43
:108380004FE7119B002B40F35281119BBAF1000F74
:1083900040F0EB80C40700F1E880089366274305AE
:1083A00070D4089B23EAE373049380E7109B169A2A
:1083B00013440893119B002B40F348816727EEE795
:1083C0002AAA0699039804F045F800287EF493AD94
:1083D000249B109A2C9CD31A0DF1B409B6E424A85E
:1083E0009DED1E0B03F05CFF00224FF07F5351EC1C
:1083F000100BF8F7C1F800220023CDE90C01F8F7C3
:1084000023FB08B101232493BA4B0893A1E65D42F4
:108410001033B94B80F29A80194610272346DDF8B5
:108420000CA00C4605E009F10809103D102D40F3A1
:108430008A8001321033072ACDE92B23C9E900478E
:10844000F1DD2AAA0699504604F004F800287EF4CB
:1084500052ADDDE92B230DF1B409E6E70AF1010184
:108460000398FDF723FC0646002800F04F8148F4EE
:1084700081730E9327F020030493A046139B0A9068
:1084800041E667271A9800220F9214920378119AF6
:10849000FF2B0CD093420ADA4178D21AB1B1149B67
:1084A000013314930B46FF2B00F10100F2D111921E
:1084B000149B0F9A08991A9013441B9A02FB0313FA
:1084C000089323EAE3730493FFF794BB0F990131F8
:1084D0000F91DDE728AA25ABCDE90032032124ABBB
:1084E00052469DED1E0B039801F0FAFF55460646D5
:1084F00000EB0A043378302B00F0C980249D2C4413
:1085000000220023DDE91E01F8F79EFA10B1234690
:10851000FFF721BB289BA342BFF41DAB30215A1C9F
:1085200028921970289B9C42F9D8FFF714BBBAF126
:10853000000F00F086800A90E5E50A904FF0060AE9
:10854000E1E57419DCE721461C460B4601322C4458
:10855000072ACDE92B24C9E9003500F3B08009F1E1
:108560000809FFF734B9994644E4169A1344534472
:108570000893662713E70DF1A70C64465F4D00E0F2
:108580001446A5FB0312D20802EB8201A3EB4103C0
:1085900003F130011346092B04F8011C04F1FF32EA
:1085A000EEDC3033023CDBB2A44502F8013C40F281
:1085B00094800DF19A04114601E011F8013B04F892
:1085C000013B8C45F9D12AAB9B1A0DF19A02134459
:1085D000FFF7F7BA01232493494B0893B9E5119BA0
:1085E000089359E628AA25ABCDE90032032124AB34
:1085F00052469DED1E0B039801F072FF554606464C
:10860000462F06EB05043FF475AF79E7139B3D4E0B
:10861000002BB6BF2D229DF88B208DF88B203A4B76
:10862000FEF76ABFC5077FF5D9AAFFF7D3BABAF13B
:10863000000F17D1C10715D40123049308936627AF
:1086400035E6CDF828A04FF0010A5CE5089AC3F1A1
:1086500001031A4422EAE27308920493672726E68C
:108660004A4656E4169B01335344089323EAE373C6
:10867000049366271BE6472F7FF463AF18F0010FC2
:108680003FF468AABCE70DF19A02FFF797BA0022FF
:108690000023DDE91E01F8F7D7F900287FF42EAF9B
:1086A000C5F1010524952AE709999BF801700B682B
:1086B00043EAE37A0B1D93460993FEF7A2BB2AAA6D
:1086C0000699039803F0C6FE00287EF414ACDDE999
:1086D0002B240DF1B409FFF77AB80DF19A03FFF7D7
:1086E00070BA039A0C2313604FF0FF330593FEF723
:1086F00011BC00BF98CE0008DCCE0008CDCCCCCC9D
:10870000ACCE000894CE000890CE0008069A93895B
:1087100043F040039381FEF7F6BB00BF024B0146D6
:10872000186801F037BE00BF0C08002010B4044CDC
:1087300013460A46014620685DF8044B03F0ECBB83
:108740000C08002010B4044C13460A460146206869
:108750005DF8044B01F092BD0C0800200000000001
:108760002DE9F04FD7B01C468946174605460390C1
:1087700002F05EFF036816931846F8F721FD08948F
:1087800015901DB1AB6B002B00F00781D9F8641078
:10879000B9F90C20C80793B202D4990540F11F81A2
:1087A0009E040AD4D9F8641042F4005321F4005115
:1087B000A9F80C30C9F864109BB21D0740F1B280D3
:1087C000D9F81020002A00F0AD8003F01A020A2A1E
:1087D00000F0C98000239FED867B1093CDE92B33F9
:1087E0001793CDE919331B93189305932DAB2A9357
:1087F0009B463B78CDF81C908DED127B002B00F052
:108800005982252B3C4602D11DE0252B03D014F8BC
:10881000013F002BF9D1E51B8DB1DDE92B3201338E
:108820002A44072BCBF80070CBF80450CDE92B324B
:1088300000F3CA800BF1080B059B2B4405932378AA
:10884000002B00F0378200236678069398468DF857
:108850008B3004F1010A4FF0FF392B250AF1010A90
:10886000A6F120035A2B00F22A84DFE813F0AA03B2
:10887000280428049C02280428042804A7022804A9
:108880002804C602D2022804D702DC022804F60219
:108890006D026D026D026D026D026D026D026D0260
:1088A0006D02280428042804280428042804280425
:1088B000FB0228043C03F303FB02FB02FB02280437
:1088C000280428042804EE03280428049A00280415
:1088D000280428045003280479032804280490035A
:1088E0002804280428042804280428042804280428
:1088F000FB0228043C03C500FB02FB02FB02D10380
:10890000C50070002804B5032804C2039C00DE03E0
:1089100070002804500372002C02280428047C02F2
:10892000280472004946039801F0BEFCA0B1D9F8B2
:108930006430D80704D4B9F80C30990540F1B783F6
:108940004FF0FF330593059857B0BDE8F08F48F01E
:1089500020089AF8006081E7B9F80C3003F01A0299
:108960000A2A7FF437AFB9F90E20002AFFF632AF9A
:10897000D9F86420D20705D49B0503D4D9F8580050
:10898000FDF782F923463A464946039801F026FC52
:108990000590059857B0BDE8F08F0398FCF7F8FEF6
:1089A000F4E648F0100818F0200F00F06C83089CE3
:1089B000073424F00703D3E9004503F108020892C5
:1089C00028F4806300228CE12AAA0799039803F017
:1089D000F7FD002841F076830DF1B40B2CE7D9F8B0
:1089E0005800FDF74FF9B9F90C2093B2D8E600BF53
:1089F000000000000000000043469F0640F12F8366
:108A0000089C073424F00704D4E9000104F10802AB
:108A1000089204460D46002871F1000205DA2D2265
:108A2000644265EB45058DF88B2056AAB9F1FF3FEE
:108A3000049200F0B284012254EA050123F0800878
:108A400040F05981B9F1000F40F01986002A40F03A
:108A5000088513F0010356AF099302D0302307F8BD
:108A6000013D00230A930F9314931193099B9DF8E2
:108A70008B204B45B8BF4B46049312B1049B013386
:108A8000049318F002030B9302D0049B0233049367
:108A900018F084032C9C0E933FD1069B04995D1A19
:108AA000002D3ADD102D2B9A29DD594620462096BF
:108AB0001023039C079EBB4604E0103D102D01F1DE
:108AC000080118DD0132BA4F1030072ACDE92B20FA
:108AD000C1E90073F1DD2AAA314620460C9303F068
:108AE0006FFD002840F03D84103D102DDDE92B2066
:108AF0002DA90C9BE6DC209E5F4604468B46013286
:108B0000AB4B2C44072ACDE92B24CBE9003500F3ED
:108B1000FF849DF88B200BF1080B72B12B9A013268
:108B200001340DF18B000121072ACDE92B24CBE97B
:108B3000000100F318840BF1080B0B9B6BB12B9B0E
:108B40000133023423A90222072BCDE92B34CBE9D0
:108B5000001200F315840BF1080B0E9B802B00F024
:108B60003183099BA9EB0305002D37DD102D2B9ACE
:108B7000904B28DD59462046BB464FF0100937463A
:108B80001C46079E04E0103D102D01F1080115DD83
:108B900001321030072ACDE92B20C1E90049F2DD6E
:108BA0002AAA3146039803F00BFD002840F0D98330
:108BB000103D102DDDE92B202DA9E9DC3E46234692
:108BC0005F4604468B4601322C44072ACDE92B240C
:108BD000CBE9003500F3EF830BF1080B18F4807F2D
:108BE00040F080822B9B099ACBF80070013314442B
:108BF000072B2C94CBF804202B9300F392830BF1DA
:108C0000080B18F0040F3BD0069B049A9D1A002D08
:108C100036DD102D2B9B21DD1026039FDDF81C80F7
:108C200004E0103D102D0BF1080B17DD0133604AF5
:108C30001034072BCDE92B34CBE90026F1DD2AAA2D
:108C40004146384603F0BCFC002840F06C85103DDE
:108C5000102DDDE92B340DF1B40BE7DC0133544A60
:108C60002C44072BCDE92B34CBE9002508DD2AAABB
:108C70000799039803F0A4FC002840F0E9822C9C9B
:108C80000499DDE905328A42ACBF9B185B18059355
:108C9000002C40F0D58200232B930A9B1BB10A992C
:108CA0000398FCF789FE0DF1B40B57463B78002B77
:108CB0007FF4A7AD2C9BDDF81C90002B41F0E780E2
:108CC00000232B93CBE243469A0640F14E81089C49
:108CD000073424F0070202F10801D2E900450891A7
:108CE000012200218DF88B10B9F1FF3F56A90491A4
:108CF0007FF4A2AE9846012A00F05083022A00F0C9
:108D00001B8356A900E03946E20842EA4572E808AA
:108D100004F0070305461446303354EA050201F80F
:108D2000013C01F1FF37EED118F0010F00F0148380
:108D3000302B00F01183049A02393023521A07F8BD
:108D4000013C09920F468CE6A6F1300300221AF886
:108D5000016B02EB820203EB4202A6F13003092B06
:108D6000F5D906927CE5144B179318F0200F00F00C
:108D70001481089C073424F00703D3E9004503F16C
:108D80000802089218F0010F09D054EA050306D032
:108D900030238DF88D6048F002088DF88C3028F46F
:108DA000806302229DE748F001089AF8006055E5CB
:108DB000ECCE0008FCCE000898CE0008039E30469A
:108DC00002F036FC436818931846F8F7F9F91B903F
:108DD0000446304602F02CFC83681A93002C3FF4C2
:108DE000B8AD9AF80060002B3FF438AD1B78002B2B
:108DF0003FF434AD48F4806830E5089B9AF8006091
:108E00001A680692002A03F10403C0F297860893B9
:108E100024E58DF88B509AF800601FE59AF8006001
:108E200048F004081AE59AF800602A2E0AF10102B7
:108E300001F0B081A6F13003092B92464FF00009F2
:108E40003FF60EAD1AF8016B09EB890903EB4909EE
:108E5000A6F13003092BF5D902E548F080089AF80D
:108E60000060FBE4089C073424F0070494ED007BC9
:108E700052EC171B22F000431D938DED1C7A083431
:108E8000DDE91C014FF0FF32BA4B08948DED127BE7
:108E9000F8F756FA002840F06F844FF0FF32B54BD8
:108EA000DDE91C01F7F7E4FD002840F065840022AD
:108EB0000023DDE91201F7F7D1FD002840F05B85C2
:108EC0009DF88B20AC4FAD4B0020032104910A90FC
:108ED00028F08008472ED8BF1F46099181460F9081
:108EE00014901190C9E50898002301688DF88B3023
:108EF0001A468DF8F4100123011D04930A9291463D
:108F00000F9214921192CDE908133DAFB9E5089B79
:108F10001F6800258DF88B501C1D002F00F039862E
:108F2000B9F1FF3F00F011874A4629463846F8F765
:108F3000B7F90A90002800F0E7850A9BDB1B09932C
:108F4000A94623EAE37308940493CDF82890CDF85A
:108F50003C90CDF85090CDF844909DF88B208CE556
:108F600048F010039A063FF5B2AE089ADF0602F108
:108F7000040100F17E835D06089A00F1E4849C05FB
:108F800040F177831478089100250122A9E67C4BF3
:108F9000179318F0200F7FF4ECAE089A18F0100F1A
:108FA00002F1040340F0548318F0400F089A40F097
:108FB000D08418F4007F00F04B83147808930025C8
:108FC000E0E69DF88B309AF80060002B7FF446AC09
:108FD00020238DF88B3041E49AF800606C2E03BF9B
:108FE0009AF8016048F020080AF1010A48F01008D8
:108FF00034E4089A18F0200F52F8043B089200F06D
:10900000A183059A1046D117C3E9000157464DE6E2
:109010009AF80060682E03BF9AF8016048F400785F
:109020000AF1010A48F0400818E40899554B0C6809
:10903000179347F630020431ADF88C2048F0020354
:1090400008910025022278264BE648F008089AF895
:10905000006003E448F010039F063FF5D1AC089987
:10906000DD0601F1040200F1FD825C06089900F1C1
:109070007584980540F1F68291F900400892E51751
:1090800020462946C7E4089A18F0100F02F104039D
:1090900040F0E38218F0400F089A40F0678418F41B
:1090A000007F00F0DA8214780893002588E4D9F86C
:1090B0005800FCF7E9FD4FF0FF33059343E4002E21
:1090C0003FF4F8AD002301211A4604918DF8F460B5
:1090D0008DF88B300A9399460F931493119309914D
:1090E0003DAFCEE4652E40F3CA8000220023DDE9C7
:1090F0001201F7F7A9FC002800F069812B9B224A96
:10910000CBF80020013301340122072BCDE92B34A9
:10911000CBF8042000F306840BF1080B249B109A73
:109120002C9C934203DB18F0010F3FF46AAD2B9B9C
:10913000169ACBF80020159ACBF80420013314447A
:10914000072BCDE92B3400F317850BF1080B109B8F
:109150005D1E002D7FF755AD102D2B9A0B4B40F364
:10916000E782194610262346039FDDF81C900C4623
:1091700014E000BFFFFFEF7F8CCE000888CE000810
:10918000ACCE000898CE0008C8CE0008FCCE00087F
:109190000BF1080B103D102D40F3C7820132103344
:1091A000072ACDE92B23CBE90046F1DD2AAA49465F
:1091B000384603F005FA00284CD1DDE92B230DF1E8
:1091C000B40BE7E7069B049A9D1A002D7FF7C9AC04
:1091D000102D2B9ABC4B27DD59462046BB461C461A
:1091E0003746079E04E0103D102D01F1080116DD01
:1091F000013210301023072ACDE92B200C604B6080
:10920000F1DD2AAA3146039803F0DAF9002840F08C
:10921000A880103D102DDDE92B202DA9E8DC3E466D
:1092200023465F4604468B4601322C44072ACDE98B
:109230002B24CBE9003500F392820BF1080B90E46C
:109240002AAA0799039803F0BBF900283FF423AD3D
:10925000DDF81C900A9911B10398FCF7ADFBD9F821
:109260006420B9F80C30D00702D4990540F1D081C0
:109270005A063FF565AB059857B0BDE8F08F109AD8
:109280002B9B012A04F1010403F101050BF10806EF
:1092900040F31C810123072DCBF80070CDE92B543E
:1092A000CBF8043000F3BB81159B169A691C1C4453
:1092B00007290B91CDE92B14C6E9002300F3BB81EC
:1092C00008360B9A531C1D460995109D0E930022DB
:1092D0000023DDE9120105F1FF3906F1080BF7F76C
:1092E000B3FB002840F0C280099DC6F80490013706
:1092F0004C44072D37602C942B9500F3F9800B9A82
:1093000006F1100302325E4609929B46199A72607A
:109310001444099A2C9426AB072A2B9233607FF7CA
:1093200070AC2AAA0799039803F04AF900288FD154
:109330002C9C0DF1B40B64E4179856AF230904F08C
:109340000F0143EA05732A091C461546435C07F8DA
:10935000013D54EA0503F1D1049BDB1B0993FFF7A0
:1093600080BBB14676E72AAA0799039803F028F94B
:1093700000287FF46DAF2C9C0DF1B40BFFF7DDBB23
:109380002AAA0799039803F01BF900287FF460AF1D
:109390002C9C0DF1B40BFFF7E0BB9846002D08BFE5
:1093A0000A2C80F0708156AF3034012307F8014D4C
:1093B0000993FFF756BB2AAA0799039803F000F90F
:1093C00000287FF445AF2C9C0DF1B40B06E4249BE0
:1093D000002B40F37382DDE910239342A8BF1346AC
:1093E000002B1D460DDD2B9BCBF8007001332C4468
:1093F000072B2C94CBF804502B9300F3C1820BF174
:10940000080B119B002DA8BF5B1B002B1D4640F3D2
:109410009980102D2B9A2C4B40F3DB831846214664
:109420005B461026BB46DDF80C90079C074604E01F
:109430000833103D102D40F3C78301321031072A45
:10944000CDE92B21C3E90076F2DD2AAA2146484660
:1094500003F0B6F8002840F0A584DDE92B212DAB00
:10946000E7E7CDF8249056AFFFF7FBBAB9F1000F4C
:109470007FF74CAFB9F1100F134B40F359861946E3
:10948000224633461027DDF80CB0079C0E9D0E4691
:1094900007E00833A9F11009B9F1100F40F3538325
:1094A00001351032072DCDE92B52C3E90067F0DDFD
:1094B0002AAA2146584603F083F8002840F0728417
:1094C000DDE92B522DABE5E7FCCE000818F0010FCB
:1094D0007FF4E0AE0122072DCBF80070CDE92B54CC
:1094E000CBF8042004DC023309930BF1100B0DE7D9
:1094F0002AAA0799039803F063F800287FF4A8AE1E
:10950000DDE92B34013309930DF1BC0B2DAEFDE6E3
:109510002AAA0799039803F053F800287FF498AE1D
:109520009DF88B202C9C0DF1B40BFFF7F6BA2AAAFC
:109530000799039803F044F800287FF489AE2C9C27
:109540000DF1B40B119B18F4806F3B44994640F029
:109550005783249B109A934249DB18F0010F46D1A0
:10956000109ABD18A5EB0905D31A9D42A8BF1D4648
:10957000002D0DDD2B9ACBF8009001322C44072AE8
:109580002C94CBF804502B9200F362840BF1080B5F
:10959000002DACBF5D1B1D46002D7FF732AB102D9B
:1095A0002B9AC54B40F3C480194610262346039FCF
:1095B000DDF81C900C4605E00BF1080B103D102D5A
:1095C00040F3B38001321033072ACDE92B23CBE9D6
:1095D0000046F1DD2AAA4946384602F0F1FF00288C
:1095E0007FF438AEDDE92B230DF1B40BE6E72B9ABF
:1095F0001699CBF800101599CBF8041001320C44E1
:10960000072A2C942B9200F38C820BF1080BA7E70E
:10961000D9F85800FCF738FBB9F80C3028E62AAA2C
:109620000799039802F0CCFF00287FF411AEDDE922
:109630002B542DAE38E62AAA0799039802F0C0FFF2
:1096400000287FF405AEDDE92B342DAE0B9338E610
:10965000146808930025FFF795BB1468089300254C
:10966000FFF7AEB90C680892E51720462946FFF7C8
:10967000D2B91468089101220025FFF732BB012AF4
:109680007FF43CAB8FE608F480630022CDE909A6A5
:10969000CDF82C8056AF9246DDF868801E460AE071
:1096A0000023204629460A22F7F700FA04460D4611
:1096B00054EA050329D00A22002320462946F7F759
:1096C000F5F9303207F8012C0AF1010A013F002EAA
:1096D000E6D098F800309A45E2D1BAF1FF0FDFD01A
:1096E000002D08BF0A2CDBD31B9B1899FF1A1A46C2
:1096F000384602F07DFE98F80130002B00F0968489
:1097000008F101084FF0000ACAE7049BCDF8688011
:10971000DB1BCDF840A00A9EDDF824A0DDF82C80EC
:109720000993FFF79EB9C14694E521461C460B46B6
:1097300001322C44072ACDE92B24CBE900357FF7F1
:109740005EAAEEE518F0100F40F0F88018F0400F18
:1097500000F05183059A1A805746FFF7A7BA2AAA44
:109760000799039802F02CFF00287FF471AD2C9C20
:109770000DF1B40BFFF7F5B9DDE9120102460B4616
:10978000F7F7DEFD002840F09184612E00F0118192
:10979000412E00F0778348F4807326F02002B9F15F
:1097A000FF3F0E930492139B00F02D84472A00F094
:1097B0002484002BC0F2F9829DED127BCDE90A00D2
:1097C0008DED1E7B662E00F0EB83462E00F07E842E
:1097D000049B0398452B0CBF09F101054D4628AAAF
:1097E00025ABCDE90032022124AB2A469DED1E0BAC
:1097F00000F076FE672E074640F09C8418F0010FBB
:1098000040F0F983289B4046DB1BDDF8388010933D
:10981000249B1193049B472B00F0E781049B462B6C
:1098200000F000830499119BF2B2412908BF0F3266
:1098300003F1FF3306BFD2B201210021002B249394
:10984000B8BF119B8DF89820BABFC3F101032D2238
:109850002B22092B8DF8992000F3F983002940F081
:10986000878430228DF89A200DF19B0230331370DB
:10987000531C26AA9B1A109A1993012A1344099380
:1098800040F34284099B159A1344099300230F93D4
:1098900014931193099B20F4806023EAE37340F44E
:1098A000807804930B9B002B40F0758299469DF8BD
:1098B0008B20FFF7E2B800BFFCCE00082B9ABD4911
:1098C000CBF80010013201340121072ACDE92B2405
:1098D000CBF8041060DC0BF1080B2BB9109A1AB905
:1098E00018F0010F3FF48DA92B9A1699CBF80010B0
:1098F0001599CBF8041001320C44072A2C942B92B2
:1099000000F382820BF1080B002BC0F2E782109B60
:1099100001321C44072ACDE92B24CBE900737FF7E1
:109920006EA9FEE42AAA0799039802F049FE0028CE
:109930007FF48EAC0DF1B40BFFF7F0BB059A1A6003
:109940005746FFF7B3B91488089100250122FFF7A5
:10995000C8B9148808930025FFF714BAB1F900407C
:109960000892E51720462946FFF755B81488089352
:109970000025FFF725B82D228DF88B20FFF7A2BA1E
:109980002AAA0799039802F01BFE00287FF460AC16
:109990002C9C0DF1B40B34E52AAA0799039802F028
:1099A0000FFE00287FF454AC249B2C9C0DF1B40BCB
:1099B00093E730238DF88C307823B9F1630F8DF85D
:1099C0008D3048F0020400F3B08248F481730E93A6
:1099D00026F0200304930022139B0A92A0463DAF79
:1099E000002BC0F2E3819DED127B8DED1E7B0023E9
:1099F0000B93612E00F05582412E7FF4E3AE24A834
:109A00009DED1E0B02F04CFC00224FF07F5351ECF9
:109A1000100BF6F7B1FD00220023CDE90C01F7F79A
:109A200013F8002840F00583634B0993CDE90FA696
:109A300009F1FF34CDF850902197B946CDF844B0E4
:109A4000CDF88080DDF824A0DDE90C6703E0F6F7AF
:109A5000FBFF20BBA9460022584B30463946F6F79B
:109A60008BFD0F460646F7F781FC8046F6F71AFD98
:109A700002460B4630463946F6F7C6FB4D461AF805
:109A800008C005F801CBB4F1FF3FA34606460F46D8
:109A90004FF000024FF0000304F1FF34D7D13046FD
:109AA00039460022464BDDF83CA0109ECDF83CB074
:109AB0004446CDF84090DDF88080DDF85090DDF828
:109AC00044B0219FCDE90C01F6F7E6FF002840F0F5
:109AD0007681DDE90C010022394BF6F7B5FF10B1B4
:109AE000E20700F16C810F9B002B07DB0F9B01331A
:109AF0002B44302205F8012BAB42FBD1EB1B404637
:109B00001093DDF8388083E6CDF81090CDF82490DE
:109B1000089481460F90149011909DF88B20FEF7C9
:109B2000ACBF2AAA0799039802F04AFD00287FF4E7
:109B30008FAB249B2C9C0DF1B40B11E55242069285
:109B40000893FFF76DB9144632461E4613462A465F
:109B50000132099206F10802C6E90039099B2B93EC
:109B60004C44072B2C943FF7C3AC0133099302F10B
:109B7000080B1646FFF7CABB2AAA0799039802F0FA
:109B80001FFD00287FF464AB2C9C0DF1B40BFFF794
:109B9000DEBA4B46062B28BF0623B9460F9714970B
:109BA00011970A973A460493CDE90843054FFEF70B
:109BB00064BF00BFC8CE0008ACCE00080000304033
:109BC0000000E03FC0CE00080C4639465F469B4689
:109BD0000B4601322C44072ACDE92B24CBE9003572
:109BE0003FF7A5AC0BF1080BACE4119BDA1C02DBD0
:109BF000994580F2B580023E26F02003049311E6D9
:109C0000109BCDF838805A46DDE91A8BFB18CDF849
:109C10002CA00C97AF4EDDF81CA009934F46DDF841
:109C20000C902146149B002B5BD00F9B002B54D132
:109C3000149B013B08F1FF3814932B9B189810607C
:109C400001335944072B2C91C2F804B02B9368DCE4
:109C50000832099898F80030C51B9D42A8BF1D46E0
:109C6000002D0BDD2B9B176001332944072B2C9112
:109C700055602B935EDC98F800300832002DACBFA5
:109C80005D1B1D46002D26DD102D2B983CDD10247C
:109C900003E00832103D102D36DD01301031072869
:109CA000CDE92B01C2E90064F3DD2AAA51464846FA
:109CB00002F086FC002850D1DDE92B012DAAE9E74E
:109CC0002AAA5146484602F07BFC002845D198F864
:109CD00000302C992DAA1F44A4E70F9B013B0F9342
:109CE000ABE70F9B002BF8D1B946109B0C9FCDF82A
:109CF0006880FB189945DDF82CA0DDF83880934684
:109D00000C4628BF994624E4013029440728CDE9B0
:109D10002B01C2E90065D3DC98F8003008321F44FB
:109D200080E72AAA5146484602F04AFCA8B92C9975
:109D30002DAA8EE72AAA5146484602F041FC60B996
:109D400098F800302C992DAA98E73846F7F738FA9A
:109D5000A94603460990FFF7F4B8D146FFF77ABA4F
:109D6000109B1946119B994200F38280C40740F171
:109D70006B81159A13440993410503D5119B002B60
:109D800000F3E680099B23EAE3730493672600232C
:109D90000F93149386E52D228DF88B204FF0000948
:109DA000FEF76CBEA146FFF755BA0A90DDE9121224
:109DB00002F100431F932D231E910B9319E6109B74
:109DC0002893099B15F8012CD97B91422B4609D188
:109DD000302003F8010C289B5A1E289213F8012CFE
:109DE0009142F6D0392A0BBF099A0132927AD2B247
:109DF00003F8012C82E618F4007F3FF49FAD059A2A
:109E00001A705746FEF752BF2AAA0799039802F024
:109E1000D7FB00287FF41CAA249BDDE92B240DF13D
:109E2000B40B71E5119B002B40F36481119BB9F1D8
:109E3000000F40F00381C60700F1008109936626F8
:109E4000430500F18680099B23EAE37304939EE7B0
:109E50002AAA0799039802F0B3FB00287FF4F8A917
:109E6000249B109A2C9CD31A0DF1B40BFFF790BBD6
:109E7000109B159A13440993119B002B40F34981C1
:109E80006726DDE730238DF88C30582395E503985D
:109E90002AAA494602F094FB00287FF4E0A9FEF7C5
:109EA0000FBF24A89DED1E0B02F0FAF900224FF01F
:109EB0007F5351EC100BF6F75FFB00220023CDE936
:109EC0000C01F6F7C1FD08B101232493024B09935D
:109ED000ACE500BFFCCE000898CE00085D42103310
:109EE000B94B80F29780194610262346DDF80C9076
:109EF0000C4605E00BF1080B103D102D40F3878058
:109F000001321033072ACDE92B23CBE90046F1DDDE
:109F10002AAA0799484602F053FB00287FF498A923
:109F2000DDE92B230DF1B40BE6E709F101010398FC
:109F3000FBF7BCFE0746002800F03B8148F4817324
:109F40000E9326F020030493A046139B0A9047E546
:109F500067261A9800220F9214920378119AFF2B09
:109F60000CD093420ADA4178D21AA9B1149B01337A
:109F700014930B46FF2B00F10100F2D11192149BB8
:109F80000F9A09991A9013441B9A02FB0313099321
:109F900023EAE373049385E40F9901310F91DEE71F
:109FA00028AA25ABCDE90032032124AB4A469DED1A
:109FB0001E0B039800F094FA4D46074600EB090487
:109FC0003B78302B00F0BE80249D2C4400220023DF
:109FD000DDE91E01F6F738FD08B1234613E4289B9E
:109FE000A342BFF410AC30215A1C28921970289B50
:109FF0009C42F9D807E47C19E8E7B9F1000F00F0BA
:10A0000092800A90ECE40A904FF00609E8E42146B9
:10A010001C460B4601322C44072ACDE92B24CBE900
:10A02000003500F3A9800BF1080B70E49A46FFF7A6
:10A0300037BB01232493654B0993F7E4159A134426
:10A040004B4409936626FBE6119B099394E60DF1B8
:10A05000A70C64465E4D00E01446A5FB0312D2082F
:10A0600002EB8201A3EB410303F130011346092BFC
:10A0700004F8011C04F1FF32EEDC3033023CDBB2A9
:10A08000A44502F8013C40F290800DF19A0411467B
:10A0900001E011F8013B04F8013B8C45F9D12AABF2
:10A0A0009B1A0DF19A021344FFF7E3BB139B494F30
:10A0B000002BB6BF2D229DF88B208DF88B20464BB0
:10A0C000FEF702BFDDF81C90FFF7C9B828AA25AB40
:10A0D000CDE90032032124AB4A469DED1E0B0398C7
:10A0E00000F0FEF94D460746462E07EB05043FF407
:10A0F00067AF6BE7B9F1000F31D1C5072FD401234A
:10A1000004930993662642E6C3077FF5BFABFFF7CA
:10A11000B9BB099AC3F101031A4422EAE273099216
:10A120000493672633E6CDF828904FF0010957E4F1
:10A130005A4611E5472E7FF45EAF18F0010F3FF449
:10A1400061ABD1E700220023DDE91E01F6F77CFCBC
:10A1500000287FF439AFC5F10105249535E7159B3B
:10A1600001334B44099323EAE373049366260EE616
:10A170000DF19A02FFF77ABB2AAA0799039802F019
:10A180001FFA00287FF464A8DDE92B240DF1B40B3D
:10A19000FFF7BDBB08999AF801600B6843EAE379C1
:10A1A0000B1D92460893FEF759BB0DF19A03FFF77A
:10A1B00060BBDDF81C90B9F80C3043F04003A9F8FF
:10A1C0000C30FFF74CB800BFFCCE0008ACCE000846
:10A1D000CDCCCCCC94CE000890CE00082DE9F04137
:10A1E0000C46ADF58D6D8989666EE589199621F06D
:10A1F00002010646E069ADF80C1017464FF4806185
:10A20000626AADF80E5098461AAD0023079016A862
:10A21000099206930095049502910591FBF72EFD96
:10A2200043463A4669463046FEF79AFA051E07DB72
:10A2300030466946FBF7ECF9002818BF4FF0FF35B0
:10A24000BDF80C305B0603D5A38943F04003A3811E
:10A250001698FBF715FD28460DF58D6DBDE8F081CC
:10A2600021B1FF2A04D80A700120704708467047C0
:10A270008A2303604FF0FF30704700BF70B50D4672
:10A28000084C114606461A46284600232360FAF772
:10A29000EAFB431C00D070BD2368002BFBD0336069
:10A2A00070BD00BFAC1D002038B5314B1B680546A2
:10A2B0000C4613B19A6B002A3AD0B4F90C2093B231
:10A2C00018070CD52069A8B113F0010220D06369EA
:10A2D00000225B42A361A26000B3002038BDD90612
:10A2E0003ED5580728D4206942F00803A3819BB2C9
:10A2F0000028E9D103F42072B2F5007FE4D02846AB
:10A30000214601F0E7F9A389206913F00102DED1AB
:10A31000990758BF6269A2600028DED1B4F90C30F9
:10A320001A06DBD543F04003A3814FF0FF3038BD60
:10A330001846FBF72DFAC0E7216B51B104F1400339
:10A34000994204D02846FBF737FBB4F90C200023D0
:10A35000236300232069636022F024022060C3E7A6
:10A3600042F0400209232B604FF0FF30A28138BD3C
:10A370000C080020024B13B1024800F005B87047EA
:10A380000000000001B30008002301461A461846E9
:10A3900002F078B938B5074C00230546084623601B
:10A3A000FAF751FB431C00D038BD2368002BFBD0CB
:10A3B0002B6038BDAC1D00202DE9F04F03690F69FB
:10A3C000BB4283B0C0F28680013F01F1140900F165
:10A3D000140A59F827205AF82730BC000132B3FB81
:10A3E000F2F80AEB0403009409EB040B0193B8F1B3
:10A3F000000F38D000252E46CE46D4465EF8044BDA
:10A40000DCF80030A2B208FB0255220C2C0C08FB31
:10A410000242ADB2751B96B2C6EB134615FA83F332
:10A4200006EB23469BB243EA0643F3454FEA124547
:10A430004CF8043B4FEA2646E0D2009B5AF8033022
:10A440008BB9019A131F9A450CD252F8043C4BB9B0
:10A45000A2F1080302E01A68043B1AB99A4507F111
:10A46000FF37F8D30761044601F02AFC00282DDBF2
:10A4700008F101085546002359F8041B28688AB2E0
:10A480009A1A0B0C12FA80F2C3EB104303EB22432F
:10A4900092B242EA0342CB4545F8042B4FEA2343EC
:10A4A000EAD25AF827200AEB87037AB91A1F924595
:10A4B0000BD253F8042C42B9083B02E01A68043B63
:10A4C0001AB99A4507F1FF37F8D32761404603B020
:10A4D000BDE8F08F002003B0BDE8F08F0000000061
:10A4E0002DE9F04F55EC104B9BB0066C0291814664
:10A4F00007920593CDE9004556B1426C7260012385
:10A500009340B360314601F0EBF90023C9F84030C5
:10A51000B5F10008249AB4BF012300231360764BE1
:10A52000BCBF28F00048CDF8048033EA080300F0EF
:10A53000A680DDE900670022002330463946F6F7A1
:10A5400083FA054678B1059A01231360259B002BF9
:10A5500000F0C080694B259A03F1FF3B1360584619
:10A560001BB0BDE8F08F18AA19A947EC106B48463C
:10A5700001F038FC5FEA1854824640F0A080DDE923
:10A5800018542C4404F23243202B40F32C84C3F1A2
:10A59000400308FA03F8009B04F2124023FA00F08B
:10A5A00048EA0000F5F76EFF01230646013CA1F1E1
:10A5B000F8770F93304639460022514BF5F724FEC9
:10A5C00047A3D3E90023F5F7D7FF47A3D3E9002337
:10A5D000F5F71CFE064620460F46F5F763FF44A339
:10A5E000D3E90023F5F7C8FF02460B46304639464B
:10A5F000F5F70CFE06460F46F6F7B8FE0022069069
:10A60000002330463946F6F729FA002840F07382D5
:10A61000069E162E00F25D823A4B03EBC603D3E989
:10A620000001DDE90023F6F737FA002800F0D783B0
:10A63000731E069300230D932C1BB4F1010800F147
:10A64000548200230893069B002BC0F24582984455
:10A650000C9300230B93029B092B5BD8052B40F333
:10A66000C083043B02930025029B023B032B00F2B4
:10A670009884DFE813F0DF03BF03E803F504059ACD
:10A6800042F20F731360009B83B9C8F313036BB9D5
:10A69000259BDFF874B0002B3FF461AF0BF108038A
:10A6A000259A584613601BB0BDE8F08F259BDFF854
:10A6B0005CB0002B3FF453AF0BF10303F0E7C7F39B
:10A6C000130343F07F570F95A4F2FF3447F440176C
:10A6D000189D6FE7DFF838B058461BB0BDE8F08F23
:10A6E00061436F63A787D23FB3C8608B288AC63F98
:10A6F000FB799F501344D33F0000F07FC9CE000880
:10A700000000F83F48D0000810D000081CD0000816
:10A71000C8CE00084FF0FF340125CDE909450023DC
:10A72000029307930021C9F844100E94484601F0A3
:10A73000B1F80E2C8346C9F8400000F2FB80002DD2
:10A7400000F0F8809DED007B069900298DED107BCF
:10A7500040F3E5839D4B01F00F0203EBC20393ED41
:10A76000007B0C11E2068DED007B40F19E84984B3E
:10A77000DDE91001D3E90823F6F728F8CDE9120145
:10A7800004F00F0403267CB1DDE90001904DE307DE
:10A7900004D5D5E90023F5F7EFFE0136641005F185
:10A7A0000805F4D1CDE90001DDE90023DDE912015E
:10A7B000F6F70CF8CDE900010D9B43B10022854B63
:10A7C000DDE90001F6F74AF9002840F0FF84304641
:10A7D000F5F768FEDDE90023F5F7CEFE7E4B00229B
:10A7E000F5F714FD099B0646A1F15077002B00F008
:10A7F0001C84069B1693099B1293DDE90001F6F772
:10A80000B5FD129A714B03EBC20313ED027B00F10D
:10A8100030058DED147BF5F745FE0B460246DDE96C
:10A820000001CDE90067F5F7EFFC0A9BEDB20646A3
:10A830000F460BF10104002B00F05884DDE91423CE
:10A8400000206649F5F7C2FFDDE90023F5F7DCFCDF
:10A850008BF8005032463B46CDE90001F6F71CF973
:10A86000002840F0028532463B4600205949F5F762
:10A87000CBFC02460B46DDE90001F6F70DF9002896
:10A8800040F0FB84129A012A50D05A44CDF85C80E3
:10A89000CDF848A0CDF850B09246CB46DDE900890E
:10A8A0000CE000204B49F5F7AFFC42464B46F6F76B
:10A8B000D5F8002840F0DC84544530D04046494665
:10A8C0000022474BF5F758FE0022454B804689464B
:10A8D00030463946F5F750FE0F460646F6F746FD78
:10A8E0000546F5F7DFFD02460B4630463946F5F7DB
:10A8F0008BFC3035EDB242464B4604F8015B064610
:10A900000F46F6F7ABF832463B460028C9D0169BF7
:10A91000DDF848A00693D946DDF850B036E2D946B6
:10A92000DDF85C80DDF848A0DDF850B0DDE91034DA
:10A93000CDE90034199B002BC0F2AE80069A0E2A96
:10A9400000F3AA80214B03EBC20393ED007B079B2E
:10A95000002B8DED027BC0F2BE82DDE90067DDE9F0
:10A96000022330463946F5F731FFF6F7FFFC05467E
:10A97000F5F798FDDDE90223F5F7FEFD0B460246EB
:10A9800039463046F5F740FC05F130038BF80030CE
:10A99000099B012B06460F460BF1010453D0002200
:10A9A0000F4BF5F7E9FD0022002306460F46F6F7A8
:10A9B0004BF8002840F0EA81CDF800A0CDF81C90BB
:10A9C000DDF82480DDE9029A17E000BF48D00008D6
:10A9D00020D000080000F03F00001C400000E03FD5
:10A9E00000002440F5F7C8FD0022002306460F466C
:10A9F000F6F72AF8002840F03D834A465346304691
:10AA00003946F5F7E3FEF6F7B1FC0546F5F74AFDE2
:10AA10004A465346F5F7B0FD02460B4630463946E6
:10AA2000F5F7F2FB05F1300C04F801CBA4EB0B0CAD
:10AA3000E04506460F464FF00002C14BD2D1DDF88B
:10AA400000A0DDF81C9032463B4630463946F5F70B
:10AA5000DDFBDDE9022306460F46F6F71DF858B97F
:10AA6000DDE9022330463946F5F7EEFF002800F015
:10AA70008D81E90740F18A8114F8015C05E09B456E
:10AA800000F0738313F8015C1C46392D04F1FF3389
:10AA9000F5D001351D7079E10A9A002A3BD0029A5F
:10AAA000012A40F30B82099B5F1E0B9BBB42C0F245
:10AAB000E682DF1B099B002BC0F20B83089A144629
:10AAC0001A44984408920121484600F0A3FF054625
:10AAD00024E001230D93AFE5089A069BD21A5B424E
:10AAE0000B93002308920C93B5E5C4F1010308937E
:10AAF0004FF00008A7E5DDF818804046F5F7D2FCD6
:10AB000032463B46F5F7A0FF00287FF481AD08F1FF
:10AB1000FF3306937CE50B9F089C0A9D002C0CDDFF
:10AB2000B8F1000F09DD4445089A2346A8BF434603
:10AB3000D21A0892E41AA8EB03080B9B6BB10A9A8D
:10AB4000002A00F09082DE1B002F40F09B815146CE
:10AB50003246484601F00EF882460121484600F090
:10AB600059FF0C9A0646002A40F02581029B012BD2
:10AB700040F36C810120404410F01F0000F0198167
:10AB8000C0F12003042B40F3AC83C0F11C00089BF0
:10AB90000344089304448044089B002B05DD514680
:10ABA0001A46484601F036F88246B8F1000F05DD36
:10ABB00031464246484601F02DF806460D9B002BD3
:10ABC00077D1099B002B40F309820A9B002B00F0F0
:10ABD0008980002C00F36B810C9B002B40F0CD8111
:10ABE000A846009ACDF82CB002F001020A92099A08
:10ABF0000BF1FF331A445F460992B346594650465B
:10AC0000FFF7DAFB29460446504601F059F8594649
:10AC100006464246484601F06FF804F130030093BF
:10AC2000C3680146002B40F0D4810890504601F0E3
:10AC300047F8089A07901146484600F051FE079BD6
:10AC400033B9029A22B90A9B002B00F01983029BA8
:10AC5000002EC0F21C8205D1029A1AB90A9A002A63
:10AC600000F01582002B07F1010400F32582009B00
:10AC70003B70099BBB4200F03082514600230A2200
:10AC8000484600F037FE4545824629464FF000030E
:10AC90004FF00A02484600F0968100F02BFE414634
:10ACA000054600230A22484600F024FE2746804637
:10ACB000A4E73146504601F003F8002881DA069FE8
:10ACC000514600230A224846013F069700F012FE33
:10ACD0000A9B8246002B40F0EB820E9B002B40F338
:10ACE000F38209935C46DDF8248002E000F002FE66
:10ACF000824631465046FFF75FFB00F1300704F80B
:10AD0000017BA4EB0B0398454FF00A024FF00003C0
:10AD100051464846EADC002300970293514601223F
:10AD2000484600F077FF3146824600F0C9FF002810
:10AD300014F8012C14DC08D1009BDB0710D404E0CC
:10AD40000000244014F8022C1C46302A04F1FF3382
:10AD5000F8D00BE09B4500F04E8113F8012C1C4607
:10AD6000392A04F1FF33F5D001321A7031464846D2
:10AD700000F0B6FD55B1029921B1A94202D0484672
:10AD800000F0AEFD2946484600F0AAFD514648466F
:10AD900000F0A6FD0022069B2270059A0133136085
:10ADA000259B002B3FF4DBAB58461C601BB0BDE875
:10ADB000F08F1C20EBE60146484600F0DBFE029BCC
:10ADC000012B064640F3D48000230C93336906EB35
:10ADD0008303186900F0CEFDC0F12000CBE60D9092
:10ADE0002AE4012540E4C3F12008009B03FA08F09F
:10ADF000FFF7D8BB00230A93DDE9063213440E9314
:10AE00000133012B1E460993B8BF01260021172EDE
:10AE1000C9F84410099C7FF789AC012204235B0028
:10AE200003F11400B042114602F10102F7D9C9F84A
:10AE300044107BE400230A93079E002E40F3E28037
:10AE40000E960996E2E701230A93F5E7009B002B93
:10AE50007FF490AEDDE90012C2F31303002B40F043
:10AE6000928122F000431B0D1B052BB1089B01337F
:10AE7000089308F1010801230C9A0C93002A3FF46F
:10AE800079AEA3E73A462946484600F073FE52469B
:10AE900001460546484600F0C7FD5146074648466C
:10AEA00000F01EFDBA46002E3FF457AE4FE629468D
:10AEB0002246484600F0AEFE05468DE60F9A002A6F
:10AEC00000F05D8103F23343089A0B9F14461A4445
:10AED00098440892F7E5099B002B3FF73EAD40F000
:10AEE000BC8051EC170B0022B24BF5F745FBDDE9B6
:10AEF0000023F5F7C7FD099E3546002876D1069A4E
:10AF00003123013206928BF800300BF101043146F7
:10AF1000484600F0E5FC002D7FF434AF36E700F042
:10AF20004281069B5C42A44B04F00F0203EBC20378
:10AF3000D3E90023DDE91001F5F71EFB2411CDE96B
:10AF4000000100F0C6819D4D00230226E70705D5CC
:10AF5000D5E90023F5F710FB01360123641005F154
:10AF60000805F3D1002B3FF427ACCDE9000123E421
:10AF7000009B002B3FF46EAF26E76968484600F05F
:10AF800089FC2B6902339A00044605F10C010C3050
:10AF9000F5F70CFF21460122484600F03BFE8046B3
:10AFA0001FE60024C9F844402146484600F072FCE0
:10AFB0004FF0FF330E930993012383460794C9F89A
:10AFC00040000A93B6E400F095FC2746054680460B
:10AFD00014E6484600F084FC012339E6029B022B6C
:10AFE0007FF7F3AD099B002B00F0CF80079BDB437D
:10AFF00006935C468BE7069A3123013206928BF862
:10B000000030B3E6012409940794FFF78BBB304668
:10B01000F5F748FADDE90023F5F7AEFA0022684BB0
:10B02000F5F7F4F80646A1F150770022614BDDE90F
:10B030000001F5F7E9F832463B4604460D46F5F7C0
:10B040002BFD00284FD1324607F100432046294608
:10B05000F5F704FD00283FF469AC00263546C5E746
:10B0600001230A93C8E651460B9A484600F082FD38
:10B07000824672E5DDF800A0DDF81C9086E60B9BA9
:10B080000C9AFB1A1A44CDE90B72002712E5002B2B
:10B0900002945E4607F10104DDF82CB000F3BA809B
:10B0A000009B02953B70454660E69DED107B0226B5
:10B0B0008DED127BFFF767BB009B392B5E46DDF8F9
:10B0C0002CB000F0B980009B029501333B704546DF
:10B0D0004CE6DDE908329C1AF5E45E460295DDF89F
:10B0E0002CB045461AE60026354608E7DDE914236C
:10B0F000DDE90001F5F740FA129B8BF80050012BB7
:10B10000CDE9000120D0129BCDF848805B449846E1
:10B1100000222C4B30463946F5F72EFA0F460646EC
:10B12000F6F724F90546F5F7BDF9303502460B462A
:10B1300030463946F5F768F804F8015B44450646A1
:10B140000F46E5D1DDF848801F4B0022DDE9000104
:10B15000F5F75CF832463B46F5F780FC002870D0E6
:10B16000169B069314F8015C8FE430238BF80030B3
:10B17000069B14F8015C013306935B4689E4189B37
:10B18000C3F13603A0E6002376E6314605224846A1
:10B1900000F0B0FB01460646504600F091FD002845
:10B1A0003FF7ADAE22E79DED107B02268DED007BD3
:10B1B000FFF702BB0000144048D0000820D0000870
:10B1C00000001C40000024400000E03F099B002BD1
:10B1D0003FF41DAF0E9C002C7FF7A8AB0022454B1F
:10B1E000DDE90001F5F7C8F9CDE90001701CF5F7BC
:10B1F00059F9DDE90023F5F7BFF93F4B0022F5F7D8
:10B2000005F8069B1294013B0646A1F15077169370
:10B21000FFF7F3BA51460122484600F0FBFC3146E5
:10B22000824600F04DFD00283BDD009B392B03D00A
:10B23000029B3133009333E7392202953A70454639
:10B240008EE5DDE9002300202C49F4F7DDFF3246CE
:10B250003B46F5F721FC10B9FFF768BB144614F81C
:10B26000013C302B04F1FF32F8D0169B06938DE59C
:10B27000D946DDF848A0DDF850B0169B069304E4EB
:10B28000009B392B2146324607F101045E46DDF86A
:10B290002CB0D1D0002A7FF703AF0B463133009397
:10B2A000FEE67FF4FDAE009BDA077FF5F9AEBCE762
:10B2B000294600230A22484600F01CFB0E9B002B67
:10B2C000054609DD099384E4029B022B0EDC0E9BEC
:10B2D00007E50226FFF770BA029B022B06DC0E9BE5
:10B2E000F0E73FF459ACC0F13C0050E40E9B0993E9
:10B2F00078E600BF0000244000001C400000E03F52
:10B3000038B50A4C0A4D641BA4100AD004F18043DE
:10B31000013B05EB8305013C55F804399847002CA7
:10B32000F9D1BDE8384001F017BB00BF30D10008AB
:10B330002CD100089368002B00F0E4802DE9F04F39
:10B34000B1F90C309BB20C46190783B08246904687
:10B3500035D522699AB313F00202D8F800603DD0C7
:10B360000027D4F824B0D4F81CC0DFF8C0923D46C2
:10B370004D452B463A4628BF4B4661465046D5B10F
:10B38000D847002840F3C680D8F808301B1A074475
:10B390002D1AC8F80830002B00F0B080D4F81CC07B
:10B3A000D4F824B04D452B463A4628BF4B4661465B
:10B3B0005046002DE4D1D6E900750836D8E721467D
:10B3C0005046FEF771FF002840F02A81B4F90C3096
:10B3D000D8F800609BB213F00202C1D113F001094A
:10B3E0005DD1A76820684D46002D54D09A0540F1E4
:10B3F0009B80AF42BB4600F2D88013F4906F2FD0F1
:10B40000D4E9041707EB4707A0EB010B07EBD7774D
:10B41000681C7F105844B8423A4684BF07463A46F3
:10B420005B0540F1D38011465046FAF73FFC0028F7
:10B4300000F0F0805A4621690190F5F7B7FCA28927
:10B44000019B22F4906242F08002A281A7EB0B02E2
:10B4500003EB0B00676123612060A2602F46AB46BF
:10B460005A46494600F0B2F9A2682368D21B5B44F1
:10B470002F46A26023600025D8F80830DB1BB944B2
:10B48000C8F80830002B39D0B4F90C30A768206810
:10B490009BB2002DAAD1D6E900950836A4E7334621
:10B4A0009146104617464E469B46002F6BD000280B
:10B4B00071D0D4E904122068B9454B4628BF3B46F9
:10B4C000884203D9A5681544AB4271DC9A4200F367
:10B4D00093801346656AE16932465046A847051EC7
:10B4E00018DDB9EB05090FD00120D8F808305B1B37
:10B4F0002E447F1BC8F80830002BD6D1002003B0A3
:10B50000BDE8F08F0020704721465046FAF780F8DA
:10B510000028EAD0B4F90C3043F040034FF0FF307C
:10B52000A38103B0BDE8F08F2369834215D361691D
:10B53000A94212D83C4B676A9D4294BF2B466FF0DC
:10B5400000434A4693FBF1F3504601FB03F3E169E4
:10B55000B847071EDEDDED1B8EE7AF4228BF2F4642
:10B560003A46494600F032F9A3682268DB1B3A44A8
:10B57000A3602260002BEED121465046FAF748F82E
:10B580000028E8D0C6E70BF1080353E902679B46A1
:10B590000833002FF9D03A460A213046F5F780FEED
:10B5A00038B30130A0EB060983E72F46AB4657E7D7
:10B5B00031462A4600F00AF923682B4423602146CD
:10B5C0005046FAF725F800288BD0A3E7504600F044
:10B5D000B9FC034600287FF439AF21695046FAF7D9
:10B5E000EBF9B4F90C300C2223F08003CAF80020E8
:10B5F00092E707F101095CE71A463146019300F032
:10B60000E5F8019BA1682268C91A1A44A16022606A
:10B610001D4666E70C23CAF80030B4F90C307BE70E
:10B620004FF0FF306BE700BFFEFFFF7F00FCFF7FA6
:10B63000044A054B1268506B002808BF1846F030CA
:10B64000704700BF0C080020380C002070B50D4674
:10B65000084C114606461A46284600232360F9F78F
:10B66000FAF9431C00D070BD2368002BFBD0336077
:10B6700070BD00BFAC1D002070B50C46B1F90E10B6
:10B68000002996B015461E460FDAA289002312F053
:10B690008000336004D14FF480632B6016B070BD1E
:10B6A000402218462A6016B070BD6A4601F000F9C3
:10B6B0000028EADB019B03F47043A3F50053B3FABF
:10B6C00083F35B094FF480624FF4006033602A60BB
:10B6D00016B070BD8A8992070B4606D501F1430268
:10B6E00001211A60C3E90421704770B582B001AB33
:10B6F0006A460C460546FFF7BFFF009906462846F6
:10B70000FAF7D4FAB4F90C30D8B11649E963019AC2
:10B710000099206043F08003A381C4E904011AB9B1
:10B720003343A38102B070BD2846B4F90E1001F076
:10B73000D3F8A0B1A38923F0030343F001031BB2A4
:10B74000EEE79A05EED423F0030304F1430243F03D
:10B7500002030121A3812260C4E90421E2E7B4F9D4
:10B760000C30DDE755570008032A70B414D940EABD
:10B770000105AD0704460B4622D11D682668AE427E
:10B780001946204603F1040304F1040418D1043AD5
:10B79000032A20461946F0D8541E72B102780B785D
:10B7A0009A4208BF641806D00CE010F8012F11F877
:10B7B000013F9A4206D1A142F7D1002070BC7047E8
:10B7C000541EEBE7D01A70BC704700BF8842F0B43B
:10B7D0000DD98B1883420AD9841832B1224613F846
:10B7E000014D02F8014D9942F9D1F0BC70470F2A82
:10B7F00049D940EA01039B0747D1A2F110031B0975
:10B8000001F1200707EB031701F1100400F1100507
:10B8100054F8106C45F8106C54F80C6C45F80C6C2E
:10B8200054F8086C45F8086C54F8046C45F8046C3E
:10B830001034BC4205F11005EAD1013302F00F05C6
:10B840001B01032D1944034421D91F1F0E462C460A
:10B85000043C56F804CB47F804CF032CF8D82C1F2F
:10B8600024F0030404342344214402F00302002A98
:10B87000BBD0013B0A4411F8014B03F8014F914240
:10B88000F9D1F0BC70470346F1E70346F1E72A46D9
:10B89000EDE700BFC36C70B505460C464BB153F8DD
:10B8A000240080B1026843F824200023C0E9033358
:10B8B00070BD2122042100F045FF0346E864002802
:10B8C000EDD1002070BD012101FA04F6721D284659
:10B8D000920000F037FF0028F3D0C0E90146E4E70A
:10B8E00031B1C36C4A6853F82200086043F8221053
:10B8F000704700BFF0B50C6983B00D46064601F1F4
:10B90000140C0027DCF8000081B202FB0133010CAB
:10B91000180C02FB01019BB2013703EB0143BC424F
:10B920004CF8043B4FEA1143ECDC3BB1AA68A2425D
:10B9300007DD05EB8402013453612C61284603B016
:10B94000F0BD6968019301313046FFF7A3FF2A6912
:10B95000023205F10C01074692000C30F5F726FA89
:10B96000F26C6968019B52F82100286042F821506E
:10B970003D46DEE7020C12040346C2B90304102060
:10B9800013F07F4F04BF1B02083013F0704F04BF49
:10B990001B01043013F0404F04BF9B000230002B0A
:10B9A00004DB5B0001D50130704720207047002088
:10B9B000E6E700BF036813F00702014607D0DA0785
:10B9C0001FD498071FD55B080B600120704798B201
:10B9D000A0B1104613F0FF0F04BF1B0A08301A076E
:10B9E00004BF1B0904309A0704BF9B080230DA0722
:10B9F00002D45B080BD001300B6070471B0C102089
:10BA0000E8E7002070479B080B6002207047202069
:10BA1000704700BF10B50C460121FFF73BFF012224
:10BA2000C0E9042410BD00BF2DE9F04F0E69146970
:10BA3000A64283B00F46154604DA32462F46264604
:10BA40000D461446D7E9011306EB04084345B8BF79
:10BA50000131FFF71FFF00F1140909EB880EF145D2
:10BA6000009005D24B46002243F8042B9E45FBD89C
:10BA700005F1140A0AEB840407F11403A24503EB51
:10BA8000860C61D2641B153C24F00304CDF804E05D
:10BA9000A24405F110029E4605E02D0C2BD19245E3
:10BAA00009F104094ED052F8045F1FFA85FBBBF17F
:10BAB000000FF2D077464E46002000E0264657F8A9
:10BAC000041B34688BB2A5B2090C240C0BFB035386
:10BAD00003440BFB014000EB134034469BB243EAA6
:10BAE0000043BC454FEA104044F8043BE6D8706080
:10BAF00015682D0CD3D0D9F8003076461846CB46C1
:10BB0000002100E0A3463488000C05FB040001443A
:10BB10009BB25C4643EA014344F8043B56F8043BBD
:10BB2000DBF804001B0C87B205FB037303EB114326
:10BB3000B4454FEA1341E5D89245CBF8043009F1FA
:10BB40000409B0D1DDF804E0B8F1000F0BDD5EF8B8
:10BB5000043CAEF1040E1BB105E05EF8043D13B9E0
:10BB6000B8F10108F9D10098C0F8108003B0BDE821
:10BB7000F08F00BF12F003032DE9F0411446074691
:10BB80002ED10D46A4101CD0BE6C96B3E3074FF027
:10BB9000000806D4641014D03068A8B10646E30744
:10BBA000F8D5324629463846FFF73EFFB5B16A68F8
:10BBB000FB6C641053F82210296043F822500546AC
:10BBC000EAD12846BDE8F081324631463846FFF7D3
:10BBD0002BFF3060C0F800800646E0E70546D9E755
:10BBE000013B0B4A52F823200023FFF783FE054652
:10BBF000C8E701213846FFF74DFE40F2712343614B
:10BC00000122002302610646B8640360BEE700BF5C
:10BC100010D100082DE9F04791460A690E464FEA17
:10BC20006914D1E9011304EB020808F101059D42F2
:10BC3000074604DD5B009D4201F10101FADC384654
:10BC4000FFF728FE002C00F1140337DD03EB84011D
:10BC5000002243F8042B8B42FBD1346906F1140314
:10BC600019F01F0903EB840C20D0C9F1200E00222B
:10BC700000E051461C688A4604FA09F414434AF865
:10BC8000044B53F8042B634522FA0EF2F1D34A60B9
:10BC90000AB108F10205FB6C7268013D53F82210ED
:10BCA0000561316043F82260BDE8F087043953F83C
:10BCB000042B41F8042F9C45F9D8ECE71946CCE752
:10BCC00030B40B6905460069C01A0FD19B001435CA
:10BCD000143119442B4401E09D4207D253F8044D1E
:10BCE00051F8042D9442F7D002D3012030BC7047A4
:10BCF0004FF0FF30FAE700BF2DE9F04113690D69FD
:10BD0000ED1A002D0E46904601F1140402F11407BD
:10BD100014D19B00E2183B4401E0A24259D952F8E9
:10BD200004CD53F8041D8C45F7D009D22246334682
:10BD30003C46464617469846012501E0F6DB0025BD
:10BD40007168FFF7A7FDD8F810303669C56007EBBA
:10BD5000830EBC4600F1140504EB860700235CF853
:10BD6000041B54F8048B8AB213FA88F3090C9A1A4C
:10BD7000C1EB184303EB224392B242EA0342E64589
:10BD800045F8042B4FEA2343E9D8A74217D9AE461A
:10BD9000A4465CF8042B13FA82F3191401EB124148
:10BDA0009BB243EA014267454EF8042B4FEA214318
:10BDB000EFD8E443274427F0030704373D44043D0C
:10BDC00022B955F8043D013E002BFAD00661BDE8CA
:10BDD000F0810021FFF75EFD01220023C0E904236A
:10BDE000BDE8F0812DE9F0430F4683B0012155EC09
:10BDF000104B1646FFF74EFDC5F30A588146C5F3B2
:10BE00001303B8F1000F01D043F48013002C019309
:10BE100024D002A840F8084DFFF7CCFD002836D109
:10BE2000DDE90023C9F81420002B0CBF01210221F9
:10BE3000C9F81830C9F81010B8F1000F1BD109EB80
:10BE40008103A0F2324038601869FFF793FDC0EB20
:10BE500041103060484603B0BDE8F08301A8FFF709
:10BE6000A9FD019BC9F8143001212030C9F8101038
:10BE7000B8F1000FE3D0A8F2334808EB0003C0F19B
:10BE800035003B603060484603B0BDE8F083DDE933
:10BE90000013C0F1200203FA02F20A43C3400193E7
:10BEA000C9F81420C0E700BFF8B50E46144607468F
:10BEB00008B1836BBBB1636ED80702D4A38999051F
:10BEC00026D5A368013B002BA3600FDBF5B22368E6
:10BED0005A1C22601E70636EDA0702D4A3899B0588
:10BEE00011D52846F8BDF9F753FCE4E7A26993425F
:10BEF00002DBF5B20A2DEAD131463846224600F07F
:10BF000069FB0546E7E7A06DF9F7BEFE2846F8BDD8
:10BF1000A06DF9F7B7FED4E770B50D46084C114691
:10BF200006461A46284600232360F8F798FD431C6E
:10BF300000D070BD2368002BFBD0336070BD00BF04
:10BF4000AC1D00202DE9F04F924683B0002900F08F
:10BF5000A1800D4680460AF10B04FAF7ABF955F8BB
:10BF6000042C162C22F00306A5F108073ED8102455
:10BF70002146A2453FD88E4207EB060974DAC74B2B
:10BF80009868484500F0AA80D9F8040020F0010321
:10BF90004B445B68DB0740F18380D20734D55146C0
:10BFA0004046F9F783FE8246E0B155F8043C23F0A1
:10BFB00001033B44A0F10802934200F0F980321FD4
:10BFC000242A00F20781132A296800F2E68003463A
:10BFD0002A4619605168596092689A60294640461D
:10BFE000F9F7EAFC4046FAF76BF94FE024F0070452
:10BFF000002C2146BDDA4FF0000A0C235046C8F849
:10C00000003003B0BDE8F08F55F8083CA7EB030BF8
:10C01000DBF8042022F00302B3188B42BFDBDA46C0
:10C02000DBF80C105AF8080F321F242AC1600BEB02
:10C030000309886000F2C680132A296840F2C08094
:10C04000CBF808106968CBF80C101B2AA96800F21D
:10C05000D8800BF110020835116069685160A96839
:10C0600091601E465F4655467B68321B0F2A03F0DF
:10C07000010322D833437B60D9F8043043F0010335
:10C08000C9F804304046FAF71BF9AA46504603B0F7
:10C09000BDE8F08F114603B0BDE8F04FF9F706BEDA
:10C0A00020F0030033188B4261DBD9E902121E46EF
:10C0B000CA6007EB03099160D6E73919234342F0C0
:10C0C00001027B604A60D9F8043043F00103083173
:10C0D000C9F804304046F9F76FFCD3E7406820F018
:10C0E0000309B14404F11000814577DAD2073FF526
:10C0F00056AF55F8082CA7EB020BDBF8042022F012
:10C1000003029144484587DCDA46DBF80C105AF804
:10C11000080F321F242AC160886000F2A180132A10
:10C12000296840F29B80CBF808106968CBF80C10A6
:10C130001B2AA96800F29B800BF1100208351160E0
:10C1400069685160A96891600BEB0401A9EB0402D6
:10C1500042F0010299604A60DBF8043003F0010309
:10C160001C434046CBF80440FAF7AAF88EE7D30701
:10C170003FF515AF55F8083CA7EB030BDBF804209F
:10C1800022F00302104483198B42FFF645AFD9E930
:10C190000212DA46CA60916042E701606B68436050
:10C1A0001B2A3AD805F1080200F10803A96810E734
:10C1B00050F8043C23F003031E4407EB060953E741
:10C1C000524649E7294650461E465F46FFF7FEFAAB
:10C1D000554649E72946FFF7F9FAFFE62744A9EB58
:10C1E000040949F001029F607A6055F8043C03F0AD
:10C1F00001031C43404645F8044CFAF761F8AA468F
:10C2000044E7CBF81010E968CBF81410242A10D0BA
:10C2100029690BF1180210351EE7AB688360EB68E3
:10C22000C360242A10D005F1100200F1100329691F
:10C23000CFE62A69CBF818206A69CBF81C20A969D7
:10C240000BF12002183507E72B6903616B69436125
:10C25000A96905F1180200F11803BAE652466EE723
:10C26000294650460193FFF7B1FA019B6CE7CBF8E2
:10C270001010E968CBF81410242A04D029690BF1B6
:10C28000180210355BE72A69CBF818206A69CBF8E9
:10C290001C20A9690BF12002183550E7A40D0020DD
:10C2A00053EC102B70B5164E23F000410025B1421F
:10C2B0000446056021DC10EE106A0E431DD0B1F576
:10C2C000801F18460CDA1946002210EE100A0D4B9A
:10C2D000F4F752F96FF035050246084621F00041A7
:10C2E00020F0FF40091520F4E000A1F2FE3140F0FB
:10C2F0007F53294443F40013216043EC102B70BD9D
:10C30000FFFFEF7F00005043C9B200F00303002994
:10C3100043D07BB10378002B67D099423CD0431CBB
:10C3200005E013F8012B002A5DD08A4234D09A0729
:10C330001846F6D170B4046841EA012646EA06467A
:10C3400086EA0405A5F10133A4F1013223EA0503CD
:10C3500022EA0402134313F0803F0FD150F8044F38
:10C3600084EA0605A5F10132A4F1013322EA0502AF
:10C3700023EA0403134313F0803FEFD0037843B163
:10C38000994202D106E08B4204D010F8013F002B05
:10C39000F9D1184670BC704770475BB10378002B29
:10C3A000FAD0431C03E002780133002AF4D0990745
:10C3B0001846F8D10268A2F1013323EA020313F010
:10C3C000803F08D150F8042FA2F1013323EA020381
:10C3D00013F0803FF6D00378002BDDD010F8013F3A
:10C3E000002BFBD17047104670471846704700BFBE
:10C3F00040EA01039B0770B42AD1032A28D90C46CE
:10C400000346214654F8046BA6F1013525EA0605DA
:10C4100015F0803F06D1043A032A43F8046B214605
:10C42000EFD89AB10C781C70013A01333CB16AB173
:10C4300011F8014F03F8014B013A002CF7D12AB152
:10C440001A44002103F8011B9342FBD170BC7047D2
:10C450000346E6E72DE9F04F936883B09046002B42
:10C460006CD017688D6882460C460868083742E031
:10C47000A38913F4906F2DD0D4E9041505EB45057D
:10C48000A0EB010B05EBD575701C6D105844A8424C
:10C490002A4684BF05462A465B0536D511465046D6
:10C4A000F9F704FC00283AD05A4621690190F4F7C4
:10C4B0007DFCA289019B22F4906242F08002A2815D
:10C4C000A5EB0B0203EB0B00656123612060A2600A
:10C4D0003546B3465A464946FFF778F9D8F808304A
:10C4E000A2682068551B58449E1BA5602060C8F8B0
:10C4F00008601EB3083757E90296AB46002EF9D004
:10C50000AE42B5D23546B346E4E75046FFF71AFDD2
:10C5100003460028D4D121695046F9F74DFA0C237F
:10C52000CAF80030A389002243F040034FF0FF30E7
:10C53000A381C8E9012203B0BDE8F08F0020C8F84C
:10C54000040003B0BDE8F08F2DE9F84F4B6E9C045A
:10C5500092462DD59368126843B30E46074602F102
:10C56000080959E9025B5FEA9B0815D0043D0024E5
:10C5700001E0A0450ED0324655F8041F384600F0C1
:10C5800065F9431C04F10104F3D10023CAE9013326
:10C59000BDE8F88FDAF808302BF0030BA3EB0B03A0
:10C5A000CAF8083009F10809002BDAD10020ECE7BD
:10C5B000FEF7C0FE0023CAE90133BDE8F88F00BFD3
:10C5C00093680BB1FFF7C0BF10B4184653605DF815
:10C5D000044B7047F8B50D461446064610B1836B00
:10C5E000002B43D0B4F90C20A369A36091B20807D3
:10C5F0001BD52369CBB1EDB289042F4622D5226821
:10C600006169D31A994229DD0133A168501C0139AF
:10C61000A1602060157062699A422AD0A389DB0765
:10C6200001D50A2D25D03846F8BD21463046FDF704
:10C630003BFE20BBB4F90C20236991B2EDB2890412
:10C640002F46DCD4616E42F4005221F40051A281E5
:10C65000226861666169D31A9942D5DC2146304669
:10C66000F8F7D6FF58B922680123CEE7F9F790F81A
:10C67000B8E721463046F8F7CBFF0028D3D04FF07B
:10C68000FF37D0E72DE9F8432B4D0646286898463A
:10C690000F469146F9F7F6FA284B1C68D4F8483152
:10C6A000002B3DD05A681F2A0DDC02F1010C16BB8D
:10C6B0000232C3F804C0286843F82270F9F7E4FA9C
:10C6C0000020BDE8F8831E4B7BB34FF4C870F9F728
:10C6D000DDFA034648B3D4F848210021C0E900211F
:10C6E0004FF0010CC4F848010A46C0F88811C0F8A0
:10C6F0008C11002EDCD003EB82010124C1F888905C
:10C70000D3F8880194402043022EC3F88801C1F871
:10C710000881CDD1D3F88C110C43C3F88C41C7E705
:10C7200004F5A673C4F84831BCE72868F9F7ACFAF9
:10C730004FF0FF30C5E700BFB411002074CE0008F1
:10C740008D5C000810B502FB01F1F9F7AFFA044661
:10C75000D8B150F8042C22F00302043A242A1DD840
:10C76000132A14D900231B2AC0E900331BD9242A19
:10C77000C0E902330ABFC0E9043300F1100200F13E
:10C7800018020023C2E900339360204610BD024620
:10C790000023C2E900339360204610BD0021F9F761
:10C7A0003FFD204610BD00F10802F1E72DE9F047FA
:10C7B00082B0814688461446F9F740FA012803D131
:10C7C00008F1FF33FE2B33D9424604F15C0301A983
:10C7D000484600F093F8421C06462FD020B39DF83F
:10C7E00004C000250DF1040A09E023685A1C2260E8
:10C7F00083F800C00135B54216D215F80AC0A36807
:10C80000013B002BA360F0DAA769BB4261462246D8
:10C81000484602DBBCF10A0FE7D1FFF7DBFE431C01
:10C82000E8D102B0BDE8F087404602B0BDE8F0872D
:10C830005FFA88FC06468DF804C0D2E7A38943F06E
:10C840004003A38102B0BDE8F08700BF30B50546C4
:10C85000506EB2F90C30C007144683B09AB201D4BE
:10C8600090051CD5900406D4626E43F4005342F444
:10C870000052A381626628462246FFF797FF636E47
:10C88000DA07054602D4A3899B0502D5284603B0E2
:10C8900030BDA06DF9F7F8F9284603B030BDA06DA2
:10C8A0000191F9F7EFF9B4F90C3001999AB2D9E78F
:10C8B00038B50B46074C0546114618460023236041
:10C8C000F7F70AFD431C00D038BD2368002BFBD0CE
:10C8D0002B6038BDAC1D002038B5074C0023054641
:10C8E00008462360F8F7B3F8431C00D038BD23682E
:10C8F000002BFBD02B6038BDAC1D0020F0B5114CD7
:10C90000246885B00646646B1F4651B10E4D002C5D
:10C9100008BF2C46D4F8E040A047431C0CD005B01B
:10C92000F0BD094A002C08BF14460A46D4F8E0407E
:10C9300001A9A047431CF2D100228A233A60336048
:10C9400005B0F0BD0C080020380C0020F8B500BF81
:10C95000F8BC08BC9E467047F8B500BFF8BC08BCE0
:04C960009E46704738
:10C968000000000000000000010203040607080997
:10C97800000000000102030400000240000402401D
:10C988000008024000000000000000000000000055
:10C9980000000000000000000000000028CD000892
:10C9A80030CD000838CD000844CD000810CD00086F
:10C9B8001CCD0008DCCC0008E8CC0008F4CC00084A
:10C9C80000CD0008B4CC0008BCCC0008C4CC0008DA
:10C9D800D0CC00086CCD000800000000000000006A
:10C9E8009D3E0008A13E0008000000000000000075
:10C9F80000000000000000000000000078CD0008E2
:10CA080001000000FD3C00085D3D0008FD3D0008F8
:10CA1800593B0008393D000800000000B13D0008FE
:10CA280000000000000000000000000000100000EE
:10CA380032000000002000004B0000000030000021
:10CA48006E0000000040000086000000005000005A
:10CA58009600000000600000C800000000700000A0
:10CA68002C01000000800000580200000090000027
:10CA7800B004000000A000000807000000B000009B
:10CA88006009000000C00000C012000000D00000D3
:10CA98008025000000E00000004B000000F00000CE
:10CAA800009600000000010000E1000000100100F5
:10CAB80000C20100002001000084030000300100D2
:10CAC800000807000040010020A1070000500100F5
:10CAD80000CA08000060010000100E00007001008C
:10CAE80040420F00008001000094110000900100F6
:10CAF80060E3160000A0010080841E0000B0010061
:10CB0800A025260000C00100C0C62D0000D00100ED
:10CB1800E067350000E0010000093D00000000006A
:10CB2800FFFFFFFF583D25336420593D253364201E
:10CB3800517569743D5E512C5E58200049726A2017
:10CB4800286B696C657065733D51554954293A00E5
:10CB5800426569727420737A6F7665673A20257327
:10CB68002028686F73737A3D2564290A0000000045
:10CB780051554954000000002F6465762F75736184
:10CB88007274310048656C6C6F0000003120736866
:10CB98006F6F742067616D65000000003220766158
:10CBA8006C616D6900000000332072656164207358
:10CBB8007472696E67000000256320706F733D25ED
:10CBC80032642062756C6C733D253264207175691E
:10CBD800743D5E512C5E5820000000002D5E2D0033
:10CBE80020202000252B356420000000313135320B
:10CBF80030302C4E2C382C31000000002573256471
:10CC0800000000004950324E000000005025632EFD
:10CC18002564206465765B25645D2E257820726521
:10CC2800675B25642C253032785D3D203078256C93
:10CC3800780A00004146202020203D20256420302D
:10CC48007825780A000000004D6F646520203D209B
:10CC580025642025730A00004F74797065203D20F3
:10CC680025782025730A00005370656564203D20EF
:10CC780025642025730A00005075506420203D204B
:10CC880025642025730A0000696E6974203D2025FB
:10CC9800730A0000496E707574203D2025640A00EF
:10CCA8004F75747075743D2025640A004E6F507579
:10CCB8005064000055702D70756C6C00446F776E71
:10CCC8002D70756C6C000000526573657276656432
:10CCD800000000004C6F772032204D487A00000099
:10CCE8004D6564203235204D487A000046756C6CDD
:10CCF800203530204D487A00486967682031303047
:10CD0800204D487A00000000507573682D70756CCE
:10CD18006C0000004F70656E2D647261696E0000D2
:10CD2800496E7075740000004F757470757400005A
:10CD380046756E6374696F6E00000000416E616C29
:10CD48006F670000504139005042370050413200AF
:10CD580050413300504438005044390050433600A5
:10CD6800504337002F6465762F6E756C6C00000099
:10CD78002F6465762F757361727400007700000068
:10CD8800082008001B5B3244000000001B5B314494
:10CD9800000000001B5B7300202000001B5B750077
:10CDA8001B5B31471B5B324B000000007474790039
:10CDB8002C3B2E7C2F2000002F6465762F7474790D
:10CDC8004D2564004F70656E3A2025730000000001
:10CDD8007463666C7573683A2025730A0000000056
:10CDE8007463676574617474723A2025730A00006D
:10CDF8007463736574617474720000001B5B25644E
:10CE0800440000001B5B25644300000025732000DC
:10CE18001B5B2564410000001B5B25644200000089
:10CE28001B5B25643B256448000000001B5B324AFD
:10CE3800000000001B5B25646D0000001B5B3F3297
:10CE4800356C00001B5B3F32356800001B5B313BD3
:10CE580032277A001B5B3F39680000001B5B3F39B3
:10CE68006C0000001B5B303B30277A001008002064
:10CE7800504F5349580000002E0000000A000000DF
:10CE8800494E4600696E66004E414E006E616E0066
:10CE98003031323334353637383961626364656628
:10CEA80000000000303132333435363738394142EA
:10CEB8004344454600000000286E756C6C2900004C
:10CEC80030000000202020202020202020202020AA
:10CED800202020203030303030303030303030308A
:10CEE80030303030202020202020202020202020FA
:10CEF800202020203030303030303030303030306A
:10CF080030303030002020202020202020202828E9
:10CF180028282820202020202020202020202020F1
:10CF28002020202020881010101010101010101031
:10CF38001010101010040404040404040404041061
:10CF480010101010101041414141414101010101EF
:10CF580001010101010101010101010101010101B9
:10CF680010101010101042424242424202020202C5
:10CF78000202020202020202020202020202020289
:10CF88001010101020000000000000000000000039
:10CF98000000000000000000000000000000000089
:10CFA8000000000000000000000000000000000079
:10CFB8000000000000000000000000000000000069
:10CFC8000000000000000000000000000000000059
:10CFD8000000000000000000000000000000000049
:10CFE8000000000000000000000000000000000039
:10CFF8000000000000000000000000000000000029
:10D008000000000000000000496E66696E697479CE
:10D01800000000004E614E000080E03779C34143B4
:10D02800176E05B5B5B89346F5F93FE9034F384D86
:10D03800321D30F94877825A3CBF737FDD4F157532
:10D04800000000000000F03F000000000000244045
:10D0580000000000000059400000000000408F4020
:10D06800000000000088C34000000000006AF8408B
:10D078000000000080842E4100000000D0126341AF
:10D088000000000084D797410000000065CDCD4125
:10D09800000000205FA00242000000E87648374206
:10D0A800000000A2941A6D42000040E59C30A242A4
:10D0B8000000901EC4BCD64200003426F56B0C4319
:10D0C8000080E03779C3414300A0D88557347643C0
:10D0D80000C84E676DC1AB43003D9160E458E14321
:10D0E800408CB5781DAF154450EFE2D6E41A4B4496
:10D0F80092D54D06CFF08044F64AE1C7022DB544DB
:10D10800B49DD9794378EA4405000000190000006D
:04D118007D00000096
:08D11C00C039FF7F0100000093
:08D1240075A30008E5010008F5
:04D12C00C101000835
:10D1300001000000100000000024F4000C000000BA
:10D1400028000000010000000A00000001000000AB
:10D1500000F00000000F00000000000000000000D0
:10D1600000000000000000000000000000000000BF
:10D1700000000000000000000000000000000000AF
:10D18000000000000000000000000000000000009F
:10D19000000000000000000000000000000000008F
:10D1A000000000000000000000000000000000007F
:10D1B000000000000000000000000000000000006F
:10D1C000000000000000000000000000000000005F
:10D1D000000000000000000000000000000000004F
:10D1E000000000000000000000000000000000003F
:10D1F000000000000000000000000000000000002F
:10D20000000000000000000000000000000000001E
:10D21000000000000000000000000000000000000E
:10D2200000000000000000000000000000000000FE
:10D23000000000000000000000100140000000009D
:10D2400000000000000000000000000000000000DE
:10D2500000000000000000000000000000000000CE
:10D2600000000000000000000000000000000000BE
:10D2700000000000000000004CCD000850CD000868
:10D280000000000000000000072500000000000072
:10D29000000000000000000000000000000000008E
:10D2A000000000000000000000000000000000007E
:10D2B000000000000000000000000000000000006E
:10D2C000000000000000000000000000000000005E
:10D2D000000000000000000000000000000000004E
:10D2E000000000000000000000000000000000003E
:10D2F000000000000000000000000000000000002E
:10D30000000000000000000000000000000000001D
:10D310000000000000000000004400400000000089
:10D3200000000000000000000000000000000000FD
:10D3300000000000000000000000000000000000ED
:10D3400000000000000000000000000000000000DD
:10D35000000000000000000054CD000858CD000877
:10D360000000000000000000072600000000000090
:10D3700000000000000000000000000000000000AD
:10D38000000000000000000000000000000000009D
:10D39000000000000000000000000000000000008D
:10D3A000000000000000000000000000000000007D
:10D3B000000000000000000000000000000000006D
:10D3C000000000000000000000000000000000005D
:10D3D000000000000000000000000000000000004D
:10D3E000000000000000000000000000000000003D
:10D3F000000000000000000000000000000000002D
:10D40000000000000000000000000000000000001C
:10D41000000000000000000000000000000000000C
:10D4200000000000000000000000000000000000FC
:10D4300000000000000000005CCD000860CD000886
:10D4400000000000000000000000000000000000DC
:10D4500000000000000000000000000000000000CC
:10D4600000000000000000000000000000000000BC
:10D4700000000000000000000000000000000000AC
:10D690000000000000000000001401400000000035
:10D6A000000000000000000000000000000000007A
:10D6B000000000000000000000000000000000006A
:10D6C000000000000000000000000000000000005A
:10D6D000000000000000000064CD000868CD0008D4
:10D6E00000000000000000000847000000000000EB
:10D6F000000000000000000000000000000000002A
:10D700000000000000000000000000000000000019
:10D710000000000000000000000000000000000009
:10D7200000000000000000000000000000000000F9
:10D9300000000000000000000100000010080020AE
:10D9400000000000FC0A0020640B0020CC0B00202B
:10D9500000000000000000000000000000000000C7
:10D9600000000000000000000000000000000000B7
:10D9700000000000000000000000000000000000A7
:10D980000000000000000000000000000000000097
:10D990000000000000000000000000000000000087
:10D9A0000000000000000000000000000000000077
:10D9B0000000000000000000000000000000000067
:10D9C0000000000000000000000000000000000057
:10D9D0000000000000000000000000000000000047
:10D9E0000000000000000000010000000000000036
:10D9F0000E33CDAB34126DE6ECDE05000B000000FB
:10DA00000000000000000000000000000000000016
:10DA10000000000000000000000000000000000006
:10DA200000000000000000000000000000000000F6
:10DA300000000000000000000000000000000000E6
:10DD60000000000000000000430000000000000070
:10DD700000000000000000000000000000000000A3
:10DD80000000000000000000430000000000000050
:10DD90000000000000000000000000000000000083
:10DDA0000000000000000000430000000000000030
:10DDB0000000000000000000000000000000000063
:10DDC0000000000000000000430000000000000010
:10DDD0000000000000000000000000000000000043
:10DDE00000000000000000004300000000000000F0
:10DDF0000000000000000000000000000000000023
:10DE000000000000000000004300000000000000CF
:10DE10000000000000000000000000000000000002
:10DE200000000000000000004300000000000000AF
:10DE300000000000000000000000000000000000E2
:10DE4000000000000000000061A20008F561000869
:10DE5000000000000CCF000880CE000874CB000842
:10DE600074CB000874CB000874CB000874CB000896
:10DE700074CB000874CB000874CB000874CB000886
:10DE8000FFFFFFFFFFFFFFFFFFFFFFFFFFFF0000A0
:10DE90000100415343494900000000000000000018
:10DEA0000000000000000000000000000000000072
:10DEB00000004153434949000000000000000000F9
:10DEC0000000000000000000000000000000000052
:10DED000000000000000000000000000A40D002071
:10DEE000A40D0020AC0D0020AC0D0020B40D0020CE
:10DEF000B40D0020BC0D0020BC0D0020C40D00207E
:10DF0000C40D0020CC0D0020CC0D0020D40D00202D
:10DF1000D40D0020DC0D0020DC0D0020E40D0020DD
:10DF2000E40D0020EC0D0020EC0D0020F40D00208D
:10DF3000F40D0020FC0D0020FC0D0020040E00203C
:10DF4000040E00200C0E00200C0E0020140E0020E9
:10DF5000140E00201C0E00201C0E0020240E002099
:10DF6000240E00202C0E00202C0E0020340E002049
:10DF7000340E00203C0E00203C0E0020440E0020F9
:10DF8000440E00204C0E00204C0E0020540E0020A9
:10DF9000540E00205C0E00205C0E0020640E002059
:10DFA000640E00206C0E00206C0E0020740E002009
:10DFB000740E00207C0E00207C0E0020840E0020B9
:10DFC000840E00208C0E00208C0E0020940E002069
:10DFD000940E00209C0E00209C0E0020A40E002019
:10DFE000A40E0020AC0E0020AC0E0020B40E0020C9
:10DFF000B40E0020BC0E0020BC0E0020C40E002079
:10E00000C40E0020CC0E0020CC0E0020D40E002028
:10E01000D40E0020DC0E0020DC0E0020E40E0020D8
:10E02000E40E0020EC0E0020EC0E0020F40E002088
:10E03000F40E0020FC0E0020FC0E0020040F002037
:10E04000040F00200C0F00200C0F0020140F0020E4
:10E05000140F00201C0F00201C0F0020240F002094
:10E06000240F00202C0F00202C0F0020340F002044
:10E07000340F00203C0F00203C0F0020440F0020F4
:10E08000440F00204C0F00204C0F0020540F0020A4
:10E09000540F00205C0F00205C0F0020640F002054
:10E0A000640F00206C0F00206C0F0020740F002004
:10E0B000740F00207C0F00207C0F0020840F0020B4
:10E0C000840F00208C0F00208C0F0020940F002064
:10E0D000940F00209C0F00209C0F0020A40F002014
:10E0E000A40F0020AC0F0020AC0F0020B40F0020C4
:10E0F000B40F0020BC0F0020BC0F0020C40F002074
:10E10000C40F0020CC0F0020CC0F0020D40F002023
:10E11000D40F0020DC0F0020DC0F0020E40F0020D3
:10E12000E40F0020EC0F0020EC0F0020F40F002083
:10E13000F40F0020FC0F0020FC0F00200410002032
:10E14000041000200C1000200C10002014100020DF
:10E15000141000201C1000201C100020241000208F
:10E16000241000202C1000202C100020341000203F
:10E17000341000203C1000203C10002044100020EF
:10E18000441000204C1000204C100020541000209F
:10E19000541000205C1000205C100020641000204F
:10E1A000641000206C1000206C10002074100020FF
:10E1B000741000207C1000207C10002084100020AF
:10E1C000841000208C1000208C100020941000205F
:10E1D000941000209C1000209C100020A41000200F
:10E1E000A4100020AC100020AC100020B4100020BF
:10E1F000B4100020BC100020BC100020C41000206F
:10E20000C4100020CC100020CC100020D41000201E
:10E21000D4100020DC100020DC100020E4100020CE
:10E22000E4100020EC100020EC100020F41000207E
:10E23000F4100020FC100020FC100020041100202D
:10E24000041100200C1100200C11002014110020DA
:10E25000141100201C1100201C110020241100208A
:10E26000241100202C1100202C110020341100203A
:10E27000341100203C1100203C11002044110020EA
:10E28000441100204C1100204C110020541100209A
:10E29000541100205C1100205C110020641100204A
:10E2A000641100206C1100206C11002074110020FA
:10E2B000741100207C1100207C11002084110020AA
:10E2C000841100208C1100208C110020941100205A
:10E2D000941100209C1100209C110020FFFFFFFFE3
:08E2E00000000200881D00206F
:04000005080052C1DC
:00000001FF
